:100000000C946D110C949E110C949E110C949E11E5
:100010000C949E110C949E110C949E110C949E11A4
:100020000C949E110C949E110C949E110C949E1194
:100030000C949E110C94BFB10C949E110C949E11C3
:100040000C949E110C944B630C949E110C949E1175
:100050000C949E110C949E110C94D1730C94C1AB12
:100060000C949E110C94331E0C949E110C949E11B2
:100070000C949E110C949E110C949E110C949E1144
:100080000C949E110C949E110C949E110C949E1134
:100090000C949E110C949E110C949E110C9481A2B0
:1000A0000C949E110C949E110C949E110C949E1114
:1000B0000C949E110C949E110C949E110C949E1104
:1000C0000C949E110C949E110C949E110C949E11F4
:1000D0000C949E110C949E110C949E110C949E11E4
:1000E0000C949E1148745774737482749C74AB742E
:1000F000C574C97446A563A565A571A577A57AA53C
:1001000084A5E5ACEAACEFACF9AC03AD7CAD0DADCC
:1001100015AD1DAD27AD31AD3BAD4AAD54AD7CAD98
:100120005EAD68AD72AD9EADA1AD90AD94AD9AAD32
:10013000D8ADA5ADA9ADAFADB3ADB7ADBDADC1AD9A
:10014000C5ADD8ADCBADCFADD3AD084AD73B3BCED7
:10015000016E84BCBFFDC12F3D6C74319ABD5683C6
:100160003DDA3D00C77F11BED9E4BB4C3E916BAA7E
:10017000AABE000000803F05A84CCDB2D44EB938CD
:1001800036A9020C50B9918688083CA6AAAA2ABEB4
:10019000000000803F004D383420582059205A205C
:1001A00045004D3234004D323320257300617574A3
:1001B0006F25692E67006572726F7220777269749D
:1001C000696E6720746F2066696C65004E6F7420DD
:1001D0005344207072696E74696E67002F00534437
:1001E000207072696E74696E672062797465200090
:1001F0002E0044656C6574696F6E206661696C657C
:10020000642C2046696C653A200046696C65206460
:10021000656C657465643A002E006F70656E2066CB
:1002200061696C65642C2046696C653A20005772E0
:100230006974696E6720746F2066696C653A200086
:100240002E006F70656E206661696C65642C2046B7
:10025000696C653A20002E006F70656E20666169DA
:100260006C65642C2046696C653A200046696C65B3
:100270002073656C6563746564002053697A653A20
:10028000200046696C65206F70656E65643A2000D9
:100290002E006F70656E206661696C65642C204667
:1002A000696C653A200053442063617264206F6B6F
:1002B000006F70656E526F6F74206661696C656463
:1002C00000766F6C756D652E696E69742066616964
:1002D0006C656400534420696E6974206661696CC2
:1002E000006563686F3A004572726F723A00486148
:1002F0007264636F6465642044656661756C742024
:1003000053657474696E6773204C6F616465640033
:1003100053746F7265642073657474696E677320BB
:100320007265747269657665640053657474696E8C
:1003300067732053746F726564006563686F3A0079
:100340004B494C4C45442E20005072696E746572C6
:100350002068616C7465642E206B696C6C282920A0
:1003600063616C6C656421006F6B00526573656E30
:10037000643A20002200556E6B6E6F776E20636FBB
:100380006D6D616E643A202200486F74656E642062
:100390006F6666736574733A007A5F6D696E3A20B2
:1003A00000795F6D696E3A2000785F6D696E3A2062
:1003B000005A3A00593A0020436F756E7420583A3B
:1003C00000453A005A3A00593A00583A0046495214
:1003D0004D574152455F4E414D453A4D54315F3383
:1003E000445072696E7465725F50524F4752414D6E
:1003F0002056455253494F4E3A312E3832204558F7
:100400005452554445525F434F554E543A32204D55
:10041000414348494E455F545950453A52657052E0
:1004200061702020576562736974653A68747470EE
:100430003A2F2F7777772E6D756C746F6F2E636FF1
:100440006D200A0042656420646F6E652E002042B4
:100450003A002054313A0054303A00426564204852
:10046000656174696E672E0048656174696E672006
:10047000646F6E652E0020573A002054313A0054C4
:10048000303A0048656174696E672E2E2E00204256
:10049000403A0020403A00202F0020423A00202F0E
:1004A000002054313A00202F006F6B2054303A0066
:1004B0002569206D696E2C202569207365630045D0
:1004C0006E642066696C65206C69737400426567B0
:1004D000696E2066696C65206C697374004E6F20CC
:1004E0006D6F76652E005072696E74696E67202E8E
:1004F0002E2E005761697420666F722075736572C5
:100500002E2E2E004D303500536C6565702E2E2E2C
:100510000046696E69736865642E00446F6E6520DD
:100520007072696E74696E672066696C6500473326
:1005300032310053544F505045442E2000507269C0
:100540006E7465722073746F707065642064756575
:1005500020746F206572726F72732E204669782046
:10056000746865206572726F7220616E64207573A5
:1005700065204D39393920746F207265737461724A
:10058000742E202854656D706572617475726520D3
:1005900069732072657365742E20536574206974C5
:1005A0002061667465722072657374617274696E1D
:1005B0006729006F6B004E6F204C696E65204E7589
:1005C0006D626572207769746820636865636B7318
:1005D000756D2C204C617374204C696E653A200057
:1005E0004E6F20436865636B73756D20776974681F
:1005F000206C696E65206E756D6265722C204C6191
:100600007374204C696E653A2000636865636B7390
:10061000756D206D69736D617463682C204C617316
:1006200074204C696E653A20004C696E65204E75E9
:100630006D626572206973206E6F74204C617374F3
:10064000204C696E65204E756D6265722B312C20D1
:100650004C617374204C696E653A20004D31313025
:1006600000446F6E6520736176696E672066696C01
:10067000652E006F6B004D3239002020506C616E8A
:100680006E657242756666657242797465733A206A
:10069000002046726565204D656D6F72793A2000C5
:1006A0004E6F76202035203230313600436F6D702A
:1006B000696C65643A20006D756C746F6F00207C06
:1006C00020417574686F723A20004E6F7620203595
:1006D00020323031362030393A30363A3238002044
:1006E0004C61737420557064617465643A20004DE8
:1006F00054310020536F66747761726520526573C0
:10070000657400205761746368646F672052657375
:100710006574002042726F776E206F757420526589
:10072000736574002045787465726E616C20526543
:1007300073657400506F77657255700073746172E1
:1007400074002200656E717565696E672022002253
:1007500000656E717565696E67202200FFFFFF00FE
:1007600000A0400000A0400000803F0000CD4300FA
:1007700000C8430000C84300000000000000000063
:100780000000000000CD430000C8430000C8430043
:1007900000000000000000000000006563686F3A80
:1007A000004572726F723A0020746F6F206C6F6E2A
:1007B0006720657874727573696F6E2070726576E4
:1007C000656E7465640020636F6C64206578747274
:1007D0007573696F6E2070726576656E74656400FE
:1007E0006563686F3A007C3C3E5E2B3D3F2F5B5D4E
:1007F0003B2C2A225C00656E6473746F70732068F2
:1008000069743A205A00205A3A00656E6473746F16
:100810007073206869743A20590020593A00656E57
:100820006473746F7073206869743A20580020589C
:100830003A00656E6473746F7073206869743A204F
:100840000024F4D43050C38E20C2A24017828B7093
:1008500011127A910D816CD90AA861E108C7586616
:1008600007615143061E4B5D05C145A7041A41119E
:1008700004093D9803713931034036DB0265339139
:1008800002D4305402802E1D02632CEE01752AC55D
:1008900001B028A001102781018F2564012B244B72
:1008A00001E0223401AC211F018D200D01801FFCCD
:1008B00000841EED00971DDF00B81CD200E61BC6A9
:1008C00000201BBC00641AB200B219A8000A19A0CB
:1008D000006A189900D117910040178B00B5168453
:1008E0000031167E00B31579003A157300C7146FF6
:1008F0000058146A00EE1366008813630025135E27
:1009000000C7125B006C12570015125400C1115140
:100910000070114F0021114B00D61049008D104777
:10092000004610440002104200C00F4000800F3EFD
:1009300000420F3C00060F3B00CB0E3800930E37F1
:10094000005C0E3500270E3400F30D3200C10D316E
:1009500000900D3000600D2E00320D2D00050D2C85
:1009600000D90C2B00AE0C2900850C29005C0C274B
:1009700000350C27000E0C2600E80B2400C40B24C5
:1009800000A00B23007D0B23005A0B2100390B2103
:1009900000180B2000F80A1F00D90A1E00BB0A1E0F
:1009A000009D0A1D00800A1D00630A1C00470A1BE7
:1009B000002C0A1B00110A1A00F7091A00DD091998
:1009C00000C4091900AB091900920917007B091826
:1009D00000630917004C0916003609160020091695
:1009E000000A091500F5081500E0081400CC0814E9
:1009F00000B8081400A4081400900813007D081221
:100A0000006B081300580812004608120034081141
:100A100000230811001208110001081100F007104E
:100A200000E0071000D0071000C0071000B0070F4B
:100A300000A107100091070E0083070F0074070F35
:100A40000065070E0057070E0049070E003B070D13
:100A5000002E070E0020070D0013070D0006070DDE
:100A600000F9060C00ED060D00E0060C00D4060CA3
:100A700000C8060C00BC060C00B0060C00A4060B57
:100A80000099060C008D060B0082060B0077060B02
:100A9000006C060B0061060A0057060B004C060AA4
:100AA0000042060A0038060A002E060A0024060A3A
:100AB000001A060A001006090007060A00FD0509CB
:100AC00000F4050900EB050900E2050900D9050954
:100AD00000D0050900C7050900BE050900B50508D5
:100AE00000AD050800A50509009C0508009405084F
:100AF000008C050800840508007C050800740508C2
:100B0000006C050700650508005D0507005605082F
:100B1000004E050700470507004005080038050797
:100B200000310507002A050700230507001C0506FC
:100B300000160507000F0507000805060002050757
:100B400000FB040600F5040700EE040600E80406B6
:100B500000E2040700DB040600D5040600CF04060B
:100B600000C9040600C3040600BD040600B704065D
:100B700000B1040500AC040600A6040600A00405AC
:100B8000009B04060095040500900406008A0405F5
:100B90000085040500800406007A0405007504053C
:100BA00000700405006B040500660405006104057F
:100BB000005C04050057040500520405004D0405BF
:100BC0000048040500430405003E0404003A0405FF
:100BD0000035040500300404002C0405002704043B
:100BE00000230405001E0404001A04040016040572
:100BF00000110404000D04040009040500040404A9
:100C00000000040400FC030400F8030400F40304DF
:100C100000F0030400EC030400E8030400E4030410
:100C200000E0030400DC030400D8030400D4030440
:100C300000D0030400CC030400C8030300C5030371
:100C40000024F404D9201BC40C5C0E9804C4095F72
:100C50000265077101F405F900FB04B3004804873D
:100C600000C10369005803550003034500BE023A62
:100C7000008402310053022A0029022500040220C8
:100C800000E4011C00C8011900AF0117009801140D
:100C90000084011300710110006101100051010E68
:100CA0000043010D0036010B002B010B0020010B4E
:100CB00000150109000C01090003010800FB0008F0
:100CC00000F3000800EB000700E4000600DE000669
:100CD00000D8000600D2000600CC000500C70005C1
:100CE00000C2000500BD000400B9000400B5000406
:100CF00000B1000400AD000400A9000400A5000339
:100D000000A20003009F0004009B00030098000362
:100D1000009500020093000300900003008D000284
:100D2000008B00030088000200860002008400039C
:100D300000810002007F0002007D0002007B0002B3
:100D400000790002007700010076000200740002C2
:100D50000072000100710002006F0002006D0001CE
:100D6000006C0002006A00010069000200670001D7
:100D700000660001006500010064000200620001DD
:100D80000061000100600001005F0002005D0001E1
:100D9000005C0001005B0001005A000100590001E5
:100DA00000580001005700010056000100550001E5
:100DB00000540001005300000053000100520001E4
:100DC0000051000100500001004F0001004E0000E2
:100DD000004E0001004D0001004C0001004B0000DE
:100DE000004B0001004A00010049000100480000DA
:100DF00000480001004700010046000000460001D5
:100E000000450000004500010044000100430000CF
:100E100000430001004200000042000100410000C8
:100E20000041000100400001003F0000003F0001C0
:100E3000003E0000003E0001003D0000003D0001BA
:100E4000003C0000003C0000003C0001003B0000B2
:100E5000003B0001003A0000003A000100390000A8
:100E6000003900010038000000380000003800019F
:100E70000037000000370001003600000036000097
:100E8000003600010035000000350000003500018B
:100E90000034000000340000003400010033000082
:100EA0000033000000330001003200000032000077
:100EB000003200010031000000310000003100016B
:100EC000003000000030000000300001002F000062
:100ED000002F0000002F0000002F0001002E000056
:100EE000002E0000002E0001002D0000002D00004B
:100EF000002D0000002D0001002C0000002C00003F
:100F0000002C0000002C0001002B0000002B000032
:100F1000002B0000002B0001002A0000002A000026
:100F2000002A0000002A000100290000002900001A
:100F3000002900000029000000290001002800000D
:100F40000028000000280000002800000028000100
:100F500000270000002700000027000000270000F5
:100F600000270001002600000026000000260000E7
:100F700000260000002600010025000000250000DA
:100F800000250000002500000025000000250001CC
:100F900000240000002400000024000000240000C1
:100FA00000240001002300000023000000230000B3
:100FB00000230000002300000023000000230001A4
:100FC0000022000000220000002200000022000099
:100FD000002200000022000100210000002100008A
:100FE000002100000021000000210000002100007D
:100FF000002100010020000000200000002000006F
:101000000020000000200000002000000020000060
:1010100000200001001F0000001F0000001F000052
:10102000001F0000001F0000001F0000001F000143
:10103000001E0000001E0000001E0000001E000038
:10104000006563686F3A00202D20496E76616C69F7
:1010500064206578747275646572206E756D626562
:1010600072202100504944204175746F74756E657B
:101070002066696E6973686564202120506C616325
:101080006520746865204B702C204B6920616E646C
:10109000204B6420636F6E7374616E747320696E8D
:1010A0002074686520636F6E666967757261746924
:1010B0006F6E2E6800504944204175746F74756ED0
:1010C00065206661696C6564212074696D656F7562
:1010D000740020403A006F6B20543A006F6B20423E
:1010E0003A00504944204175746F74756E652066EE
:1010F00061696C6564212054656D706572617475F9
:10110000726520746F206869676800204B643A201C
:1011100000204B693A2000204B703A200020436C9D
:10112000617369632050494420002054753A2000BF
:10113000204B753A2000206D61783A2000206D69BF
:101140006E3A200020643A200020626961733A20E0
:10115000004572726F723A00A0007201B0006D011A
:10116000B0006801C0006301D0005E01D0005901E9
:10117000E0005401F0004F0100014A011001450157
:101180002001400130013B01400136016001310185
:1011900070012C0190012701B0012201C0011D0145
:1011A000F00118011002130130020E016002090162
:1011B00090020401C002FF000003FA004003F500A2
:1011C0008003F000D003EB002004E6007004E1008F
:1011D000E004DC004005D700C005D2004006CD0089
:1011E000D006C8008007C3003008BE00F008B90070
:1011F000C009B400B00AAF00B00BAA00D00CA50023
:10120000000EA000500F9B00C010960050129100DD
:1012100000148C00C0158700B0178200B0197D0043
:10122000D01B7800001E730040206E0090226900E1
:10123000F024640040275F0090295A00E02B5500FD
:10124000102E500020304B0010324600E033410099
:1012500090353C001037370070383200A0392D002F
:10126000B03A2800A03B2300603C1E00103D19004E
:10127000903D1400103E0F00703E0A00C03E050075
:10128000003F0000436172642072656D6F76656493
:10129000004361726420696E736572746564004D09
:1012A0003234004D3233202573002573002573003E
:1012B0005175697400517569740051756974004EF7
:1012C0006578742050616765002E2E00507265208D
:1012D00050616765004D61696E00506175736564AA
:1012E0002E004D6174657269616C206973206F75A1
:1012F000742E002D2D3A2D2D002320002320004D8B
:1013000038340046494E495348004241434B004E51
:1013100045585400466C6F7700466C6F7700466105
:101320006E2073706565640046616E20737065653C
:1013300064004E6F7A7A6C6532004E6F7A7A6C6513
:1013400032004E6F7A7A6C65004E6F7A7A6C650067
:101350005370656564005370656564004D61696E26
:101360000053746F7265206D656D6F7279004E6FFA
:101370007A7A6C65004E6F7A7A6C650046616E20F1
:1013800073706565640046616E2073706565640006
:1013900054656D70657261747572650053746F7217
:1013A00065206D656D6F7279004E6F7A7A6C65009D
:1013B0004E6F7A7A6C650046616E20737065656465
:1013C0000046616E2073706565640054656D7065DC
:1013D0007261747572650041626F75742075730077
:1013E00052657365742044656661756C7400507253
:1013F00065686561742041425320436F6E660050FA
:1014000072656865617420504C4120436F6E6600C0
:1014100046616E2073706565640046616E2073706E
:10142000656564004F6666004F6E20004F6666007B
:101430004F6E2000456E61626C65204657004C611E
:1014400073657220456E67726176696E67204D6FB5
:10145000646500436F6F6C646F776E0050726568EF
:101460006561742041425300507265686561742063
:10147000504C41004D6F76652041786973004732CA
:1014800038205900486F6D65205900473238205880
:1014900000486F6D65205800473238205A00486F69
:1014A0006D65205A004D38340044697361626C6583
:1014B000205374657070657273004D61696E0047EA
:1014C000323800526573756D65205072696E740014
:1014D000473332320046696E69736865642E004D89
:1014E0003834004D383420582059205A20450025E2
:1014F000730025732573004D6F766520302E316D96
:101500006D004D6F766520316D6D004D6F766520F5
:1015100031306D6D00507265706172650058005910
:1015200000457874727564657200457874727564EC
:101530006572004D6F7665205A004D6F76652059B3
:10154000004D6F76652058004D6F766520417869B3
:1015500073005A004D3035004D30330041626F75D5
:101560007420757300536176652064697374616ECD
:10157000636500466F63616C2064697374616E63B8
:101580006500466F63616C2064697374616E6365A6
:10159000005475726E206F6666204C617365720030
:1015A0005475726E206F6E204C61736572004D6FC2
:1015B0007665205A00473238205A3000486F6D65F2
:1015C000205A004C61736572204D656E75004E6F38
:1015D000204361726400456E6772617665206672B1
:1015E0006F6D20534420636172640053746F7020E8
:1015F000456E67726176696E6700526573756D65D9
:1016000020456E67726176696E670050617573651B
:1016100020456E67726176696E6700473130310030
:10162000536574206261736520706F696E74004F3A
:10163000626A65637420686569676874004F626AEE
:101640006563742068656967687400466F63616CE0
:101650002053657474696E67730053706565640028
:101660005370656564004E6F204361726400507270
:10167000696E742066726F6D2053442063617264DA
:101680000053746F70205072696E740052657375E8
:101690006D65205072696E740050617573652050DD
:1016A00072696E7400506C617465204C6576656C6F
:1016B000696E670047323800486F6D6520616C6C59
:1016C0000050726570617265004F6666004F6E2053
:1016D000004F6666004F6E2000456E61626C6520AB
:1016E00046570054756E65005374617475732073AA
:1016F000637265656E00000B1000000D00000000B5
:101700003039000D000D00090D1A0B0000FF80FF9D
:1017100080C180C180C180C180C180C180C180C1C1
:1017200080C180FF80FF80040D0D060000F0F030C6
:1017300030303030303030303030090D1A0A00008F
:10174000FF80FF80018001800180FF80FF80C0005A
:10175000C000C000C000FF80FF80090D1A0B000010
:10176000FF80FF80018001800180FF80FF80018079
:10177000018001800180FF80FF800B0D1A0D0000A9
:101780000180038007800D80198031806180FFE037
:10179000FFE00180018001800180090D1A0A00002C
:1017A000FF80FF80C000C000C000FF80FF8001807C
:1017B000018001800180FF80FF80090D1A0A00006E
:1017C000FF80FF80C000C000C000FF80FF80C1809C
:1017D000C180C180C180FF80FF80090D1A0A00000E
:1017E000FF80FF80018001800180018001800180F5
:1017F00001800180018001800180090D1A0B000029
:10180000FF80FF80C180C180C180FF80FF80C180D8
:10181000C180C180C180FF80FF80090D1A0B0000CC
:10182000FF80FF80C180C180C180FF80FF80018078
:10183000018001800180FF80FF8000060900000711
:1018400001850308207FFE07FE07FE00000005005B
:101850000001070702000080808080800080030272
:1018600002040005A0A0060707060000C0D8242037
:101870002024180507070600002078A07028F02013
:1018800007070708000042A44810244A84060505FB
:1018900007000210387C10F0FF0307070400002047
:1018A0004080808040200307070400008040202003
:1018B000204080050505060000A870F870A8050501
:1018C000050600002020F820200203030300FF404B
:1018D0004080030101040002E001020202000080D6
:1018E00080050707060000080810204080800507D3
:1018F00007060000F88888888888F8020707030030
:1019000000C0404040404040050707060000F8087E
:1019100008F88080F8050707060000F80808F808AE
:1019200008F806070707000008182848FC080805FB
:101930000707060000F88080F80808F80507070682
:101940000000F88080F88888F8050707060000F88E
:10195000080808080808050707060000F88888F83E
:101960008888F8050707060000F88888F80808F84E
:10197000010505020000808000808002050503004B
:10198000FF400040408005050506000018608060AB
:1019900018040303050001F000F00505050600002A
:1019A000C0300830C0050707070100708808102004
:1019B00000200807070900003C4299A999423C050C
:1019C0000707060000205088F88888880507070662
:1019D0000000F08888F08888F0050707060000708E
:1019E000888080808870050707060000F088888856
:1019F0008888F0040707050000F08080F08080F000
:101A0000040707050000F08080F08080800507074C
:101A1000060000708880B8888870050707060000F7
:101A2000888888F8888888010707020000808080FD
:101A300080808080050707060000080808080888DD
:101A4000700507070600008890A0C0A090880407D2
:101A500007050000808080808080F007070708006D
:101A60000082C6AA92828282050707060000888843
:101A7000C8A89888880507070600007088888888A5
:101A80008870050707060000F08888F080808005D0
:101A900008080600FF70888888888870080507078E
:101AA000060000F08888F08888880507070600008F
:101AB00070888070088870050707060000F82020ED
:101AC000202020200507070600008888888888884D
:101AD0007005070706000088888888885020070757
:101AE000070800008292929292926C050707060006
:101AF00000888850205088880507070600008888DD
:101B00005020202020050707060000F8081020407C
:101B100080F8020707030000C08080808080C00535
:101B2000070707010080804020100808020707030C
:101B30000000C04040404040C0FF050101060000D9
:101B4000F8FF050505060000700878887805070786
:101B50000600008080F0888888F0050505060000F2
:101B60007088808870050707060000080878888854
:101B700088780505050600007088F8807803070757
:101B8000030000608080C08080800507070600FE9B
:101B9000788888887808300507070600008080F07C
:101BA0008888888801070702000080008080808084
:101BB000800209090300FE40004040404040408050
:101BC0000507070600008890A0C0A09088010707BD
:101BD000020000808080808080800705050800006A
:101BE000EC92929292050505060000F0888888889C
:101BF000050505060000708888887005070706003F
:101C0000FEF0888888F080800507070600FE788847
:101C10008888780808040505050000B0C080808029
:101C200005050506000078807008F003070704002A
:101C3000004040E04040404005050506000088881F
:101C400088887805050506000088888850200705E3
:101C500005080000929292926C0505050600008826
:101C6000502050880507070600FE88888888780875
:101C700030050505060000F8102040F803070704AA
:101C80000000204040804040200107070200008003
:101C9000808080808080030707040000804040200F
:101CA000404080FFFF000000000000000000000036
:101CB0000000000000000000000000000000000024
:101CC0000000000000000000000000000000000014
:101CD0000000000000000000000000000000000004
:101CE00000000000000000000000000000000000F4
:101CF00000000000000000000000000000000000E4
:101D000000000000000000000000000000000000D3
:101D100000000000000000000000000000000000C3
:101D200000000000000000000000000000000000B3
:101D300000000000000000000000000000000000A3
:101D40000000000000000000000000000000000093
:101D500000000000000000F000000000E0000000B3
:101D600000000000000001980000000720000000B3
:101D7000000000000000030C0000001C2000000018
:101D80000000000000000205C000007020000000FC
:101D90000001F70000000205300001C020000090A3
:101DA000000014800000030D0C000700200D92B904
:101DB0008C0014400000019903001C002012529274
:101DC0005201F440000000F100C070002012529255
:101DD00052001440000000010031C0002012529255
:101DE0005200148000000001000E000020124E99E5
:101DF0008C01F700000003FD00040010200000002B
:101E000000000000000002058004003020000000F7
:101E10000000000000000204600400D02000000068
:101E2000000000000000020418040310200000005D
:101E3000000000000000020406040C102000000056
:101E400000000000000002040184301020000000A7
:101E500000000000000002040064C0102000000028
:101E60000000000000000204001F00102010023FCC
:101E7000F880000000000204000400102018060191
:101E800000800000000002040000001020140A017D
:101E90000080000000000204000000102012120167
:101EA0000080000000000204000000102011220148
:101EB0000080000000000204000000102010C20199
:101EC0000080000000000204000000102010020149
:101ED0000080000000000204000000102010020139
:101EE0000080000000000204000000102010020129
:101EF000008000000000020400000010200000002C
:101F0000000000000000020400000010200000009B
:101F1000000000000000020400000010200000008B
:101F2000000000000000020400000010200000007B
:101F3000000000000000020400000010200000006B
:101F4000000000000000020400000010200000005B
:101F5000000000000000020400000010200000004B
:101F60000000000000000108000000102000000038
:101F700000000000000000900000001FE0000000D2
:101F800000000000000000600000000000000000F1
:101F90000000000000000000000000000000000041
:101FA0000000000000000000000000000000000031
:101FB0000000000000000000000000000000000021
:101FC0000000000000000000000000000000000011
:101FD0000000000000000000000000000000000001
:101FE00000000000000000000000000000000000F1
:101FF00000000000000000000000000000000000E1
:1020000000000000000000000000000000000000D0
:1020100000000000000000000000000000000000C0
:1020200000000000000000000000000000000000B0
:1020300000000000000000000000000000000000A0
:102040000000000000000000000000000000000090
:102050000000000000000000000000000000000080
:102060000000000000000000000000000000000070
:102070000000000000000000000000000000000060
:102080000000000000000000000000000000000050
:102090000000000000000000000000000000000040
:1020A00000000000000000000002010000040080A9
:1020B0000008004000100020002000100040000830
:1020C00000FFFFFC008048040080480400804804B2
:1020D00000804804008048040080480400FFCFFCD2
:1020E00000000000000000000000000000000000F0
:1020F000000000000000300C000060060000C0037B
:102100000001800180030000C0060000600C000098
:1021100030180000183000000C600000067FFFFF40
:10212000FE7FFFFFFE600FF006600C3006600C3093
:1021300006600C3006600C3006600C3006600C3017
:10214000067FFC3FFE3FF81FFC000000000000007F
:10215000000000000000000000000000000000007F
:102160000000000000FFE0FFD11000FFFEFFD0FFE5
:10217000E0FFC1FFD140A0C8A6A22FF8002381270D
:10218000AC00AFFF64A5FF64FF64A4FFD0FFFE00B6
:10219000000A0B02090C0D0E0807030401000000E1
:1021A000000000000000000000000000000000002F
:1021B00000000000000000000000001211100000EC
:1021C000000000000000000000000000000000000F
:1021D000000000000001021020200808102040101C
:1021E00020408002010201080402010102040810DB
:1021F00020408080402010080402018004020180F9
:102200004020100804020108040201010204081021
:1022100020408001020408102040800505050507C4
:102220000508080808020202020A0A080804040451
:10223000040101010101010101030303030303037D
:1022400003040707070C0C0C0C0C0C0C0C0202020C
:102250000206060606060606060B0B0B0B0B0B0BFF
:102260000B00002200250028002B002E0031003436
:102270000002010000050108010B010000210024FB
:102280000027002A002D0030003300010100000467
:102290000107010A01024E414E494E495459494E27
:1022A00046CDCCCC3D0AD7233C17B7D13877CC2BC1
:1022B000329595E6241FB14F0A000020410000C866
:1022C0004200401C4620BCBE4CCA1B0E5AAEC59DE7
:1022D00074002640A4A155A22A4011241FBECFEFAE
:1022E000D1E2DEBFCDBF00E00CBF15E0A0E0B2E060
:1022F000E6E4FBE701E00BBF02C007900D92A439B2
:10230000B107D9F724E1A4E9B5E001C01D92AC33CF
:10231000B207E1F712E2C8EDD2E200E006C0229770
:102320000109FE010BBF0E941EB7C23DD10780E02C
:102330000807A9F70E9448AE0C9492BD0C940000C7
:10234000FC0114821782138212828FE094E0918341
:10235000808308952FE034E0FC01318320832781BE
:10236000222319F004960C947C5908950F931F931F
:10237000CF93DF93EC018F96E3DFCE01805B9F4F1D
:10238000DFDFCE0181599F4FDBDFCE0182579F4FA8
:10239000D7DFFE01E355FF4F89E181831482359633
:1023A000178ACE0180539F4FCBDFFE01E151FF4FD3
:1023B0001082118212821382389610821182128248
:1023C00013821A821B82188219828E010D501F4FB0
:1023D000F8011082118212821382389681E0808384
:1023E0001EA61DA60E940BAC68577C4E8F4F9F4FB8
:1023F000F8016083718382839383DF91CF911F9172
:102400000F910895FC0120E03EE2DB014C91403247
:1024100041F0283011F430833196DB014C91408338
:1024200031962F5F6F5F7F4F2B3079F710820895C1
:102430003F924F925F926F927F928F929F92AF9254
:10244000BF92CF92DF92EF92FF920F931F93CF93A1
:10245000DF93CDB7DEB7C758D1090FB6F894DEBF0A
:102460000FBECDBF8C016B017A01312C84E0E80EE8
:10247000F11C2801E1E14E0E511C5801FCEFAF0E9A
:10248000B11C48018EEF880E911C80E4682E712CDF
:102490006C0E7D1EE4E06E0E711CA201BE016F5F2A
:1024A0007F4FC7010E94E65718160CF029C12C85F2
:1024B000322F3871303109F09CC0F5018081918153
:1024C0000197029708F495C0BE016F5F7F4FCE0160
:1024D00087589F4F97DFA0961FAEA097F601808187
:1024E000811107C062EF72E0CE01815A9F4F0E94B6
:1024F00041BAB601CE01815A9F4F0E9441BABE0136
:1025000067587F4FCE01815A9F4F0E9441BA62EFB8
:1025100072E0CE01815A9F4F0E9441BACE01805C89
:102520009F4F0EDF21E0AE0147585F4FB701C30157
:102530000E94735B811139C0F50180819181892BE3
:10254000A1F5E1EEF2E08491882341F09091C00082
:1025500095FFFCCF8093C6003196F5CFE4EFF2E013
:102560008191882339F09091C00095FFFCCF809332
:10257000C600F6CF8091C00085FFFCCF8AE0809333
:10258000C600FE01E758FF4F8191882339F09091F2
:10259000C00095FFFCCF8093C600F6CF8091C000AD
:1025A00085FFFCCF8AE08093C6008BE1FE01EC5BE7
:1025B000FF4FDE01959601900D928A95E1F72496E2
:1025C0008EAD9FAD24979CA38BA38FE094E09AA33C
:1025D00089A3AE014F5D5F4FBE01615A7F4FC801B5
:1025E00027DFCE018196B6DECE01805C9F4FB2DE42
:1025F00054CF8981882309F483C0853E09F44DCFE7
:102600008E3209F44ACF8F3509F447CFF80181891A
:10261000882331F08E3209F440CF8F3509F43DCF55
:1026200023FD3BCF81E0303109F080E0F80184A741
:10263000811110C09091FD088985992321F08E3475
:1026400009F02BCF03C0873409F027CF8A858E3756
:1026500009F423CF98012C5F3F4FBE016F5F7F4F7E
:10266000C901CA57DF4F2883C658D040C957DF4F2A
:102670003883C758D040C6DEF50180819181CA57A2
:10268000DF4F2881C658D040C957DF4F3881C7581F
:10269000D0400097F1F4F6018191882339F09091B0
:1026A000C00095FFFCCF8093C600F6CFF901819161
:1026B000882339F09091C00095FFFCCF8093C6002D
:1026C000F6CF8091C00085FFFCCF8AE08093C600E2
:1026D000E4CE8130910539F4F40180819181019635
:1026E00091838083DACE029709F0D7CE232D30E094
:1026F000F401808191812817390711F03394CDCEF0
:10270000C957DF4F0FB6F894DEBF0FBECDBFDF91C4
:10271000CF911F910F91FF90EF90DF90CF90BF90DE
:10272000AF909F908F907F906F905F904F903F9071
:102730000895EF92FF920F931F93CF93DF93CDB73E
:10274000DEB76F970FB6F894DEBF0FBECDBF8C011A
:10275000FC01E450FF4F118210827C0183E3E80EFC
:10276000F11C40E050E0BA01C7010E9499588BE18A
:10277000F701DE01159601900D928A95E1F7F801B7
:1027800081A992A99C838B838FE094E09A838983AB
:10279000AE014F5F5F4F63EE74E0C80149DECE01CA
:1027A0000196D8DD6F960FB6F894DEBF0FBECDBF91
:1027B000DF91CF911F910F91FF90EF9008952BE142
:1027C000FB013496DC01149601900D922A95E1F7F5
:1027D000FB0122813381FC01338322830895EF9230
:1027E000FF920F931F93CF93DF93EC011B828EA96F
:1027F000882321F0CE01C3960E947C597E018DEA88
:10280000E80EF11C45E360E0C7010E94FD53811111
:102810001FC0E1EEF2E08491882341F09091C00066
:1028200095FFFCCF8093C6003196F5CFE4EDF2E042
:102830008491882341F09091C00095FFFCCF809354
:10284000C6003196F5CF8091C00085FFFCCF76C0E1
:102850008E010E541F4F41E0B701C8010E9466610E
:10286000811126C040E0B701C8010E946661811154
:102870001FC0E7EEF2E08491882341F09091C00000
:1028800095FFFCCF8093C6003196F5CFE1ECF2E0E6
:102890008491882341F09091C00095FFFCCF8093F4
:1028A000C6003196F5CF8091C00085FFFCCF46C0B1
:1028B000B801CE01C3960E948A5681111FC0E7EE6F
:1028C000F2E08491882341F09091C00095FFFCCF05
:1028D0008093C6003196F5CFE1EBF2E08491882336
:1028E00041F09091C00095FFFCCF8093C6003196D7
:1028F000F5CF8091C00085FFFCCF20C081E08B83A5
:10290000E1EEF2E08491882341F09091C00095FFC0
:10291000FCCF8093C6003196F5CFE6EAF2E08491D1
:10292000882341F09091C00095FFFCCF8093C600B2
:102930003196F5CF8091C00085FFFCCF8AE080936F
:10294000C6008E01015D1F4FB801CE01805B9F4F15
:1029500036DFC25BDF4F19830883DF91CF911F9170
:102960000F91FF90EF900895FC0112821382089559
:10297000FC012381222311F021E022830895FC0130
:1029800022812111128208952F923F924F925F92DD
:102990006F927F928F929F92AF92BF92CF92DF926F
:1029A000EF92FF920F931F93CF93DF93CDB7DEB7D4
:1029B000AD970FB6F894DEBF0FBECDBF7C016B01A3
:1029C0004DA7FC018381882309F4A7C14701F4EDD9
:1029D0008F0E911CC4010E947C59F7011282CE0116
:1029E00001965C01ADDC17019EE4290E311CC70184
:1029F0008F96F10191838083F60180818F3209F0F7
:102A00007FC06FE270E0C6010E944CBA8C010F5F7C
:102A10001F4F09F47BC06FE270E0C8010E944CBAFE
:102A20002C01009709F473C00817190708F06FC04C
:102A30003C01601A710AA301B801CE0180960E9480
:102A40006CBAE0E2F0E0EC0FFD1FE60DF71D10821E
:102A5000FE01B0968191882339F09091C00095FFD6
:102A6000FCCF8093C600F6CF8091C00085FFFCCFDD
:102A7000FAE0F093C600F101608171816115710582
:102A800019F06C5F7F4F02C060E070E021E0AE01A2
:102A9000405E5F4FCE0105960E94735B81112BC093
:102AA000E2E9F2E08491882341F09091C00095FF23
:102AB000FCCF8093C6003196F5CFFE01B096819190
:102AC000882339F09091C00095FFFCCF8093C60019
:102AD000F6CFE0E9F2E08491882341F09091C000C4
:102AE00095FFFCCF8093C6003196F5CF8091C00052
:102AF00085FFFCCFE7C0F101B182A082820187CFC0
:102B0000C701805B9F4FF101918380838601FDA502
:102B1000FF2309F49CC0F101608171816115710589
:102B200019F06C5F7F4F02C060E070E021E0A80107
:102B3000C4010E94735B882309F45FC0F40181899A
:102B40009289A389B489F701E151FF4F8083918372
:102B5000A283B383E2E8F2E08491D701A151BF4F91
:102B6000882349F09091C00095FFFCCF8093C60068
:102B700031968491F5CFF8018191882339F09091B5
:102B8000C00095FFFCCF8093C600F6CFEAE7F2E0E5
:102B90008491882341F09091C00095FFFCCF8093F1
:102BA000C6003196F5CF4D915D916D917C912AE0F3
:102BB00030E084E995E00E94AC1F8091C00085FF61
:102BC000FCCF8AE08093C600F701E950FF4F1082E6
:102BD000118212821382ECE6F2E08491882341F0A4
:102BE0009091C00095FFFCCF8093C6003196F5CF41
:102BF0008091C00085FFFCCF88C0E8E5F2E08491B9
:102C0000882341F09091C00095FFFCCF8093C600CF
:102C10003196F5CFF8018191882339F09091C00069
:102C200095FFFCCF8093C600F6CFE6E5F2E08491F5
:102C3000882341F09091C00095FFFCCF8093C6009F
:102C40003196F5CF8091C00085FFFCCF3BC0F101EC
:102C5000608171816115710519F06C5F7F4F02C051
:102C600060E070E026E5A801C4010E94735B811159
:102C70002DC0E2E4F2E08491882341F09091C000FD
:102C800095FFFCCF8093C6003196F5CFF801819176
:102C9000882339F09091C00095FFFCCF8093C60047
:102CA000F6CFE0E4F2E08491882341F09091C000F7
:102CB00095FFFCCF8093C6003196F5CF8091C00080
:102CC00085FFFCCF8AE08093C60025C081E0F70134
:102CD0008083EEE2F2E08491882341F09091C0007D
:102CE00095FFFCCF8093C6003196F5CFF601819118
:102CF000882339F09091C00095FFFCCF8093C600E7
:102D0000F6CF8091C00085FFFCCF8AE08093C6009B
:102D1000C8010E941F85C5011DDBAD960FB6F89452
:102D2000DEBF0FBECDBFDF91CF911F910F91FF90FE
:102D3000EF90DF90CF90BF90AF909F908F907F905B
:102D40006F905F904F903F902F90089521E0FC018D
:102D5000218340E019CE3F924F925F926F927F9213
:102D60008F929F92AF92BF92CF92DF92EF92FF929B
:102D70000F931F93CF93DF93CDB7DEB7AC970FB60A
:102D8000F894DEBF0FBECDBF7C015B01FC018381E7
:102D9000882309F400C1C7018C529F4F0E947C59BF
:102DA000F7011282CE0101966C01CADA27019EE476
:102DB000490E511CC7018F96F20191838083F50162
:102DC00080818F3209F084C06FE270E0C5010E94FB
:102DD0004CBA8C010F5F1F4F9AE0392E0115110577
:102DE00009F47CC06FE270E0C8010E944CBA4C014B
:102DF000009709F474C00817190708F070C03C0167
:102E0000601A710AA301B801CE0180960E946CBAC3
:102E1000E0E2F0E0EC0FFD1FE60DF71D1082FE0171
:102E2000B0968191882339F09091C00095FFFCCF36
:102E30008093C600F6CF8091C00085FFFCCF309212
:102E4000C600F201608171816115710519F06C5F36
:102E50007F4F02C060E070E021E0AE01405E5F4F56
:102E6000CE0105960E94735B81112BC0EAE1F2E06E
:102E70008491882341F09091C00095FFFCCF80930E
:102E8000C6003196F5CFFE01B0968191882339F0C6
:102E90009091C00095FFFCCF8093C600F6CFE8E18B
:102EA000F2E08491882341F09091C00095FFFCCF1F
:102EB0008093C6003196F5CF8091C00085FFFCCF8E
:102EC00065C0F201D182C08284010F5F1F4F86CF9F
:102ED000C701805B9F4FF201918380838501F201DE
:102EE00080819181009711F0049602C080E090E00B
:102EF000B8010E94495C882301F1EAE0F2E0849184
:102F0000882341F09091C00095FFFCCF8093C600CC
:102F10003196F5CFF8018191882339F09091C00066
:102F200095FFFCCF8093C600F6CFF701E950FF4F25
:102F300010821182128213822CC0E2EFF1E08491A0
:102F4000882341F09091C00095FFFCCF8093C6008C
:102F50003196F5CFF8018191882339F09091C00026
:102F600095FFFCCF8093C600F6CFE0EFF1E08491AF
:102F7000882341F09091C00095FFFCCF8093C6005C
:102F80003196F5CF8091C00085FFFCCF8AE0809319
:102F9000C600C601DFD9AC960FB6F894DEBF0FBEEF
:102FA000CDBFDF91CF911F910F91FF90EF90DF90F8
:102FB000CF90BF90AF909F908F907F906F905F90D9
:102FC0004F903F900895CF93DF93EC018B8188233E
:102FD000B1F1EEEDF1E08491882341F09091C000D1
:102FE00095FFFCCF8093C6003196F5CFFE01E950E6
:102FF000FF4F40815181628173812AE030E084E992
:1030000095E0AAD7ECEDF1E08491882341F090910E
:10301000C00095FFFCCF8093C6003196F5CFC1511B
:10302000DF4F488159816A817B812AE030E084E961
:1030300095E092D78091C00085FFFCCF11C0ECECE9
:10304000F1E08491882341F09091C00095FFFCCF7E
:103050008093C6003196F5CF8091C00085FFFCCFEC
:103060008AE08093C600DF91CF910895AF92BF921E
:10307000CF92DF92EF92FF920F931F93CF93DF9344
:103080005C01EB01FB0101900020E9F78F01015089
:103090001109061B170B6C01F4EDCF0ED11CF601C4
:1030A00010826EE470E0CE010E944CBA7C01009761
:1030B00029F4F8013197EC0FFD1F0DC060E270E0BC
:1030C0000E944CBAEC0121966AE270E0C7010E94AE
:1030D0004CBAFC0131978DE081838AE082831382B0
:1030E000BE01C50180539F4F0E940F5EF601808193
:1030F000882309F1E7EEF2E08491882341F0909172
:10310000C00095FFFCCF8093C6003196F5CFE6EB6B
:10311000F1E08491882341F09091C00095FFFCCFAD
:103120008093C6003196F5CF8091C00085FFFCCF1B
:103130008AE08093C600DF91CF911F910F91FF909D
:10314000EF90DF90CF90BF90AF9008952F923F9275
:103150004F925F926F927F928F929F92AF92BF92A7
:10316000CF92DF92EF92FF920F931F93CF93DF9353
:10317000CDB7DEB7CC55D1090FB6F894DEBF0FBE80
:10318000CDBF8C0185509F4F5C01662339F0F5015E
:103190001082F801838181111DC015C0FC0180815E
:1031A000882309F4ADC0F801ED50FF4FC080D180F5
:1031B000E280F3800E940BACC616D706E806F9063B
:1031C00008F49EC0E4CFC8010ADBF801838188239C
:1031D00009F496C0F80186A58F9385A58F938DEA93
:1031E00091E09F938F937E01FFE3EF0EF11CFF921E
:1031F000EF920E94B7BA0F900F900F900F900F9020
:103200000F90B12CF70101900020E9F73197EE19EA
:10321000FF09BE1684F46701CB0CD11CB7FCDA940D
:10322000F6018081992787FD90950E94D2B9F60119
:103230008083B394E7CF4801F3E38F0E911C40E005
:1032400050E0BA01C4010E949958512CCE01019658
:103250006C0126EA622E21E0722E5E0191E2A90E37
:10326000B11C40E050E0B601C4010E94E6571816B8
:10327000DCF5412CF60101900020E9F73197EC19BB
:10328000FD094E1674F41601240C311C47FC3A94C7
:10329000F101808190E00E94D2B9F10180834394D2
:1032A000E9CF8A858E37E9F245E050E0B701C601E3
:1032B0000E945EBA892BA9F6FF92EF927F926F92DD
:1032C000BF92AF920E94B7BAC5010E940B2282EA58
:1032D00091E00E947E220F900F900F900F900F9020
:1032E0000F9055245394BDCF511004C08FEF9FEF22
:1032F000F80104C0F80185A596A5019696A785A7B3
:10330000C45ADF4F0FB6F894DEBF0FBECDBFDF91BA
:10331000CF911F910F91FF90EF90DF90CF90BF90D2
:10332000AF909F908F907F906F905F904F903F9065
:103330002F9008950F931F93CF93DF93EC018C018F
:103340000C521F4FC8010E943259C8010E947C597B
:1033500018821982DF91CF911F910F910895EF92FA
:10336000FF920F931F93CF93DF93CDB7DEB76F9785
:103370000FB6F894DEBF0FBECDBF8C017C018EE48A
:10338000E80EF11CC801805B9F4FF7019183808399
:10339000E255FF4F22E030E031832083329670E027
:1033A0007183608340E050E0BA0104960E9499580E
:1033B000F701808191812BE1FC013496DE011596A5
:1033C00001900D922A95E1F7FC01828193819C8303
:1033D0008B838FE094E09A838983AE014F5F5F4FC8
:1033E00063EE74E0C80124D8CE0101960E94AA11B0
:1033F0006F960FB6F894DEBF0FBECDBFDF91CF91B1
:103400001F910F91FF90EF900895CF92DF92EF926E
:10341000FF920F931F93CF93DF93CDB7DEB76F97D4
:103420000FB6F894DEBF0FBECDBF8C016C012EE449
:10343000C20ED11C805B9F4FF60191838083E255C1
:10344000FF4F21E030E0318320837801FEEFEF0E63
:10345000F11CF7011182108240E050E0BA0104969D
:103460000E949958F601808191812BE1FC013496EC
:10347000DE01159601900D922A95E1F7FC018281FB
:1034800093819C838B838FE094E09A838983AE0140
:103490004F5F5F4F63EE74E0C8010E941812CE01C7
:1034A00001960E94AA11F701808191816F960FB653
:1034B000F894DEBF0FBECDBFDF91CF911F910F916A
:1034C000FF90EF90DF90CF9008950F931F93CF93CD
:1034D000DF93EC01FC01E95AFF4F8081825082307A
:1034E00088F08E0101591F4FB801CE01805B9F4FBC
:1034F00066D9BE0162577F4FC801DF91CF911F91FE
:103500000F915DC9DF91CF911F910F910895CF93D6
:10351000DF93EC010E94726A0E94E86ACE018C522D
:103520009F4F0E947C591A8286E991E0E7D78091EB
:10353000E30E8823F9F01092E30EC091CA08D0E0A0
:10354000CC0FDD1FC85CDD4E68817981882777FD4F
:103550008095982F0E949BB3209148023091490298
:1035600040914A0250914B020E94FCB4181614F488
:1035700019821882DF91CF910895EF92FF920F93F5
:103580001F93CF93DF931F92CDB7DEB78C017B01E2
:10359000460FF70161917F01F80180819181498394
:1035A0000E94DBBCF8018081918101969183808328
:1035B00049814E11EECF0F90DF91CF911F910F9166
:1035C000FF90EF900895EF92FF920F931F93CF9388
:1035D000DF931F92CDB7DEB78C017B01460FF80158
:1035E0008081918149830E94D3BCF70181937F013F
:1035F000F8018081918101969183808349814E11E8
:10360000EECF0F90DF91CF911F910F91FF90EF9030
:1036100008950F931F93CF93DF93CDB7DEB72A970B
:103620000FB6F894DEBF0FBECDBF80E390E3A0E3FA
:10363000B0E08D839E83AF83B88704E610E01A87DD
:10364000098744E0BE016B5F7F4FCE01099695DF8D
:1036500040E164E47FE0CE0109968FDF40E164E55C
:103660007FE0CE01099689DF40E164E37FE0CE018F
:10367000099683DF44E06CE27FE0CE0109967DDFAE
:1036800044E068E27FE0CE01099677DF44E060E342
:103690007FE0CE01099671DF44E068E17FE0CE0172
:1036A00009966BDF44E064E67FE0CE01099665DFB2
:1036B00044E064E27FE0CE0109965FDF44E060E22F
:1036C0007FE0CE01099659DF44E06CE17FE0CE0156
:1036D000099653DF4CE067ED78E0CE0109964DDFA7
:1036E00042E066E079E0CE01099647DF42E061EC16
:1036F00072E1CE01099641DF42E06FEB72E1CE014B
:1037000009963BDF42E06DEB72E1CE01099635DFB1
:1037100042E06BEB72E1CE0109962FDF42E069EBEC
:1037200072E1CE01099629DF42E067EB72E1CE013A
:10373000099623DF44E06AE672E0CE0109961DDFB8
:1037400044E066E672E0CE01099617DF44E062E6E7
:1037500072E0CE01099611DF86E590E3A7E3B0E0C1
:1037600089839A83AB83BC831A87098744E0BE01AF
:103770006F5F7F4FCE01099600DFEAE3F3E08491AB
:10378000882341F09091C00095FFFCCF8093C60044
:103790003196F5CFEAE2F3E08491882341F09091ED
:1037A000C00095FFFCCF8093C6003196F5CF809185
:1037B000C00085FFFCCF8AE08093C6002A960FB632
:1037C000F894DEBF0FBECDBFDF91CF911F910F9157
:1037D0000895AF92BF92CF92DF92EF92FF920F9334
:1037E0001F93CF93DF93CDB7DEB7E0970FB6F89472
:1037F000DEBF0FBECDBF80E1E2ECF2E0DE019196CC
:1038000001900D928A95E1F780E1E2EDF2E0DE01B0
:10381000519601900D928A95E1F780E1E2EEF2E097
:10382000DE01119601900D928A95E1F76E0181E219
:10383000C80ED11C84E4E82E8FE0F82E8E010F5EB6
:103840001F4F64E57FE0AE014F5F5F4F94E3A92E09
:103850009FE0B92E20E030E0F60181919191A19195
:10386000B1916F01F70181939193A193B1937F017E
:10387000F80181919191A191B1918F01FB01819307
:103880009193A193B193BF01FA0181919191A1917B
:10389000B191AF01F50181939193A193B1935F0130
:1038A0002F5F3F4F24303105B9F60E94C85280E0A7
:1038B00090E8ABE3B5E480932C0F90932D0FA09389
:1038C0002E0FB0932F0F8093280F9093290FA09362
:1038D0002A0FB0932B0F1092300F1092310F1092CD
:1038E000320F1092330F80E29EE4A0E0B0E08093AC
:1038F000640F9093650FA093660FB093670F1092BB
:10390000180F1092190F10921A0F10921B0F80E0CF
:1039100090E0A0EAB1E48093240F9093250FA09348
:10392000260FB093270F8DEC9CECACECBEE380939C
:10393000200F9093210FA093220FB093230F80E0CC
:1039400090E0A0EAB0E480931C0F90931D0FA09329
:103950001E0FB0931F0F1092DF081092E008109214
:10396000E1081092E2081092DB081092DC08109235
:10397000DD081092DE081092D7081092D808109235
:10398000D9081092DA0883E690E0909307098093B3
:1039900006091092FF088EEB90E09093C21280937C
:1039A000C1128CE390E09093C0128093BF128FEF0E
:1039B00090E09093BE128093BD1220EF30E03093E0
:1039C000BC122093BB122AE530E03093BA12209348
:1039D000B9129093B8128093B7128AE999E9A1EBD2
:1039E000B1E480936A0290936B02A0936C02B0934F
:1039F0006D0261E77DE38AE89FE30E942975609389
:103A0000660270936702809368029093690260E097
:103A100070E084EE92E40E943575609362027093C8
:103A2000630280936402909365020E94626C80E05E
:103A300090E0A0E8BFE380935E0290935F02A093C2
:103A40006002B0936102E5DDEAE3F3E0849188234C
:103A500041F09091C00095FFFCCF8093C600319655
:103A6000F5CFEEEEF2E08491882341F09091C00012
:103A700095FFFCCF8093C6003196F5CF8091C000B2
:103A800085FFFCCF8AE08093C600E0960FB6F894DD
:103A9000DEBF0FBECDBFDF91CF911F910F91FF9081
:103AA000EF90DF90CF90BF90AF900895CF93DF93CA
:103AB000CDB7DEB72A970FB6F894DEBF0FBECDBFE5
:103AC00084E690E09A87898786E590E3A7E3B0E0F3
:103AD00089839A83AB83BC8344E0BE016B5F7F4FD5
:103AE000CE01099670DD43E050E0BE016B5F7F4F71
:103AF000CE0101960E945EBA892B09F0AAC040E16E
:103B000064E47FE0CE0109965EDD40E164E57FE09C
:103B1000CE01099658DD40E164E37FE0CE010996CD
:103B200052DD0E94C85244E06CE27FE0CE0109966B
:103B30004ADD44E068E27FE0CE01099644DD44E0DE
:103B400060E37FE0CE0109963EDD44E068E17FE07E
:103B5000CE01099638DD44E064E67FE0CE010996A7
:103B600032DD44E064E27FE0CE0109962CDD44E0E2
:103B700060E27FE0CE01099626DD44E06CE17FE063
:103B8000CE01099620DD4CE067ED78E0CE01099684
:103B90001ADD42E066E079E0CE01099614DD42E0EC
:103BA00061EC72E1CE0109960EDD42E06FEB72E14D
:103BB000CE01099608DD42E06DEB72E1CE01099677
:103BC00002DD42E06BEB72E1CE010996FCDC42E0E3
:103BD00069EB72E1CE010996F6DC42E067EB72E137
:103BE000CE010996F0DC44E06AE672E0CE01099667
:103BF000EADC44E066E672E0CE010996E4DC44E0EB
:103C000062E672E0CE010996DEDC0E94626CEAE3B5
:103C1000F3E08491882341F09091C00095FFFCCFA0
:103C20008093C6003196F5CFE0E1F3E084918823DC
:103C300041F09091C00095FFFCCF8093C600319673
:103C4000F5CF8091C00085FFFCCF8AE08093C6004D
:103C500001C0BFDD2A960FB6F894DEBF0FBECDBF00
:103C6000DF91CF9108951F920F920FB60F921124FA
:103C70000BB60F922F933F934F935F936F938F9356
:103C80009F93EF93FF936091C600209115063091AA
:103C90001606C90101968F77992740911706509112
:103CA00018068417950741F0F901EB56FA4F608327
:103CB0009093160680931506FF91EF919F918F9137
:103CC0006F915F914F913F912F910F900BBE0F908D
:103CD0000FBE0F901F9018959A01AB01211581EE30
:103CE00038074105510549F182E08093C00060E04A
:103CF00079E08DE390E00E94ECB621503109410952
:103D00005109CA01B90122E030E040E050E00E94D0
:103D1000ECB63093C5002093C4008091C10080614F
:103D20008093C1008091C10088608093C100809120
:103D3000C10080688093C10008951092C00020E106
:103D400030E0E7CF209117063091180680911506D4
:103D5000909116068217930771F0F901EB56FA4F0E
:103D600080812F5F3F4F2F773327309318062093A2
:103D7000170690E008958FEF9FEF08958091170642
:103D800090911806909316068093150608954F9209
:103D90005F926F927F928F929F92AF92BF92CF92DB
:103DA000DF92EF92FF920F931F93CF93DF93CDB7E4
:103DB000DEB7A0970FB6F894DEBF0FBECDBF5C0193
:103DC0004115510561057105E9F420E030E040E35B
:103DD00050E060E070E0A0960FB6F894DEBF0FBE32
:103DE000CDBFDF91CF911F910F91FF90EF90DF90AA
:103DF000CF90BF90AF909F908F907F906F905F908B
:103E00004F905BC08E010F5F1F4FC12CD12C7601EC
:103E10004801422E512C612C712C8FEFC81AD80A00
:103E2000E80AF80ACB01BA01A30192010E94CAB6BE
:103E3000CA01F80161938F01A901BC014115510527
:103E40006105710551F7F1E0CF1AD108E108F108D9
:103E5000F401EC0DFD1D80818A3010F440E301C0B7
:103E600047E3480F552747FD5095652F752F20E0F4
:103E700030E0C50122D081E0C81AD108E108F1087C
:103E8000EFEFCE16DE06EE06FE0611F7A0960FB691
:103E9000F894DEBF0FBECDBFDF91CF911F910F9180
:103EA000FF90EF90DF90CF90BF90AF909F908F905A
:103EB0007F906F905F904F9008952115310539F4F0
:103EC0008091C00085FFFCCF4093C60008952A3042
:103ED000310509F41CC05BCFCF93DF93EC0120E0E8
:103EE00030E04DE050E060E070E0E7DF20E030E0FF
:103EF0004AE050E060E070E0CE01DF91CF91DDCF8D
:103F00009A01AB01662757FD6095762FD6CFCF92E9
:103F1000DF92EF92FF92CF93DF93EC016A017B0176
:103F200077FF0FC020E030E04DE250E060E070E04D
:103F3000C4DFF094E094D094C094C11CD11CE11C67
:103F4000F11C2AE0B701A601CE01DF91CF91FF90CD
:103F5000EF90DF90CF901BCF2115310539F4809180
:103F6000C00085FFFCCF4093C600089510CF9A0192
:103F7000462F50E060E070E0EFCFCF93DF93EC018D
:103F80009A01AB0160E070E0E7DFCE01DF91CF91F5
:103F9000A3CF8F929F92AF92BF92CF92DF92EF9278
:103FA000FF921F93CF93DF93EC016A017B01122FE5
:103FB00020E030E0A901C701B6010E94F9B287FFF5
:103FC0000CC020E030E04DE250E060E070E0CE0157
:103FD00074DFF7FAF094F7F8F094B12C60E070E039
:103FE00080E09FE3B11641F020E030E040E251E490
:103FF0000E9400B3B394F6CF9B01AC01C701B60198
:104000000E9420B26B017C010E946DB34B015C01E8
:104010000E9499B39B01AC01C701B6010E941FB277
:104020006B017C012AE0B501A401CE01B0DE1123B1
:1040300061F0E2E7F4E08191882339F09091C000CB
:1040400095FFFCCF8093C600F6CF112319F120E035
:1040500030E040E251E4C701B6010E94CEB56B01E9
:104060007C010E9468B34B01AA2497FCA094BA2C4F
:10407000B501A401CE014BDFC501B4010E949BB381
:104080009B01AC01C701B6010E941FB26B017C010C
:104090001150DBCFDF91CF911F91FF90EF90DF9018
:1040A000CF90BF90AF909F908F90089572CFFC01FA
:1040B000659175918591949108957F928F929F92C9
:1040C000AF92BF92CF92DF92EF92FF920F931F9326
:1040D000CF93DF93EC018C01000F111F000F111F14
:1040E000F801ED51F74F10821182128213822FEEE8
:1040F00038E04BEE58E067EE78E083EE98E00E94FF
:10410000FD51C8018559984FD2DF9E01245A384F7E
:104110005901F90174904E01880C991C880C991C66
:1041200084010854174F20E030E040EC5FE30E9428
:10413000CEB56B017C01672D772767FD7095872FC2
:10414000972F0E949BB39B01AC01C701B6010E944F
:10415000CEB5F8016083718382839383F401E05DBF
:10416000FD4F608171818281938160930B02709316
:104170000C0280930D0290930E0220E030E040E7A5
:1041800052E40E9400B33AECC32E38E0D32E7B01F8
:104190008C0124EC38E040EC58E06CEB78E088EBE4
:1041A00098E00E9471480E94726AF401ED51F74F45
:1041B00010821182128213822FEE38E04BEE58E00B
:1041C00067EE78E083EE98E00E94FD519401215A59
:1041D000384F4901C9016BDFF50124918E01000FB1
:1041E000111F000F111F0854174F6B017C01F7FAC4
:1041F000F094F7F8F094622F772767FD7095872F7A
:10420000972F0E949BB39B01AC01C701B6010E948E
:10421000CEB5F801608371838283938320E030E020
:1042200040E752E460910B0270910C0280910D0204
:1042300090910E020E9400B35AECC52E58E0D52E84
:104240007B018C0124EC38E040EC58E06CEB78E02A
:1042500088EB98E00E9471480E94726AC40127DFCF
:10426000F5011491CC0FDD1FCC0FDD1F9E012854EA
:10427000374F59019B01AC010E9420B26B017C01B8
:10428000612F772767FD7095872F972F0E949BB32B
:104290009B01AC01C701B6010E94CEB5F501608358
:1042A000718382839383FE01E05DFD4F20E030E067
:1042B00040E05FE360817181828193810E94CEB58D
:1042C00060930B0270930C0280930D0290930E0288
:1042D00020E030E040E752E40E9400B3FAECCF2E39
:1042E000F8E0DF2E7B018C0124EC38E040EC58E054
:1042F0006CEB78E088EB98E00E9471480E94726A4B
:10430000CE018958984FD3DE9E012D51374F790148
:104310008E010952174FF80120813181428153816A
:104320000E9420B2F7016083718382839383CE0160
:104330008157984FBCDE9E012553374F6901F80124
:1043400020813181428153810E9420B2F601608335
:10435000718382839383CE018D57984FA8DEC05E10
:10436000DD4FF80120813181428153810E9420B2CA
:10437000688379838A839B83F70180819181A281FD
:10438000B381F50180839183A283B38310920B02E2
:1043900010920C0210920D0210920E02DF91CF913A
:1043A0001F910F91FF90EF90DF90CF90BF90AF9053
:1043B0009F908F907F900C943B63FC01249122236B
:1043C00041F03091C00035FFFCCF2093C60001962C
:1043D000F4CF22E030E084E995E068CECF93DF931C
:1043E0001F921F92CDB7DEB780913614909137148B
:1043F0009E012F5F3F4F009719F42C53344102C0A8
:10440000281B390B3A83298389819A810F900F9059
:10441000DF91CF91089520910D0730910E07243040
:1044200031050CF06AC040910F075091100760E60B
:10443000649F9001659F300D1124BC01C901895E04
:10444000984F0E9457BAEBE9F7E08491882341F036
:104450009091C00095FFFCCF8093C6003196F5CFB8
:10446000E1E5F7E08491882341F09091C00095FF49
:10447000FCCF8093C6003196F5CF80910F079091C5
:10448000100720E6289FF001299FF00D1124E95E16
:10449000F84F8191882339F09091C00095FFFCCFAF
:1044A0008093C600F6CFEFE4F7E08491882341F0D3
:1044B0009091C00095FFFCCF8093C6003196F5CF58
:1044C0008091C00085FFFCCF8AE08093C600809178
:1044D0000F0790911007019664E070E00E94B7B654
:1044E0009093100780930F0780910D0790910E070E
:1044F000019690930E0780930D07089520910D0764
:1045000030910E07243031050CF06AC040910F073E
:104510005091100760E6649F9001659F300D112453
:10452000BC01C901895E984F0E94DAB9EBE9F7E056
:104530008491882341F09091C00095FFFCCF809337
:10454000C6003196F5CFE4E4F7E08491882341F08A
:104550009091C00095FFFCCF8093C6003196F5CFB7
:1045600080910F079091100720E6289FF001299F66
:10457000F00D1124E95EF84F8191882339F0909174
:10458000C00095FFFCCF8093C600F6CFE2E4F7E0D1
:104590008491882341F09091C00095FFFCCF8093D7
:1045A000C6003196F5CF8091C00085FFFCCF8AE030
:1045B0008093C60080910F0790911007019664E0E8
:1045C00070E00E94B7B69093100780930F07809118
:1045D0000D0790910E07019690930E0780930D079B
:1045E000089560E080E40E94D9AD9FB7F894E8E0B8
:1045F000F1E08081846080839FBF0895269A2E9881
:104600000895EFDFFBDF40E950ED63E070E084E9FF
:1046100095E062DBECE3F7E08491882341F0909130
:10462000C00095FFFCCF8093C6003196F5CF8091F6
:10463000C00085FFFCCF8AE08093C60084B780FF6E
:1046400014C0E4E3F7E09491992341F02091C00075
:1046500025FFFCCF9093C6003196F5CF9091C00016
:1046600095FFFCCF9AE09093C60081FF14C0E4E26E
:10467000F7E09491992341F02091C00025FFFCCFF1
:104680009093C6003196F5CF9091C00095FFFCCF76
:104690009AE09093C60082FF14C0E3E1F7E09491A2
:1046A000992341F02091C00025FFFCCF9093C600D4
:1046B0003196F5CF9091C00095FFFCCF9AE0909392
:1046C000C60083FF14C0E3E0F7E09491992341F022
:1046D0002091C00025FFFCCF9093C6003196F5CF06
:1046E0009091C00095FFFCCF9AE09093C60085FFA3
:1046F00014C0E3EFF6E08491882341F09091C0006C
:1047000095FFFCCF8093C6003196F5CF8091C00015
:1047100085FFFCCF8AE08093C60014BEEFEEF6E082
:104720008491882341F09091C00095FFFCCF809345
:10473000C6003196F5CF8091C00085FFFCCF8AE09E
:104740008093C600EFEDF6E08491882341F09091CC
:10475000C00095FFFCCF8093C6003196F5CFEAEC00
:10476000F6E08491882341F09091C00095FFFCCF42
:104770008093C6003196F5CFEEEBF6E08491882366
:1047800041F09091C00095FFFCCF8093C600319618
:10479000F5CFE7EBF6E08491882341F09091C000DB
:1047A00095FFFCCF8093C6003196F5CF8091C00075
:1047B00085FFFCCF8AE08093C600ECEAF6E08491A6
:1047C000882341F09091C00095FFFCCF8093C600F4
:1047D0003196F5CFE0EAF6E08491882341F090919C
:1047E000C00095FFFCCF8093C6003196F5CF809135
:1047F000C00085FFFCCF8AE08093C600E1E9F6E0C7
:104800008491882341F09091C00095FFFCCF809364
:10481000C6003196F5CFE2DD4AE050E0BC0184E904
:1048200095E06EDBEAE7F6E08491882341F0909111
:10483000C00095FFFCCF8093C6003196F5CF4AE0CB
:1048400050E060ED74E084E995E05ADB8091C000AF
:1048500085FFFCCF8AE08093C60010921307109268
:10486000140710921507109216071092FF081ED910
:104870000E94966E0E940B470E94E5690E941E8668
:104880001092F60680910602813019F081E0809343
:104890000602109204098BE0809308091092030924
:1048A000109202091092F908109200091092FC0867
:1048B0001092FD08109201090895809107079091C8
:1048C000080760E070E001960C9431B7809107070B
:1048D000909108074AE050E060E070E001960C9487
:1048E00099B8682F772767FD70952091110730914F
:1048F000120740E6429FC001439F900D1124895E3C
:10490000984F0E944CBA909308078093070721E0C4
:10491000892B09F420E0822F08950E940BAC60934C
:104920000307709304078093050790930607E091AF
:104930001107F0911207ED5EF84F8081811114C0CC
:10494000E8E6F3E08491882341F09091C00095FF60
:10495000FCCF8093C6003196F5CF8091C00085FFD3
:10496000FCCF8AE08093C600089584E995E006DADA
:10497000EBE6F3E08491882341F09091C00095FF2D
:10498000FCCF8093C6003196F5CF40919C085091A2
:104990009D0860919E0870919F084F5F5F4F6F4F19
:1049A0007F4F2AE030E084E995E087DA8091C0000B
:1049B00085FFFCCF8AE08093C600AFCF4F925F9215
:1049C0006F927F929F92AF92BF92CF92DF92EF92BF
:1049D000FF920F931F93CF93DF93C0E6BC2EC4E0EA
:1049E000D0E00DE315E08AE0A82E93EBE92E95E0E8
:1049F000F92E992493948091150690911606209192
:104A0000170630911806821B930B8F779927892BF5
:104A100009F422C280910D0790910E0704970CF0C3
:104A20001BC284E995E08ED980930C071092FF0891
:104A300020910A0730910B078A3061F08D3051F0D8
:104A40008A3321F490910907992321F02F353105FC
:104A50000CF427C12115310509F441C180910F07DC
:104A600090911007B89E6001B99ED00C1124F601F8
:104A7000E20FF31FE95EF84F108220910907211120
:104A80000BC1FC01ED5EF84F1082C601895E984FA4
:104A90003C016EE470E00E944CBA0097F1F19093F3
:104AA000080780930707861997098C0D9D1D4AE01A
:104AB00050E060E070E0885E984F0E9499B8609383
:104AC000A0087093A1088093A2089093A308409037
:104AD0009C0850909D0860909E0870909F08EFEF92
:104AE0004E1A5E0A6E0A7E0AC0900F07D090100719
:104AF000641575058605970509F4F4C0BC9CC001D2
:104B0000BD9C900D11246CE576E0895E984F0E9463
:104B100011BA892B09F0E6C073C16AE270E0C301E3
:104B20000E944CBA892B09F443C0E1EAF7E0849172
:104B3000882341F09091C00095FFFCCF8093C60080
:104B40003196F5CFE6EBF5E08491882341F0909122
:104B5000C00095FFFCCF8093C6003196F5CF409101
:104B60009C0850919D0860919E0870919F082AE0D2
:104B700030E084E995E0A1D98091C00085FFFCCFA9
:104B80008AE08093C60010920B0710920A077AC23F
:104B90008091A0089091A108A091A208B091A308CB
:104BA00080939C0890939D08A0939E08B0939F08C3
:104BB00080910F0790911007B89E6001B99ED00CAC
:104BC0001124C601895E984F3C0167E470E00E94A1
:104BD0004CBA009709F44BC09093080780930707DD
:104BE000861997098C0D9D1D60E070E0885E984FD6
:104BF0000E9431B70E9468B36430710508F037C075
:104C00008091190681111AC080910B0981112FC062
:104C1000F7018491E3EBF5E0882349F09091C0001F
:104C200095FFFCCF8093C60031968491F5CF80919B
:104C3000C00085FFFCCFA092C60019C0F801849186
:104C4000EDE3F5E0882349F09091C00095FFFCCF9B
:104C50008093C60031968491F5CF8091C00085FF86
:104C6000FCCFA092C60083E395E00E942E85809140
:104C70000F07909110070196BE010E94B7B690935E
:104C8000100780930F0780910D0790910E070196F2
:104C900090930E0780930D0710920B0710920A074E
:104CA000AACE8B3311F490920907909109079111C4
:104CB000A2CE40910F0750911007B9016F5F7F4F4F
:104CC00070930B0760930A07B49EF001B59EF00D38
:104CD0001124E20FF31FE95EF84F80838CCE10920F
:104CE0000907D0C1BC9C3001BD9C700C1124C301CC
:104CF000895E984F2C016AE270E00E944CBA0097DE
:104D000081F5E1EAF7E08491882341F09091C000B9
:104D100095FFFCCF8093C6003196F5CFE0EEF5E02D
:104D20008491882341F09091C00095FFFCCF80933F
:104D3000C6003196F5CF40919C0850919D08609136
:104D40009E0870919F082AE030E084E995E0B5D88C
:104D50008091C00085FFFCCF8AE08093C60005DE0D
:104D600012CF20E0D12CF301E20FF11DE95EF84FE4
:104D700030813A3219F02F5FD326F5CF9093080790
:104D80008093070784199509860D971D60E070E0F0
:104D9000885E984F0E9431B70E9468B32D2D30E095
:104DA0002617370709F4F4CEE1EAF7E08491882367
:104DB00041F09091C00095FFFCCF8093C6003196E2
:104DC000F5CFEAE0F6E08491882341F09091C000AD
:104DD00095FFFCCF8093C6003196F5CF40919C089B
:104DE00050919D0860919E0870919F082AE030E0E4
:104DF00084E995E062D88091C00085FFFCCFACCFFC
:104E0000E1EAF7E08491882341F09091C00095FF9A
:104E1000FCCF8093C6003196F5CFE9E2F6E08491AD
:104E2000882341F09091C00095FFFCCF8093C6008D
:104E30003196F5CF40919C0850919D0860919E0855
:104E400070919F082AE030E084E995E036D880919F
:104E5000C00085FFFCCF80CF80910D09882389F0A9
:104E600080910A0790910B07892B59F4A0E6EA2E4E
:104E7000FF24F394C4E0D0E00BE115E0BAE0DB2EB0
:104E8000AFC08091FF08882309F4FCC0809100091D
:104E900087FDF8C08068809300098EE295E0DF917D
:104EA000CF911F910F91FF90EF90DF90CF90BF9027
:104EB000AF909F907F906F905F904F901FCB8091AD
:104EC0000D0790910E0704970CF0DCC08091E70964
:104ED0009091E809A091E909B091EA098093020A4A
:104EE0009093030AA093040AB093050A8FED99E00A
:104EF0000E94D057482F80930C078A3019F04D300C
:104F000009F085C04091020A5091030A6091040A99
:104F10007091050A8091FA099091FB09A091FC0912
:104F2000B091FD09481759076A077B0738F1F80166
:104F30008491EBE1F5E081117EC08091C00085FF96
:104F4000FCCFD092C60081E195E00E942E85F092C0
:104F5000F9081092FC080E940BAC6093F70670935E
:104F6000F8068093F9069093FA068BE099E00E9488
:104F7000871A61E08BE099E00E94A61820910A0749
:104F800030910B072115310509F4A9CE80910F0747
:104F900090911007E89EF001E99EF00D1124E20FB8
:104FA000F31FE95EF84F1082FC01ED5EF84FF082CE
:104FB00020910D0730910E072F5F3F4F30930E0762
:104FC00020930D070196BE010E94B7B6909310077B
:104FD00080930F071092090710920B0710920A078F
:104FE0004091020A5091030A6091040A7091050AE7
:104FF0008091FA099091FB09A091FC09B091FD09FB
:10500000481759076A077B0708F03CC058CF4A3356
:1050100029F420910907222309F474CF20910A076B
:1050200030910B072F3531050CF06CCF8F3FFFEF20
:105030009F0751F467CF9091C00095FFFCCF8093FC
:10504000C6003196849177CF4B3311F4F092090763
:10505000409109074111C4CF40910F0750911007AB
:10506000B9016F5F7F4F70930B0760930A07E49E4F
:10507000F001E59EF00D1124E20FF31FE95EF84FF9
:105080008083AECFDF91CF911F910F91FF90EF9072
:10509000DF90CF90BF90AF909F907F906F905F9088
:1050A0004F9008958F929F92AF92BF92CF92DF92CE
:1050B000EF92FF920F931F93CF93DF9327E0E22E9F
:1050C00024E0F22E03EE18E0C8EBD8E035EFC32E53
:1050D00038E0D32EF70181917F0103DC882311F1A1
:1050E000ECDB4B015C01F6018081811103C0609112
:1050F000970801C061E070E080E090E00E949BB3FF
:10510000F80120813181428153810E94CEB59B01FB
:10511000AC01C501B4010E9420B2688379838A83FF
:105120009B8309C0F80180819181A281B38188832A
:105130009983AA83BB830C5F1F4F2496FFEFCF1A7E
:10514000DF0A8BE0E81684E0F80621F686E4C9DB86
:105150008823D1F0B2DB6B017C016093A8087093C7
:10516000A9088093AA089093AB0820E030E0A90139
:105170000E94FCB4181644F4C0920B02D0920C02A8
:10518000E0920D02F0920E02DF91CF911F910F91EC
:10519000FF90EF90DF90CF90BF90AF909F908F9057
:1051A000089580DF89E49DDB882351F086DB6093DE
:1051B000AC087093AD088093AE089093AF0808C018
:1051C0001092AC081092AD081092AE081092AF0881
:1051D0008AE487DB882351F070DB6093B00870931A
:1051E000B1088093B2089093B30808951092B00864
:1051F0001092B1081092B2081092B3080895CF929D
:10520000DF92EF92FF92CF93DF93EC01C090CB0837
:10521000D090CC08E090CD08F090CE08A701960180
:10522000688179818A819B810E94F9B287FF04C0DD
:10523000C882D982EA82FB82C090CF08D090D00881
:10524000E090D108F090D208A70196016C817D8191
:105250008E819F810E94F9B287FF04C0CC82DD82DB
:10526000EE82FF82C090D308D090D408E090D50899
:10527000F090D608A7019601688579858A859B8577
:105280000E94F9B287FF04C0C886D986EA86FB86E9
:10529000C0902002D0902102E0902202F0902302E0
:1052A000A7019601688179818A819B810E94FCB463
:1052B000181624F4C882D982EA82FB82C0902402A4
:1052C000D0902502E0902602F0902702A7019601D7
:1052D0006C817D818E819F810E94FCB4181624F41C
:1052E000CC82DD82EE82FF82C0902802D09029021B
:1052F000E0902A02F0902B02A7019601688579853B
:105300008A859B850E94FCB4181624F4C886D98629
:10531000EA86FB86DF91CF91FF90EF90DF90CF90F0
:105320000895CF92DF92EF92FF920F931F93809197
:10533000F606811103C088EB98E061DF0E940BAC98
:105340006093030770930407809305079093060703
:105350002091B8083091B9084091BA085091BB0823
:105360006091E3087091E4088091E5089091E60867
:105370000E94F9B2811179C02091BC083091BD081A
:105380004091BE085091BF086091E7087091E8080D
:105390008091E9089091EA080E94F9B2811165C0F4
:1053A00020E030E040E752E460910B0270910C0283
:1053B00080910D0290910E020E9400B34AECC42E1F
:1053C00048E0D42E7B018C0124EC38E040EC58E01E
:1053D0006CEB78E088EB98E00E9471488091B80807
:1053E0009091B908A091BA08B091BB088093E308E6
:1053F0009093E408A093E508B093E6088091BC0878
:105400009091BD08A091BE08B091BF088093E708B5
:105410009093E808A093E908B093EA088091C00847
:105420009091C108A091C208B091C3088093EB0885
:105430009093EC08A093ED08B093EE088091C40817
:105440009091C508A091C608B091C7088093EF0855
:105450009093F008A093F108B093F2081F910F9178
:10546000FF90EF90DF90CF90089560912E027091A1
:105470002F02882777FD8095982F0E949BB320915B
:105480000B0230910C0240910D0250910E020E94CD
:10549000CEB520E030E040E752E40E9400B320E0C7
:1054A00030E048EC52E488CFAF92BF92CF92DF92C7
:1054B000EF92FF920F931F93CF93DF93D82F2091FA
:1054C000B0083091B1084091B2085091B308609192
:1054D000AC087091AD088091AE089091AF080E9421
:1054E00009B5C62F172F082FF92E60912E02709143
:1054F0002F02882777FD8095982F0E949BB32091DB
:105500000B0230910C0240910D0250910E020E944C
:10551000CEB520E030E040E752E40E9400B320E046
:1055200030E048EC52E40E9400B32091CA082F9367
:10553000DF93FF920F931F93CF935B016C0152E0B7
:10554000E52E01E020E04CEA58E068EB78E083EEDD
:1055500098E00E943E408091B8089091B908A091CF
:10556000BA08B091BB088093E3089093E408A09335
:10557000E508B093E6088091BC089091BD08A09121
:10558000BE08B091BF088093E7089093E808A09305
:10559000E908B093EA088091C0089091C108A091F1
:1055A000C208B091C3088093EB089093EC08A093D5
:1055B000ED08B093EE088091C4089091C508A091C1
:1055C000C608B091C7088093EF089093F008A093A5
:1055D000F108B093F2080E940BAC6093030770933C
:1055E000040780930507909306070F900F900F9084
:1055F0000F900F900F90DF91CF911F910F91FF901F
:10560000EF90DF90CF90BF90AF9008952091FD086C
:1056100021111092FF088091F9088D30E1F48091FA
:10562000090990910A09843F31E0930709F42C9805
:10563000813D974020F010920A091092090980914B
:10564000090990910A09009709F42C9A0196909300
:105650000A09809309098091F9088D7F813031F41E
:10566000222321F08091050981112C988091FF0857
:10567000882329F180910D09882319F19CB1929515
:105680009170309103012091FE0880910009213032
:1056900039F0223081F4911105C030FD03C00BC0F8
:1056A000992349F08160809300098091F908823044
:1056B00041F40C94AB858078809300090895109292
:1056C00000090895F8940E947D6F5F9A8A9A9FB7A7
:1056D000F894809108018160809308019FBF129A1D
:1056E000479A60E08CE00E94D9ADE1EAF7E084914E
:1056F000882341F09091C00095FFFCCF8093C600B5
:105700003196F5CFE9E4F3E08491882341F090915C
:10571000C00095FFFCCF8093C6003196F5CF8091F5
:10572000C00085FFFCCF8AE08093C60080E493E050
:105730000E94BC85FFCFCF92DF92EF92FF920F9332
:105740001F930E940BAC0091FF061091000720915F
:10575000010730910207C0900307D0900407E09042
:105760000507F09006076C197D098E099F09061739
:1057700017072807390728F4012B022B032B09F000
:10578000A1DF8091070290910802A0910902B091D7
:105790000A02892B8A2B8B2BC9F18091F90887305B
:1057A000D1F40E940BAC00910307109104072091E3
:1057B000050730910607601B710B820B930B653C4C
:1057C00079408105910510F19091120A8091110A9A
:1057D00098131CC027C00E940BAC009103071091C6
:1057E00004072091050730910607601B710B820B9F
:1057F000930B009107021091080220910902309149
:105800000A02061717072807390780F0809106015A
:1058100082FFB6CF1F910F91FF90EF90DF90CF9056
:105820000C94544881E08093ED06F0CF9091120AD9
:105830008091110A9813EACF5F9A8A9A9FB7F894D9
:10584000809108018160809308019FBF129A479A56
:10585000DDCFCF93DF93EC018091CA0880931A06C5
:1058600084E53FD8811102C080E064C026D80E9440
:105870006DB360931A066230B8F3EBE9F7E08491F8
:10588000882341F09091C00095FFFCCF8093C60023
:105890003196F5CFC936D10599F034F4C836D10523
:1058A000C9F5ECE4F3E015C0CD36D10531F0CA3DC1
:1058B000D10581F5E7E0F3E02AC0EEE1F3E01DC099
:1058C000E5E3F3E010C09091C00095FFFCCF80931A
:1058D000C60081918111F7CF1DC09091C00095FF46
:1058E000FCCF8093C60081918111F7CF13C09091B6
:1058F000C00095FFFCCF8093C60081918111F7CF46
:1059000009C09091C00095FFFCCF8093C6008191A3
:105910008111F7CF40E050E060911A0684E995E0EC
:105920000E94B71F8091C00085FFFCCF8AE0809362
:10593000C60081E0DF91CF9108953F924F925F9230
:105940006F927F928F929F92AF92BF92CF92DF928F
:10595000EF92FF920F931F93CF93DF93CDB7DEB7F4
:10596000A2970FB6F894DEBF0FBECDBF87E40E94AA
:105970007124882309F4C5C30E945D240E9468B382
:105980006A35710509F4A2C2ACF46230710509F4FC
:10599000B8C024F477FFADC00C94F23D64307105BB
:1059A00009F4BFC00CF4B4C06C31710509F400C136
:1059B0000C94F23D6636710509F466C30CF051C0D3
:1059C0006C35710509F48BC20CF484C2653671051F
:1059D00011F00C94F23D84E095E00E947E226091EB
:1059E0000209709103098091060990910709680FD7
:1059F000791F6B537109882777FD8095982F0E9436
:105A00009BB36093EB087093EC088093ED08909340
:105A1000EE08198220E030E040EA50E4609138025C
:105A20007091390280913A0290913B020E9400B33A
:105A3000FE0131966F017B018C012FEE38E04BEEB9
:105A400058E067EE78E083EE98E00E9471480E948B
:105A5000726A8DE08093F9088EE0809308090C94B7
:105A6000F23D623421E0720709F413C3683E33E06B
:105A7000730709F4A6C26134714011F00C94F23D31
:105A800020E030E040E251E46091EB087091EC08D6
:105A90008091ED089091EE080E9420B26093EB088F
:105AA0007093EC088093ED089093EE08198220E043
:105AB00030E040EA50E46091380270913902809100
:105AC0003A0290913B020E9400B39E012F5F3F4F2C
:105AD00069017B018C012FEE38E04BEE58E067EE58
:105AE00078E083EE98E00E9471480E94726A0C94FC
:105AF000F23D80911906811104C0D4DA12DC0C94B5
:105B0000893F80911906811103C04BDB81E006C0FB
:105B100080911906811105C044DB80E0C5DC0C943E
:105B2000893F88E095E00E942E8580E50E947124DF
:105B3000882339F00E945D240E946DB34B015C0103
:105B400003C0812C912C540183E50E947124882389
:105B500061F00E945D2420E030E04AE754E40E94B6
:105B6000CEB50E946DB34B015C010E94726A0E9427
:105B70000BAC6B017C01C80CD91CEA1CFB1C0E94FD
:105B80000BAC609303077093040780930507909311
:105B900006070E940BAC6C157D058E059F0510F065
:105BA0000C94F23D0E948C6CC6DD0E944486F1CFBD
:105BB00080910B0290910C02A0910D02B0910E0207
:105BC0008093A4089093A508A093A608B093A70873
:105BD00080912E0290912F029093F4088093F30805
:105BE00084E690E090932F0280932E020E940BACEB
:105BF000609303077093040780930507909306074B
:105C000081E00E9442638091E3089091E408A091B2
:105C1000E508B091E6088093B8089093B908A0937E
:105C2000BA08B093BB088091E7089091E808A0916A
:105C3000E908B091EA088093BC089093BD08A0934E
:105C4000BE08B093BF088091EB089091EC08A0913A
:105C5000ED08B091EE088093C0089093C108A0931E
:105C6000C208B093C3088091EF089091F008A0910A
:105C7000F108B091F2088093C4089093C508A093EE
:105C8000C608B093C70810920B0210920C02109233
:105C90000D0210920E0288E50E947124882311F0F3
:105CA00090E00AC089E50E9471248111F9CF8AE54C
:105CB0000E94712491E0982790930F02992309F490
:105CC0004BC020E030E0A9016091E3087091E40846
:105CD0008091E5089091E6080E94F9B281113CC0DC
:105CE00080E090E0A0EAB0E48093E3089093E408B9
:105CF000A093E508B093E6086091300270913102FC
:105D0000809132029091330260930B0270930C02E7
:105D100080930D0290930E0220E030E040E752E4C1
:105D20000E9400B32AECC22E28E0D22E7B018C0107
:105D30002FEE38E04BEE58E067EE78E083EE98E027
:105D40000E9471480E94726A1092E3081092E4085F
:105D50001092E5081092E60880910F0281110C94D0
:105D6000F53D89E50E94712481110C94F53D8091E7
:105D70000F0281110C94FB3D88E50E947124811172
:105D80000C94FB3D80910F0281110C94013E8AE539
:105D90000E94712481110C94013E88E50E947124B7
:105DA0008823D1F00E946624672B682B692BA1F011
:105DB0000E945D242091D7083091D8084091D908DD
:105DC0005091DA080E9420B26093E3087093E408CF
:105DD0008093E5089093E60889E50E947124882362
:105DE000D1F00E946624672B682B692BA1F00E94DA
:105DF0005D242091DB083091DC084091DD08509152
:105E0000DE080E9420B26093E7087093E808809350
:105E1000E9089093EA088AE50E9471248823D1F06A
:105E20000E946624672B682B692BA1F00E945D24D9
:105E30002091DF083091E0084091E1085091E2089C
:105E40000E9420B26093EB087093EC088093ED08F9
:105E50009093EE082FEE38E04BEE58E067EE78E0D6
:105E600083EE98E00E94FD5180E00E9442638091A1
:105E7000A4089091A508A091A608B091A7088093C6
:105E80000B0290930C02A0930D02B0930E0280912E
:105E9000F3089091F40890932F0280932E020E94B1
:105EA0000BAC6093030770930407809305079093EE
:105EB00006070E943B638091F908853011F00C942D
:105EC000F23D86E08093F9080C94F23D1092970819
:105ED0000C94F23D81E0809397080C94F23D85E4A8
:105EE0000E947124811102C00E94726A17E0C12EC3
:105EF00014E0D12E07EDE02E08E0F02E03EE18E0BE
:105F0000B12CD6018D916D010E947124882309F472
:105F10004DC0B3E0BB1232C08091F606882311F168
:105F2000809106028230F1F42091CA088091EF0836
:105F30009091F008A091F108B091F208222349F065
:105F40008093EE069093EF06A093F006B093F106CF
:105F50002DC08093F2069093F306A093F406B093BD
:105F6000F50624C00E945D24F8016083718382835A
:105F700093838FEE98E00E94A25218C00E945D2485
:105F8000D7012D913D914D915C910E9420B2F80175
:105F900060837183828393832FEE38E04BEE58E069
:105FA00067EE78E083EE98E00E94FD51B394F4E050
:105FB000EF0EF11C0C5F1F4F24E0B212A2CF0C9425
:105FC000F23D8FE0809308091092E3081092E408F4
:105FD0001092E5081092E6082FEE38E04BEE58E0FC
:105FE00067EE78E083EE98E00E94FD511092E7089A
:105FF0001092E8081092E9081092EA082FEE38E0B3
:106000004BEE58E067EE78E083EE98E00E94FD5199
:106010006091020970910309809106099091070926
:10602000680F791F63517109882777FD8095982F34
:106030000E949BB36093EB087093EC088093ED088B
:106040009093EE08198220E030E040EA50E460913D
:1060500038027091390280913A0290913B020E947D
:1060600000B3DE0111966D017B018C012FEE38E04B
:106070004BEE58E067EE78E083EE98E00E947148BE
:106080000E94726A0C94F23D81E0809304090C94A2
:10609000F23D20E030E040E251E46091EB08709185
:1060A000EC088091ED089091EE080E941FB2609379
:1060B000EB087093EC088093ED089093EE0819823A
:1060C00020E030E040EA50E46091380270913902FB
:1060D00080913A0290913B020E9400B3DE0111963A
:1060E0006D017B018C012FEE38E04BEE58E067EE3E
:1060F00078E083EE98E00E9471480E94726A0C94E6
:10610000F23D88E50E947124882309F454C00E945E
:106110005D240E9468B362307105F9F06330710547
:1061200099F16130710511F00C94F23D81E080939A
:10613000F606809306021092F2061092F306109271
:10614000F4061092F5061092EE061092EF061092E9
:10615000F0061092F1060C94F23D8EE40E94712438
:10616000882311F40C94F23D0E945D240E9468B3D0
:106170006230710514F40C94F23D809106028F5F39
:10618000809306020C94F23D1092F60681E0809313
:1061900006021092F2061092F3061092F406109284
:1061A000F5061092EE061092EF061092F00610928D
:1061B000F1060C94F23D8DE40E947124882311F4C1
:1061C0000C947D3C0E945D240E9468B36D3671057D
:1061D00009F4B3C40CF0D9C06C31710509F471C273
:1061E0000CF041C06431710509F4F8C1FCF463306E
:1061F000710509F4D9C134F46230710508F47AC12B
:106200000C94F23D6131710509F4D6C1623171051A
:1062100009F409C66530710511F00C94F23D0E9435
:10622000726A2C98109205090C94F23D6831710540
:1062300009F420C264F46631710509F4FDC10CF063
:1062400001C28BE099E00E94EF130C94F23D6A3199
:10625000710509F422C20CF02EC28BE099E00E9475
:10626000BF140C94F23D6335710509F4D8C50CF0E8
:106270005BC06A32710509F417C30CF046C06E3179
:10628000710509F453C26F31710511F00C94F23DA0
:106290000E940BAC6093F7067093F8068093F906A2
:1062A0009093FA060091FB061091FC062091FD06E2
:1062B0003091FE06601B710B820B930B28EE33E0CE
:1062C00040E050E00E94CAB6CA01B9012CE330E0B8
:1062D00040E050E00E94CAB67F936F933F932F93A4
:1062E00080EB94E09F938F93CE0101969F938F93C1
:1062F0000E94B7BAEBE9F7E084910FB6F894DEBFDD
:106300000FBECDBFEBE9F7E08BC26135710509F433
:1063100080C50CF081C56035710511F00C94F23D1B
:10632000269A2E980C94F23D6836710509F4E7C25E
:10633000DCF46535710509F4AFC50CF474C56C3532
:10634000710511F00C94F23D27E034E038A32F8F53
:1063500004E41FE0E4E58E2EEFE09E2EF8E0AF2E81
:10636000FFE0BF2E312C0FC66A36710509F423C534
:106370000CF4F4C26B36710511F00C94F23D1092DE
:10638000C9081092C8080C94F23D6C3D710511F4D7
:106390000C94DB3A0CF047C06C38710509F4CDC29F
:1063A0000CF56537710509F40BC664F462377105A5
:1063B00009F427C66337710511F00C94F23DEDEC3A
:1063C000F3E0FAC56837710509F4FAC66937710553
:1063D00009F4FAC66737710511F00C94F23DE2E753
:1063E000F3E0FCC66C3C710509F4B0C774F4693C79
:1063F000710509F46FC76B3C710509F48BC76E3BDF
:10640000710511F00C94F23D19C46E3C710511F444
:106410000C94243A0CF4BAC76A3D710511F40C943B
:10642000403A0C94F23D643FB1E07B0711F40C94C8
:10643000333C2CF56D32F1E07F0711F40C94273BCF
:1064400064F46D3D710511F40C94EA3A6C327140BC
:1064500011F40C94F93A0C94F23D6F3281E0780714
:1064600011F40C94FB3B14F40C94ED3B6039714037
:1064700011F00C94F23D0E94726A0C94F23D673E5A
:10648000B3E07B0711F40C943C3C7CF4663FF1E0F4
:106490007F0711F40C94393C14F40C94363C603AA8
:1064A000734009F481C10C94F23D693E83E07807A2
:1064B00011F40C94693C14F40C94533C6A3E734000
:1064C00011F00C94F23D1092F60681E080930602E2
:1064D0001092F2061092F3061092F4061092F5064E
:1064E0001092EE061092EF061092F0061092F1064E
:1064F0000C94F23D83EF94E00E942E8580E50E948B
:106500007124882339F00E945D240E946DB36B01D1
:106510007C0103C0C12CD12C760183E50E9471243B
:10652000882361F00E945D2420E030E04AE754E4D3
:106530000E94CEB50E946DB36B017C010E94726A0D
:106540000E940BAC609303077093040780930507C8
:1065500090930607C114D104E104F104A9F00E944C
:106560000BAC4B015C018C0C9D1CAE1CBF1C0E9433
:106570000BAC681579058A059B0580F40E944A8753
:1065800081110CC00C94073E0E944A87811106C0FD
:106590000E948C6CD0D80E944486F6CF86EE94E0A0
:1065A0000E942E850C94F23D0E94726A2C9A81E022
:1065B000809305090C94F23D8DED94E00E942E85A8
:1065C0005F988A989FB7F894809108018E7F809396
:1065D00008019FBF129847980C94F23DEDECF4E04F
:1065E0008491882341F09091C00095FFFCCF809367
:1065F000C6003196F5CF8091C00085FFFCCF8AE0C0
:106600008093C6008BE099E00E949913EFEBF4E0D1
:106610008491882341F09091C00095FFFCCF809336
:10662000C6003196F5CF8091C00085FFFCCF8AE08F
:106630008093C6000C94F23D8BE099E00E94B41464
:106640000C94F23D00910707109108070C5F1F4F53
:106650006AE270E0C8010E944CBA009719F0FC0190
:106660003197108241E0B8018BE099E00E94C41498
:106670000C94F23D8BE099E00E94B8140E940BACA0
:106680006093FB067093FC068093FD069093FE06D4
:1066900082E08093F9080C94F23D80910E098823E2
:1066A00011F40C94F23D83E50E94712481110C9445
:1066B0000F3E0C94F23D8BE099E00E94E3170C949E
:1066C000F23D80910707909108076AE270E0049616
:1066D0000E944CBA8C010097E1F020911107309193
:1066E000120740E6429FC001439F900D11246EE4C3
:1066F00070E0895E984F0E944CBA60E270E00E94A0
:106700004CBA01969093080780930707F8013197D8
:10671000108260910707709108076C5F7F4F40E01F
:106720008BE099E00E94C4140C94F23D80910E0914
:10673000882311F40C94F23D8BE099E00E949A19A1
:1067400080910707909108076AE270E004960E9422
:106750004CBA8C010097E1F020911107309112079B
:1067600040E6429FC001439F900D11246EE470E00B
:10677000895E984F0E944CBA60E270E00E944CBA69
:1067800001969093080780930707F80131971082CC
:1067900060910707709108076C5F7F4F8BE099E06D
:1067A0000E94AB160C94F23D809107079091080768
:1067B0006AE270E005960E944CBA8C010097E1F005
:1067C000209111073091120740E6429FC001439F7C
:1067D000900D11246EE470E0895E984F0E944CBACF
:1067E00060E270E00E944CBA019690930807809393
:1067F0000707F80131971082609107077091080729
:106800006B5F7F4F8BE099E00E94A6160C94F23DDF
:106810009091C00095FFFCCF8093C6003196849183
:106820008111F6CFFE0131968191882339F0909144
:10683000C00095FFFCCF8093C600F6CF8091C000CA
:1068400085FFFCCF8AE08093C600CE0101960E94AE
:106850001F858091E30E882311F40C94F23D109271
:10686000E30E0091CA0810E0000F111F085C1D4ED6
:10687000D8016D917C91882777FD8095982F0E9493
:106880009BB3209148023091490240914A025091B5
:106890004B020E94FCB4181614F00C94F23DF8015F
:1068A000118210820C94F23D83E50E9471248823AA
:1068B00011F40C94F23D0E945D246B017C0180E593
:1068C0000E947124882351F0C701B6010E9468B369
:1068D0006F3F710509F010F40C94203E6DE070E0FC
:1068E00020E0E22FEE0FFF0BE953FC4F80819181F6
:1068F0008617970711F40C94F23D2F5FF2CF88E6CC
:1069000090E00E94292C81110C94F23D83E50E94B5
:106910007124882371F000911A060E945D2410E012
:10692000000F111F085C1D4E0E9468B3D8016D93C3
:106930007C930E947C6F0C94F23D83E50E9471244D
:10694000882311F40C94F23D0E945D240E9468B3E8
:1069500070933712609336120C94F23D89E690E002
:106960000E94292C81110C94F23DE9EAF4E0849113
:10697000882341F09091C00095FFFCCF8093C60022
:106980003196F5CF40912A1250912B1260912C1222
:1069900070912D1221E030E084E995E00E945620AC
:1069A000E6EAF4E08491882341F09091C00095FFDD
:1069B000FCCF8093C6003196F5CF6091381270916C
:1069C0003912882777FD8095982F0E949BB3AB01E1
:1069D000BC0121E030E084E995E00E945620E1EA24
:1069E000F4E08491882341F09091C00095FFFCCFA2
:1069F0008093C6003196F5CF40912E1250912F1200
:106A0000609130127091311221E030E084E995E01C
:106A10000E945620EEE9F4E08491882341F09091A1
:106A2000C00095FFFCCF8093C6003196F5CF6091F2
:106A30003A1270913B12882777FD8095982F0E941B
:106A40009BB3AB01BC0121E030E084E995E00E94FA
:106A50005620EAE9F4E08491882341F09091C00047
:106A600095FFFCCF8093C6003196F5CF409124125C
:106A700050912512609126127091271221E030E08A
:106A800084E995E00E945620E7E9F4E084918823A8
:106A900041F09091C00095FFFCCF8093C6003196E5
:106AA000F5CF6091361270913712882777FD809567
:106AB000982F0E949BB3AB01BC0121E030E084E938
:106AC00095E00E945620E3E9F4E08491882341F0A8
:106AD0009091C00095FFFCCF8093C6003196F5CF12
:106AE00080911A0690E00E94816C4AE050E0BC015F
:106AF00084E995E00E94801FEEE8F4E08491882309
:106B000041F09091C00095FFFCCF8093C600319674
:106B1000F5CF8FEF9FEF0E94816C4AE050E0BC01FF
:106B200084E995E00E94801F8091C00085FFFCCF22
:106B30008AE08093C6000C94893F8DE690E00E9425
:106B4000292C81110C94F23D83E894E00E942E855B
:106B50001092E30E1092F60683E50E9471248823BA
:106B600071F000911A060E945D2410E0000F111FC1
:106B7000085C1D4E0E9468B3F8017183608383E551
:106B80000E947124882351F00E945D246093480282
:106B90007093490280934A0290934B0282E40E94D0
:106BA0007124882351F00E945D2460934C027093FD
:106BB0004D0280934E0290934F0286E40E9471240E
:106BC000882369F00E945D2460934402709345021B
:106BD000809346029093470281E08093E30E0E94E7
:106BE0007C6F0E940BAC4B015C0100911A0610E017
:106BF000F801EE0FFF1FE85CFD4E60817181882770
:106C000077FD8095982F0E949BB32B013C01F801E2
:106C1000EE0FFF1FEE0FFF1FE65DFD4E808191819D
:106C2000A281B3818F8F98A3A9A3BAA3CC24CA94BD
:106C3000DC2C7601EAE03E2E0C948B3E8BE594E052
:106C40000E942E8583E50E947124882341F00E94D2
:106C50005D240E9468B370933712609336120E94CD
:106C60000BAC4B015C011092F60607E514E0A2E5BF
:106C7000EA2EA4E0FA2EBEE4CB2EB4E0DB2E8AE0AE
:106C8000782E6091361270913712882777FD8095A3
:106C9000982F0E949BB3209124123091251240918D
:106CA0002612509127120E94FCB418160CF074C0E2
:106CB0000E940BAC681979098A099B09693E7340E7
:106CC0008105910508F461C0F8018491E7E5F4E0DD
:106CD000882349F09091C00095FFFCCF8093C600B7
:106CE00031968491F5CF40912A1250912B126091E8
:106CF0002C1270912D1222E030E084E995E00E9480
:106D00005620F7018491E2E5F4E0882349F0909160
:106D1000C00095FFFCCF8093C60031968491F5CFDB
:106D200040912E1250912F126091301270913112B9
:106D300022E030E084E995E00E945620F60184913B
:106D4000EEE4F4E0882349F09091C00095FFFCCF79
:106D50008093C60031968491F5CF409124125091D2
:106D60002512609126127091271221E030E084E90B
:106D700095E00E9456208091C00085FFFCCF709264
:106D8000C6000E940BAC4B015C010E948C6C0E94FF
:106D90009B2B0E94448675CF84E494E00E942E854C
:106DA0000E940BAC60930307709304078093050760
:106DB0009093060717C783E50E947124882311F179
:106DC0000E945D2420E030E0A9010E94F9B287FD15
:106DD0000FC00E945D2420E030E04FE753E40E94A2
:106DE000FCB4181644F00E945D240E9468B305C0EC
:106DF00060E070E002C06FEF70E07093C9086093CC
:106E0000C808F0C68FEF90E09093C9088093C80837
:106E1000E9C6269A2E9AE6C61092F808E3C681E0E3
:106E20008093F808DFC683E50E947124882399F0D7
:106E30000E945D2420E030E04AE754E40E94CEB591
:106E40000E946DB360930702709308028093090259
:106E500090930A021EC088E50E94712481110C944F
:106E6000653F89E50E94712481110C94653F8AE594
:106E70000E94712481110C94653F85E40E94712465
:106E800081110C94653F0E94726A129A479A0E947F
:106E9000DA6A1092FC08A6C683E50E9471240E945B
:106EA0005D2420E030E04AE754E40E94CEB50E9421
:106EB0006DB36093FF067093000780930107909372
:106EC000020790C6B3E03B1268C00E945D246B01CC
:106ED0007C0120E030E040EA51E40E94F9B287FFF3
:106EE0003FC0A7019601F801608171818281938181
:106EF0000E9400B32B013C019B01AC0160911C0F6F
:106F000070911D0F80911E0F90911F0F0E94CEB5A2
:106F100060931C0F70931D0F80931E0F90931F0F93
:106F2000A3019201D4016D917D918D919C910E945C
:106F3000CEB5F4016083718382839383D5016D9113
:106F40007D918D919C910E9499B3A30192010E9421
:106F5000CEB50E946DB3F501608371838283938304
:106F6000D801CD92DD92ED92FC92139733940C5F91
:106F70001F4FF4E08F0E911C24E0A20EB11C34E0F0
:106F8000331609F42FC6AF8DB8A18D91B8A3AF8F7A
:106F90000E947124882351F395CF0E945D24F8014B
:106FA0006083718382839383E1CF9091C00095FFCA
:106FB000FCCF8093C600319684918111F6CF12C622
:106FC00000910707109108070B5F1F4F6AE270E0FE
:106FD000C8010E944CBA009719F0FC013197108249
:106FE000C8010E941F850E940BAC6093FB06709342
:106FF000FC068093FD069093FE0681E08093FC08DA
:10700000F1C5EAECF3E08491882341F09091C0004F
:1070100095FFFCCF8093C6003196F5CF4091E308F1
:107020005091E4086091E5087091E60822E030E0B4
:1070300084E995E00E945620E7ECF3E084918823F0
:1070400041F09091C00095FFFCCF8093C60031962F
:10705000F5CF4091E7085091E8086091E9087091F8
:10706000EA0822E030E084E995E00E945620E4EC52
:10707000F3E08491882341F09091C00095FFFCCF0C
:107080008093C6003196F5CF4091EB085091EC0803
:107090006091ED087091EE0822E030E084E995E01F
:1070A0000E945620E1ECF3E08491882341F0909116
:1070B000C00095FFFCCF8093C6003196F5CF40917C
:1070C000EF085091F0086091F1087091F20822E009
:1070D00030E084E995E00E945620E7EBF3E08491EC
:1070E000882341F09091C00095FFFCCF8093C600AB
:1070F0003196F5CF0E94CC6A0E949BB32091440F39
:107100003091450F4091460F5091470F0E9400B3B8
:10711000AB01BC0122E030E084E995E00E945620FA
:10712000E4EBF3E08491882341F09091C00095FF57
:10713000FCCF8093C6003196F5CF81E00E94CC6AE7
:107140000E949BB32091480F3091490F40914A0F04
:1071500050914B0F0E9400B3AB01BC0122E030E024
:1071600084E995E00E945620E1EBF3E084918823C6
:1071700041F09091C00095FFFCCF8093C6003196FE
:10718000F5CF82E00E94CC6A0E949BB320914C0F05
:1071900030914D0F40914E0F50914F0F0E9400B310
:1071A000AB01BC0122E030E084E995E00E9456206A
:1071B0008091C00085FFFCCF8AE08093C60012C595
:1071C00080E00E9442630EC581E00E9442630AC5CE
:1071D0009091C00095FFFCCF8093C60081918111F2
:1071E000F7CF8091C00085FFFCCF8AE08093C60076
:1071F000E9EAF3E08491882341F09091C00095FF83
:10720000FCCF8093C6003196F5CF659903C0E3E6C5
:10721000F3E009C0EDE6F3E006C09091C00095FFF1
:10722000FCCF8093C60081918111F7CF8091C0007F
:1072300085FFFCCF8AE08093C600E1EAF3E0849109
:10724000882341F09091C00095FFFCCF8093C60049
:107250003196F5CF8091030181FD03C0E3E6F3E0B1
:1072600009C0EDE6F3E006C09091C00095FFFCCFA9
:107270008093C60081918111F7CF8091C00085FF76
:10728000FCCF8AE08093C600E9E9F3E0849188238B
:1072900041F09091C00095FFFCCF8093C6003196DD
:1072A000F5CF4B9903C0E3E6F3E009C0EDE6F3E068
:1072B00006C09091C00095FFFCCF8093C6008191DD
:1072C0008111F7CF8091C00085FFFCCF8AE08093C9
:1072D000C60088C407E014E074E3E72E7FE0F72ED1
:1072E000D8018D918D010E947124882349F00E945C
:1072F0005D240E946DB3F701608371838283938361
:10730000F4E0EF0EF11C24E00B30120749F70E9465
:10731000C85268C407E014E064E5E62E6FE0F62E7C
:10732000D8018D918D010E947124882339F00E942B
:107330005D24F7016083718382839383F4E0EF0E11
:10734000F11C24E00B30120759F74CC483E50E946E
:107350007124882351F00E945D2460932C0F709358
:107360002D0F80932E0F90932F0F84E50E94712490
:10737000882309F437C40E945D246093280F70931A
:10738000290F80932A0F90932B0F2CC483E50E9422
:107390007124882351F00E945D246093300F709314
:1073A000310F8093320F9093330F84E50E94712444
:1073B000882351F00E945D246093180F7093190F79
:1073C00080931A0F90931B0F82E40E9471248823EC
:1073D00061F00E945D240E946DB36093640F70930E
:1073E000650F8093660F9093670F88E50E94712464
:1073F000882351F00E945D246093240F7093250F21
:107400008093260F9093270F8AE50E94712488238A
:1074100051F00E945D246093200F7093210F8093A0
:10742000220F9093230F85E40E947124882309F48E
:10743000D9C30E945D2460931C0F70931D0F80932D
:107440001E0F90931F0FCEC307E014E057EDE52EFB
:1074500058E0F52ED8018D918D010E94712488236A
:1074600039F00E945D24F7016083718382839383E6
:10747000F4E0EF0EF11C24E00A30120759F7B2C312
:107480008AED90E00E94292C8111ACC388E50E940E
:107490007124882381F000911A0610E00E945D2477
:1074A000F801EE0FFF1FEE0FFF1FE05FFD4F60833F
:1074B00071838283938389E50E947124882381F0FC
:1074C00000911A0610E00E945D24F801EE0FFF1FE4
:1074D000EE0FFF1FE85EFD4F60837183828393830D
:1074E000EBE9F7E08491882341F09091C00095FF8B
:1074F000FCCF8093C6003196F5CFE9E8F3E08491A4
:10750000882341F09091C00095FFFCCF8093C60086
:107510003196F5CF10921A0680911A06823008F043
:1075200042C0E2EEF4E08191882339F09091C000EE
:1075300095FFFCCF8093C600F6CFE0911A0634E0A9
:10754000E39FF0011124E05FFD4F40815181628192
:10755000738122E030E084E995E00E945620EDE856
:10756000F3E08191882339F09091C00095FFFCCF22
:107570008093C600F6CFE0911A0684E0E89FF00100
:107580001124E85EFD4F408151816281738122E0C8
:1075900030E084E995E00E94562080911A068F5FC2
:1075A00080931A06B9CF8091C00085FFFCCF8AE096
:1075B0008093C60017C383E50E947124882309F4D1
:1075C00011C30E945D240E9468B370932F026093E0
:1075D0002E0208C383E50E947124882309F402C3A4
:1075E0000E945D240E9468B370932D0260932C0268
:1075F000F9C283E50E947124882331F00E945D2442
:107600000E9468B38B0102C000E911E080E50E948E
:107610007124882331F00E945D240E9468B37B01AD
:1076200004C028EEE22E23E0F22E20E030E0A90193
:10763000B80185E20E949BAEB701882777FD80954F
:10764000982F0E943AAC85E20E94ACB1CBC280E593
:107650000E947124882351F00E945D2460936A0285
:1076600070936B0280936C0290936D0289E40E9488
:107670007124882361F00E945D240E942975609323
:10768000660270936702809368029093690284E4B3
:107690000E947124882361F00E945D240E94357548
:1076A0006093620270936302809364029093650218
:1076B00083E40E947124882351F00E945D2460932A
:1076C0005E0270935F0280936002909361020E9459
:1076D000626CEFE8F3E08191882339F09091C0006B
:1076E00095FFFCCF8093C600F6CFE2E9F3E08191ED
:1076F000882339F09091C00095FFFCCF8093C6009D
:10770000F6CF40916A0250916B0260916C027091C9
:107710006D0222E030E084E995E00E945620E6E91F
:10772000F3E08191882339F09091C00095FFFCCF60
:107730008093C600F6CF60916602709167028091D7
:107740006802909169020E942F75AB01BC0122E092
:1077500030E084E995E00E945620EAE9F3E0819167
:10776000882339F09091C00095FFFCCF8093C6002C
:10777000F6CF6091620270916302809164029091F1
:1077800065020E943B75AB01BC0122E030E084E958
:1077900095E00E945620EEE9F3E08191882339F0CC
:1077A0009091C00095FFFCCF8093C600F6CF40912A
:1077B0005E0250915F02609160027091610222E06E
:1077C00030E084E995E00E9456208091C00085FF5A
:1077D000FCCF8AE08093C60005C283E50E94712435
:1077E000882319F00E945D2403C060E070E0CB01A3
:1077F0000E94BF52F7C185E40E947124882341F0A2
:107800000E945D240E9468B38B0177FD0AC002C00C
:1078100000E010E0C12CD12C96E1E92E93E4F92E82
:1078200006C0C12CD12C8CE8E82E82E4F82E83E52A
:107830000E947124882321F00E945D246B017C0149
:1078400083E40E947124882331F00E945D240E9409
:1078500068B39B0102C025E030E0A801C701B60172
:107860000E94A36FBFC10E94091BBCC10E94561D8C
:10787000B9C10E94E91BB6C1109219060E94C285C7
:107880008091980890919908A0919A08B0919B08CE
:1078900080939C0890939D08A0939E08B0939F08A6
:1078A0000E94B5249FC181E08093F6068093060272
:1078B0001092F2061092F3061092F4061092F5065A
:1078C0001092EE061092EF061092F0061092F1065A
:1078D00089C18EE40E947124882309F483C10E9427
:1078E0005D240E9468B3623071050CF47BC1809105
:1078F00006028F5F8093060275C184E50E947124A1
:10790000882309F42BC10E945D240E946DB360930B
:107910001A066230A8F1EBE9F7E08491882341F080
:107920009091C00095FFFCCF8093C6003196F5CFB3
:10793000E2EAF3E08191882339F09091C00095FF4D
:10794000FCCF8093C600F6CF40E050E060911A066D
:1079500084E995E00E94B71FE4EAF3E0819188236F
:1079600039F09091C00095FFFCCF8093C600F6CF10
:107970008091C00085FFFCCF8AE08093C60032C1B1
:107980008091F6068823D9F0662349F08091EE06AF
:107990009091EF06A091F006B091F10608C0809199
:1079A000F2069091F306A091F406B091F50680934B
:1079B000EF089093F008A093F108B093F20886E4E2
:1079C0000E9471248823E1F00E945D246B017C01F8
:1079D0006093A8087093A9088093AA089093AB08B5
:1079E00020E030E0A9010E94FCB418165CF4C092BB
:1079F0000B02D0920C02E0920D02F0920E0202C035
:107A0000D12C02C0DD24D394C0901A06E090CA089D
:107A1000CE1409F479C080E1E3EEF8E0A8EBB8E019
:107A200001900D928A95E1F78091FC08882309F472
:107A300057C0F12C0C2D10E0F701EE0FFF1FEE0FD9
:107A4000FF1FE05FFD4F20813181428153816091B2
:107A5000E3087091E4088091E5089091E6080E949F
:107A60001FB2F801EE0FFF1FEE0FFF1FE05FFD4F8B
:107A700020813181428153810E9420B26093E308CA
:107A80007093E4088093E5089093E608F701EE0F01
:107A9000FF1FEE0FFF1FE85EFD4F20813181428105
:107AA00053816091E7087091E8088091E90890910E
:107AB000EA080E941FB2F801EE0FFF1FEE0FFF1F32
:107AC000E85EFD4F20813181428153810E9420B2C6
:107AD0006093E7087093E8088093E9089093EA08B8
:107AE000C092CA082FEE38E04BEE58E067EE78E01F
:107AF00083EE98E00E94FD51DD2031F0809119065F
:107B0000811102C00E949129EBE9F7E0849188235A
:107B100041F09091C00095FFFCCF8093C600319654
:107B2000F5CFE5EBF3E08191882339F09091C00027
:107B300095FFFCCF8093C600F6CF6091CA0870E035
:107B40004AE050E084E995E00E94801F8091C000E7
:107B500085FFFCCF8AE08093C60044C0EBE9F7E0E4
:107B60008491882341F09091C00095FFFCCF8093D1
:107B7000C6003196F5CFE6E7F3E08491882341F023
:107B80009091C00095FFFCCF8093C6003196F5CF51
:107B9000809111079091120720E6289FF001299FFC
:107BA000F00D1124E95EF84F8191882339F090910E
:107BB000C00095FFFCCF8093C600F6CFE4E7F3E06A
:107BC0008491882341F09091C00095FFFCCF809371
:107BD000C6003196F5CF8091C00085FFFCCF8AE0CA
:107BE0008093C6000E948D2494C181E090E00E94A1
:107BF0005D200C94B72E80E090E00E945D200C94F4
:107C0000C22E82E090E00E945D200C94CD2E0E9456
:107C10008C6C0E949B2B0E9444860C94B7320E946D
:107C20006624AB01BC014093020A5093030A60939F
:107C3000040A7093050A8FED99E00E949958D2CFFB
:107C40000E945D240E9468B30C9470340E940BACB7
:107C50008B019C01C701B601605F784D8F4F9F4F2C
:107C6000601B710B820B930B28EE33E040E050E079
:107C70000E94CAB6BA01A9012AE030E084E995E081
:107C80000E94AC1F8091C00085FFFCCF3092C600DF
:107C90000E940BAC4B015C010E948C6C0E949B2BE0
:107CA0000E944486FFEFCF16DF06EF06FF0609F0BD
:107CB000ACC02F8D38A149A15AA1C301B2010E94C5
:107CC000FCB4E0911A06F0E08F01000F111F000FC5
:107CD000111F065D1D4EEE0FFF1FE85CFD4E60811B
:107CE000718118160CF079C0882777FD8095982F40
:107CF0000E949BB320E030E040E85FE30E941FB2A7
:107D00009B01AC01D8016D917D918D919C910E9458
:107D1000FCB487FFB6C00E940BAC681979098A09C8
:107D20009B09693E73408105910508F4B5CFEFE7E3
:107D3000F4E08491882341F09091C00095FFFCCF3E
:107D40008093C6003196F5CF40912A1250912B12A4
:107D500060912C1270912D1222E030E084E995E0C0
:107D60000E945620EAE7F4E08491882341F0909144
:107D7000C00095FFFCCF8093C6003196F5CF4091AF
:107D80002E1250912F12609130127091311222E018
:107D900030E084E995E00E945620E6E7F4E0849123
:107DA000882341F09091C00095FFFCCF8093C600DE
:107DB0003196F5CFF7FE4ACFEBE8F3E006C090919D
:107DC000C00095FFFCCF8093C60081918111F7CF51
:107DD0008091C00085FFFCCF59CF882777FD809523
:107DE000982F0E949BB320E030E040E85FE30E94C0
:107DF00020B29B01AC01F801608171818281938185
:107E00000E94F9B21816ECF586CFF7FC2FC0E0916E
:107E10001A06F0E08F01000F111F000F111F065D01
:107E20001D4EEE0FFF1FE85CFD4E608171818827BB
:107E300077FD8095982F0E949BB39B01AC01D801E0
:107E40006D917D918D919C910E941FB20E9468B3AB
:107E500097FF07C090958095709561957F4F8F4FE4
:107E60009F4F64307105810591055CF4F7FC14C0E7
:107E70000E940BAC6C197D096031774208F44BCF3E
:107E80000BC00E940BAC6B017C019FEFC916D90699
:107E9000E906F90659F73FCF88E694E00E942E855F
:107EA0000E940BAC6093FB067093FC068093FD066A
:107EB0009093FE060E940BAC609303077093040737
:107EC00080930507909306078DCE0E94726A88E51D
:107ED0000E94712481115F9A89E50E9471248111A9
:107EE0008A9A8AE50E947124882341F09FB7F8940A
:107EF000809108018160809308019FBF85E40E9402
:107F00007124882311F40C944937129A479A0C94DF
:107F10004937A2960FB6F894DEBF0FBECDBFDF91F2
:107F2000CF911F910F91FF90EF90DF90CF90BF9076
:107F3000AF909F908F907F906F905F904F903F9009
:107F40000895CF93DF9380910D0790910E070397CB
:107F500014F40E94DE2460E08BE099E00E94A618F1
:107F600080910D0790910E07892B09F463C08091D1
:107F70000B098823E1F0809111079091120720E608
:107F8000289FE001299FD00D1124C95ED84F66E7D4
:107F900076E0CE010E9411BA892BF1F4BE018BE08C
:107FA00099E00E94361880910C09882319F00E94EC
:107FB0009D2C2AC0E3E7F6E08491882341F090915C
:107FC000C00095FFFCCF8093C6003196F5CF80911D
:107FD000C00085FFFCCF15C08BE099E00E949A1984
:107FE000E1E6F6E08491882341F09091C00095FF8E
:107FF000FCCF8093C6003196F5CF8091C00085FFFD
:10800000FCCF8AE08093C60080910D0790910E0707
:10801000019790930E0780930D078091110790911F
:108020001207019664E070E00E94B7B690931207C1
:10803000809311070E948C6C0E949B2B0E94A0626F
:108040000E94062BDF91CF910C9444868BE099E03F
:108050000C94B6118BED99E00E94AA1189E999E080
:108060000E94AA118AE799E00E94AA118BE599E083
:108070000E94AA118AE399E00C94AA112F923F92D0
:108080004F925F926F927F928F929F92AF92BF9228
:10809000CF92DF92EF92FF920F931F93CF93DF93D4
:1080A000CDB7DEB7C454D1090FB6F894DEBF0FBE0A
:1080B000CDBF3C011B014A012FA309A7EBA62196C6
:1080C000ACAEBDAECEAEDFAE219734E0239F200133
:1080D0001124440D551D5AAB49ABDA01CD90DD900A
:1080E000ED90FC90FC01E40DF51D20813181428171
:1080F0005381C701B6010E9420B26BAB7CAB8DAB44
:108100009EABB4E00B9F80011124F401E00FF11F3E
:10811000F8AFEFAB80809180A280B380F301E00FD5
:10812000F11F2081318142815381C501B4010E9438
:1081300020B269AF7AAF8BAF9CAF2BA5F4E02F9F35
:10814000C0011124F301E80FF91F20813181428120
:108150005381298F3A8F4B8F5C8FF101E80FF91F04
:1081600060817181828193810E941FB26F8F78A399
:1081700089A39AA3D1011C968D919D910D90BC91DC
:10818000A02D8DA79EA7AFA7B8ABD3011C962D91AC
:108190003D914D915C911F972BA33CA34DA35EA3F2
:1081A000A701960150582D8B3E8B4F8B588FD501D0
:1081B000C401B058898B9A8BAB8BBC8BF101E40D59
:1081C000F51D2BA93CA94DA95EA960817181828111
:1081D00093810E941FB26B017C01F101E00FF11F3E
:1081E00029AD3AAD4BAD5CAD6081718182819381E7
:1081F0000E941FB24B015C01A70196016D897E8927
:108200008F89988D0E94CEB52B013C01A501940168
:1082100069897A898B899C890E94CEB59B01AC01C2
:10822000C301B2010E9420B22B013C01A5019401BF
:108230006D897E898F89988D0E94CEB54B015C0136
:10824000A701960169897A898B899C890E94CEB59C
:108250009B01AC01C501B4010E941FB2A3019201B0
:108260000E9493B26B017C0120E030E0A9010E94E2
:10827000F9B287FF0AC02BED3FE049EC50E4C7019B
:10828000B6010E9420B26B017C016F968FAD6F9793
:10829000882351F02BED3FE049EC50E4C701B601D3
:1082A0000E941FB26B017C016E962CAD3DAD4EADB0
:1082B0005FAD6E97C701B6010E94CEB52F8D38A174
:1082C00049A15AA15F770E9409B54B015C012FE6D5
:1082D00032E143E85AE30E94F9B287FDC8C1C50103
:1082E000B4010E94D6B30E946DB37E8F6D8FDB0107
:1082F000AB2B21F4E1E0F0E0FE8FED8F2D8D3E8D74
:10830000B90180E090E00E9499B34B015C019B01B0
:10831000AC01C701B6010E9400B32B013C01A501CD
:1083200094016F8D78A189A19AA10E9400B325962E
:108330006CAF7DAF8EAF9FAF25972BA13CA14DA118
:108340005EA16DA57EA58FA598A90E941FB2A5016B
:1083500094010E9400B36DA77EA78FA798AB20E081
:1083600030E040E05FE3C301B2010E94CEB5A3015B
:1083700092010E94CEB59B01AC0160E070E080E804
:108380009FE30E941FB26F8F78A389A39AA3CE01A7
:108390000196FC014BA534E0439FE00DF11D112433
:1083A000298D3A8D4B8D5C8D20833183428353839D
:1083B0002BA13CA14DA15EA12D873E874F87588BF5
:1083C000B12C41E050E05A8F498F81E090E08C0F52
:1083D0009D1FBFA1A4E0BA9F800D911D11249CA7F1
:1083E0008BA721E030E02C0F3D1F59A544E0549F9E
:1083F000200D311D11243AA729A7F8A7EFA3498D15
:108400005A8D8D8D9E8D4817590708F01BC188E144
:108410008B150CF444C02F8D38A149A15AA169894C
:108420007A898B899C890E94CEB56B017C01A3015E
:1084300092016D897E898F89988D0E94CEB5A701A2
:1084400096010E9420B2A62E172F982E892E2F8DCE
:1084500038A149A15AA16D897E898F89988D0E9482
:10846000CEB56B017C01A301920169897A898B8960
:108470009C890E94CEB59B01AC01C701B6010E9448
:108480001FB26D8B7E8B8F8B988FB3948A2D912F1B
:10849000A92DB82D898B9A8BAB8BBC8B6AC0A98D0B
:1084A000BA8DBD0180E090E00E9499B3A3019201D2
:1084B0000E94CEB56B017C010E94FDB2698B7A8B64
:1084C0008B8B9C8BC701B6010E9431B64B015C01BE
:1084D000E9A9FAA9C080D180E280F380F7FAF0948C
:1084E000F7F8F094AFA9B8AD2D913D914D915C9105
:1084F0002BA33CA34DA35EA329893A894B895C89B0
:10850000C701B6010E94CEB56D8B7E8B8F8B988F85
:10851000A50194016BA17CA18DA19EA10E94CEB565
:108520009B01AC016D897E898F89988D0E9420B254
:108530006D8B7E8B8F8B988FA5019401C701B6013F
:108540000E94CEB56B017C0129893A894B895C89EF
:108550006BA17CA18DA19EA10E94CEB59B01AC0117
:10856000C701B6010E941FB2698B7A8B8B8B9C8BE3
:10857000B12C2D893E894F89588D6BA97CA98DA975
:108580009EA90E9420B2EBA5FCA560837183828323
:10859000938329893A894B895C8969AD7AAD8BAD22
:1085A0009CAD0E9420B2A9A5BAA56D937D938D9331
:1085B0009C93139725962CAD3DAD4EAD5FAD2597A1
:1085C000EFA1F8A560817181828193810E9420B220
:1085D000AFA1B8A56D937D938D939C9313972DA513
:1085E0003EA54FA558A96D857E858F8598890E94E7
:1085F00020B26D877E878F87988B8091F6068111D8
:1086000004C0CE0101960E94FF28FE01E15AFF4FEF
:108610006F012196ECACFDAC0EAD1FAD21979E0114
:10862000235F3F4FAE01475F5F4FBE016B5F7F4FE0
:10863000CE01019656D5298D3A8D2F5F3F4F3A8F47
:10864000298FDDCE9101245F3F4FA101485F5F4F2D
:10865000B1016C5F7F4FDE01A15ABF4F6D012196C2
:10866000ECACFDAC0EAD1FAD2197C1013AD5CC5B92
:10867000DF4F0FB6F894DEBF0FBECDBFDF91CF91B5
:108680001F910F91FF90EF90DF90CF90BF90AF9030
:108690009F908F907F906F905F904F903F902F9022
:1086A00008952F923F924F925F926F927F928F9296
:1086B0009F92AF92BF92CF92DF92EF92FF920F9371
:1086C0001F93CF93DF93CDB7DEB768970FB6F894BB
:1086D000DEBF0FBECDBF1C012A013B01480159017D
:1086E000DC01D8966D917D918D919C91DB970E94D4
:1086F00099B36B017C01A30192010E94CEB50E9447
:10870000E6B20E946DB36D877E878F87988BA50137
:108710009401C701B6010E94CEB50E94E6B20E9444
:108720006DB3698B7A8B8B8B9C8B2D853E854F85AA
:108730005889283731054105510540F488E790E014
:10874000A0E0B0E08D879E87AF87B88B29893A89F2
:108750004B895C89283731054105510540F488E78C
:1087600090E0A0E0B0E0898B9A8BAB8BBC8B910141
:108770002C5B3F4FD9018D919D910D90BC91A02D07
:108780008D839E83AF83B887BC01CD010E949BB3CC
:1087900069837A838B839C83F10164AD75AD86AD6B
:1087A00097AD0E9499B369877A878B879C8720E071
:1087B00030E0A90169817A818B819C810E94F9B2A4
:1087C000882339F1A7019601C701B6010E94CEB5F1
:1087D0004B015C0129853A854B855C85CA01B9014D
:1087E0000E94CEB59B01AC01C501B4010E941FB22D
:1087F0004B015C0129813A814B815C81CA01B9013D
:108800000E9420B29B01AC01C501B4010E9400B3DB
:1088100003C060E070E0CB010E94E6B20E9468B342
:108820002B013C016D817E818F819885909580958B
:10883000709561957F4F8F4F9F4F0E949BB34B0167
:108840005C01F101E05CFF4F608171818281938165
:108850000E9499B36D837E838F83988720E030E0F8
:10886000A901C501B4010E94F9B2882349F12D8103
:108870003E814F815885CA01B9010E94CEB56D8BEA
:108880007E8B8F8B988FA7019601C701B6010E943E
:10889000CEB59B01AC016D897E898F89988D0E9430
:1088A0001FB26B017C01A5019401C501B4010E94B6
:1088B00020B29B01AC01C701B6010E9400B303C006
:1088C00060E070E0CB010E94D6B3D10150968D904C
:1088D0009D90AD90BC90539775016401C418D50864
:1088E000E608F7080E9468B3C61AD70AE80AF90A28
:1088F000F7FE6BC020E030E0A90169817A818B81AD
:108900009C810E94F9B2882309F447C029813A81E9
:108910004B815C81CA01B9010E9420B26B017C01CC
:10892000C501B4010E9499B39B01AC01C701B60116
:108930000E94CEB56B017C0129853A854B855C850B
:10894000CA01B9010E94CEB59B01AC01C701B601B5
:108950000E941FB26B017C012D813E814F815885A1
:10896000CA01B9010E94CEB59B01AC01C701B60195
:108970000E9420B26B017C0120E030E040E850E42E
:1089800069817A818B819C810E94CEB59B01AC016B
:10899000C701B6010E9400B303C060E070E0CB01E4
:1089A0000E94E6B20E9468B32B013C0197FF03C00E
:1089B000412C512C3201481459046A047B0410F0F4
:1089C00024013501C12CD12C76018FB7F894F10127
:1089D000E45BFF4F9081911121C0F101448A558AD7
:1089E000668A778AC40CD51CE61CF71CD101C08EA0
:1089F000D18EE28EF38E2D853E854F85588924AF2A
:108A000035AF46AF57AFA05CBF4F29893A894B8934
:108A10005C892D933D934D935C9313978FBF68961C
:108A20000FB6F894DEBF0FBECDBFDF91CF911F917F
:108A30000F91FF90EF90DF90CF90BF90AF909F90FD
:108A40008F907F906F905F904F903F902F90089500
:108A50004F925F926F927F92AF92BF92CF92DF92CE
:108A6000EF92FF920F931F93CF93DF93EB017A0165
:108A7000209709F458C04115510509F454C0AAA41F
:108A8000BBA40CA51DA59501A8016EA17FA188A579
:108A900099A50E94F9B2882309F445C08FA98111D4
:108AA0003AC0F70146A057A060A471A4A3019201A7
:108AB000B501C8010E94FCB418166CF5A30192011F
:108AC000C301B2010E94CEB56B017C018AA99BA9AA
:108AD000ACA9BDA9BC01CD0190589B01AC010E947D
:108AE00020B22EA53FA548A959A90E94CEB59B0149
:108AF000AC01C701B6010E941FB20E943BB66B01D8
:108B00007C019B01AC01B501C8010E94F9B287FD4F
:108B100002C056018701A501B8014EA35FA368A753
:108B200079A781E08EABDF91CF911F910F91FF90DC
:108B3000EF90DF90CF90BF90AF907F906F905F905D
:108B40004F900895DF92EF92FF920F931F93CF9370
:108B5000DF938091120A8FB7F894E090110A8FBFCB
:108B60008091120A90E08E1991098F7099270497CD
:108B7000F4F01091120A13501F7040E050E000E032
:108B8000F12C8DE4D82E1E1591F0111101C010E1C9
:108B90001150D19EE0011124CD5ED54F602F7F2D65
:108BA000CE0156DF402F5F2D0C2FFD2EECCFDF9135
:108BB000CF911F910F91FF90EF90DF9008954F920A
:108BC0005F926F927F92AF92BF92CF92DF92EF92BD
:108BD000FF920F931F93CF93DF938C01EB010097CC
:108BE00009F453C0FC0187A981114FC046A057A0CA
:108BF00060A471A4AEA0BFA0C8A4D9A49501A60189
:108C0000C301B2010E94F9B287FF3FC0A3019201E4
:108C1000C301B2010E94CEB52B013C01F80182A92B
:108C200093A9A4A9B5A9BC01CD0190589B01AC01A1
:108C30000E9420B2F80126A537A540A951A90E949B
:108C4000CEB59B01AC01C301B2010E941FB20E94CC
:108C50003BB67B018C019B01AC01B501C6010E94B2
:108C6000F9B287FF02C0750186019701A801B5011D
:108C7000C6010E94F9B2882341F0A701B8014EA3B2
:108C80005FA368A779A781E08EABDF91CF911F9199
:108C90000F91FF90EF90DF90CF90BF90AF907F90BB
:108CA0006F905F904F900895EF92FF920F931F93F4
:108CB000CF93DF93F090110A00E010E080E090E0A5
:108CC0002DE4E22E2091120AF21689F0EF9CE001C9
:108CD0001124CD5ED54FAE01B80171DF81E08F0D5B
:108CE000803109F480E0F82EC8018E01EBCF40E01E
:108CF00050E0B801DF91CF911F910F91FF90EF905D
:108D00005ECF4F925F926F927F928F929F92AF92BF
:108D1000BF92CF92DF92EF92FF920F931F93CF9368
:108D2000DF939090110AC0E0D0E03DE4832E892DBE
:108D3000992787FD90952091120A30E082179307BA
:108D4000B9F1889E5001899EB00C1124C5018D5E39
:108D5000954F5C01209729F18EA9811104C0F5017E
:108D600086A98823F1F0CAA0DBA0ECA0FDA0A70192
:108D70009601F50166A177A180A591A50E9400B397
:108D80002B013C01A70196016EA17FA188A599A5A1
:108D90000E9400B3AB01BC0193018201CE0181DCD2
:108DA0001EAA9394F0E19F1201C0912CE501BFCF60
:108DB0002097E9F0CAA0DBA0ECA0FDA0A7019601D6
:108DC0006DEC7CEC8CE49DE30E9400B34B015C01F4
:108DD000A70196016EA17FA188A599A50E9400B365
:108DE000AB01BC0195018401CE015BDC1EAADF91C1
:108DF000CF911F910F91FF90EF90DF90CF90BF9098
:108E0000AF909F908F907F906F905F904F9008955C
:108E100099DE4ADF76CF1092120A1092110A80E191
:108E2000E8EFFEE0DF011D928A95E9F71092E80E67
:108E30001092E90E1092EA0E1092EB0E1092EC0EC8
:108E40001092ED0E1092EE0E1092EF0E1092F00EA8
:108E50001092F10E1092F20E1092F30E1092F40E88
:108E60001092F50E1092F60E1092F70E1092E40E7C
:108E70001092E50E1092E60E1092E70E08954F92B2
:108E80005F926F927F928F929F92AF92BF92CF929A
:108E9000DF92EF92FF920F931F93CF93DF93809116
:108EA000E30E882309F4EFC0C0904802D090490235
:108EB000E0904A02F0904B026091381270913912A2
:108EC000882777FD8095982F0E949BB320E030E0A3
:108ED00040E050E40E9420B29601A7010E94F9B23E
:108EE00087FDD1C05090110A612C712C00E010E078
:108EF0004DE4442E8091120A581609F453C0852D72
:108F000090E0489EF001499EF00D1124ED5EF54F72
:108F10004081518162817381452B462B472B81F41F
:108F20004481558166817781452B462B472B41F43F
:108F30004085518562857385452B462B472B69F10A
:108F4000489EE001499ED00D1124CD5ED54F6C8521
:108F50007D858E859F850E949BB34B015C0168894E
:108F600079898A899B890E9499B39B01AC01C501CB
:108F7000B4010E9400B32AA13BA14CA15DA10E94B3
:108F8000CEB55B01D82FC92F9301A8010E94FCB474
:108F900018161CF435010D2F1C2F5394852D8F703E
:108FA000582EA8CF209144023091450240914602AC
:108FB00050914702B301C8010E94CEB59B01AC019C
:108FC000B601C7010E9420B28B01D82FC92F96018C
:108FD000A7010E94F9B287FD03C06801ED2EFC2EA7
:108FE00000914C0210914D02D0914E02C0914F025F
:108FF00098014D2F5C2FB601C7010E94FCB41816D2
:109000001CF08601DE2DCF2D80900D0A90900E0A67
:10901000A0900F0AB090100A98014D2F5C2FC50147
:10902000B4010E94FCB41816D4F420E037ED43EAF2
:109030005CE3B8018D2F9C2F0E94CEB56B017C01A3
:1090400028E431EE4AE75FE3C501B4010E94CEB5E2
:10905000A70196010E9420B28B01D82FC92FC80109
:10906000AD2FBC2F80930D0A90930E0AA0930F0A88
:10907000B093100AB8018D2F9C2F0E9468B3709393
:10908000391260933812DF91CF911F910F91FF90A9
:10909000EF90DF90CF90BF90AF909F908F907F9098
:1090A0006F905F904F9008956091C8089091110A59
:1090B0008091120A981781F08091110A9DE4899F8E
:1090C000F0011124E55AF54F60819091120A891739
:1090D00019F08F5F8F70F9CF70E089E00E94C1AC0A
:1090E000CECE2F923F924F925F926F927F928F924D
:1090F0009F92AF92BF92CF92DF92EF92FF920F9327
:109100001F93CF93DF93CDB7DEB7CC56D1090FB6FF
:10911000F894DEBF0FBECDBF2C015B014A013901BF
:10912000EBAAFFAAD9AEC8AE2091120A2F5F2196F2
:109130002FAF2197203119F421961FAE2197219648
:109140003FAD2197E32EFF24E7FCF0948091110AB4
:1091500090E08E159F0539F40E948C6C0E949B2B29
:109160000E944486F3CF2091440F3091450F4091E7
:10917000460F5091470FD2016D917D918D919C9139
:109180000E94CEB50E949EB569966CAF7DAF8EAF42
:109190009FAF69972091480F3091490F40914A0F36
:1091A00050914B0FF50160817181828193810E9402
:1091B000CEB50E949EB56D966CAF7DAF8EAF9FAF62
:1091C0006D9720914C0F30914D0F40914E0F509163
:1091D0004F0FD4016D917D918D919C910E94CEB5E0
:1091E0000E949EB5A1966CAF7DAF8EAF9FAFA19749
:1091F0002091500F3091510F4091520F5091530FC9
:10920000F30160817181828193810E94CEB50E94B9
:109210009EB56CAF7DAF8EAF9FAF8091040F9091E4
:10922000050FA091060FB091070F2CAD3DAD4EADCF
:109230005FAD281739074A075B0709F4A7C0E0911B
:10924000CA0834E0E39FF0011124E65DFD4E209151
:1092500040023091410240914202509143026081AC
:109260007181828193810E94F9B287FF2DC08CADFC
:109270009DADAEADBFAD8093040F9093050FA0934D
:10928000060FB093070FE0EEF7E08491882341F0DA
:109290009091C00095FFFCCF8093C6003196F5CF2A
:1092A000E6ECF7E08491882341F09091C00095FFAF
:1092B000FCCF8093C6003196F5CF8091C00085FF2A
:1092C000FCCF8AE08093C6008091040F9091050F37
:1092D000A091060FB091070F2CAD3DAD4EAD5FAD27
:1092E000281B390B4A0B5B0BCA01B90157FF07C09A
:1092F00090958095709561957F4F8F4F9F4F0E94FD
:109300009BB36B017C0120E030E84AE454E46091B7
:10931000500F7091510F8091520F9091530F0E94F6
:10932000CEB59B01AC01C701B6010E94FCB4181672
:109330006CF58CAD9DADAEADBFAD8093040F909339
:10934000050FA093060FB093070FE0EEF7E08491AE
:10935000882341F09091C00095FFFCCF8093C60018
:109360003196F5CFE8EAF7E08491882341F09091B7
:10937000C00095FFFCCF8093C6003196F5CF809159
:10938000C00085FFFCCF8AE08093C6008091120A5E
:109390009DE4899F10011124D101AD5EB54F1D01DF
:1093A000FD01E45BFF4F10822091F80E3091F90E21
:1093B0004091FA0E5091FB0E2BA33CA34DA35EA34C
:1093C00069964CAC5DAC6EAC7FAC6997421A530A9F
:1093D000640A750A77FE08C07094609450944094B3
:1093E000411C511C611C711CD1014D925D926D920A
:1093F0007C9213972091FC0E3091FD0E4091FE0E51
:109400005091FF0E2FA338A749A75AA76D968CAC91
:109410009DACAEACBFAC6D97821A930AA40AB50A94
:10942000B7FE08C0B094A09490948094811C911CC5
:10943000A11CB11CD10114968D929D92AD92BC924B
:1094400017972091000F3091010F4091020F50911A
:10945000030F2FA738AB49AB5AABA196CCACDDAC10
:10946000EEACFFACA197C21AD30AE40AF50AF7FEE4
:1094700008C0F094E094D094C094C11CD11CE11CAD
:10948000F11CD1011896CD92DD92ED92FC921B97C2
:109490002091040F3091050F4091060F5091070F56
:1094A0002BA73CA74DA75EA72CAD3DAD4EAD5FAD44
:1094B0008BA59CA5ADA5BEA5281B390B4A0B5B0B44
:1094C00057FF07C050954095309521953F4F4F4F1E
:1094D0005F4FA0912C02B0912D020E9418B724E694
:1094E00030E040E050E00E94ECB6D1011C962D9394
:1094F0003D934D935C931F97C814D904EA04FB0471
:1095000014F475016401C216D306E406F50614F4DA
:1095100069017A01D301C2014C145D046E047F0419
:1095200014F4D701C601F101808B918BA28BB38B10
:109530000697A105B10508F446C7E85BFF4F809187
:10954000C8089091C908AA2797FDA095BA2F8083D3
:109550009183A283B38369962CAD3DAD4EAD5FADD3
:1095600069978BA19CA1ADA1BEA1281739074A0715
:109570005B0724F0D10190961C9203C081E0F101B9
:1095800080A36D962CAD3DAD4EAD5FAD6D978FA1B7
:1095900098A5A9A5BAA5281739074A075B073CF47F
:1095A000D10190968C919097826090968C93A19621
:1095B0002CAD3DAD4EAD5FADA1978FA598A9A9A9E2
:1095C000BAA9281739074A075B073CF4D1019096DE
:1095D0008C919097846090968C932CAD3DAD4EAD60
:1095E0005FAD8BA59CA5ADA5BEA5281739074A0779
:1095F0005B073CF4D10190968C919097886090968F
:109600008C93E8ADF9AD8081D10191968C9345287A
:109610004628472809F05F98F10184819581A68149
:10962000B781892B8A2B8B2B09F08A98F1018085D1
:109630009185A285B385892B8A2B8B2B41F09FB70F
:10964000F894809108018E7F809308019FBFF101FB
:1096500084859585A685B785892B8A2B8B2B11F060
:1096600012984798D1011C962D913D914D915C9196
:109670001F9725962CAF3DAF4EAF5FAF2597232B9D
:10968000242B252BF1F4B091180FBBA3E091190FF7
:10969000EFA3F0911A0FFFA720911B0F2BA72B2FE1
:1096A0003E2F4F2F5BA56BA97FA9C8010E94F9B27D
:1096B00087FD18C03BA93BA34FA94FA30FA71BA72A
:1096C00011C05091300F5BA38091310F8FA3909107
:1096D000320F9FA7A091330FABA7252F382F492F0B
:1096E0005A2FE1CF8091F80E9091F90EA091FA0EC9
:1096F000B091FB0E69962CAD3DAD4EAD5FAD699757
:10970000281B390B4A0B5B0BCA01B9010E949BB3A2
:109710002091440F3091450F4091460F5091470FD3
:109720000E9400B32B013C01698B7A8B8B8B9C8B45
:109730008091FC0E9091FD0EA091FE0EB091FF0E57
:109740006D962CAD3DAD4EAD5FAD6D97281B390BC1
:109750004A0B5B0BCA01B9010E949BB32091480FD1
:109760003091490F40914A0F50914B0F0E9400B326
:109770004B015C016D8B7E8B8F8B988F8091000FDE
:109780009091010FA091020FB091030FA1962CAD03
:109790003DAD4EAD5FADA197281B390B4A0B5B0B5E
:1097A000CA01B9010E949BB320914C0F30914D0F1B
:1097B00040914E0F50914F0F0E9400B36B017C01FE
:1097C000698F7A8F8B8F9C8F8091040F9091050FFA
:1097D000A091060FB091070F2CAD3DAD4EAD5FAD22
:1097E000281B390B4A0B5B0BCA01B9010E949BB3C2
:1097F0002091500F3091510F4091520F5091530FC3
:109800000E9400B36BAB7CAB8DAB9EAB60912C0226
:1098100070912D02882777FD8095982F0E949BB329
:109820009B01AC016BA97CA98DA99EA90E94CEB514
:1098300020E030E048EC52E40E9400B36D8F7E8F50
:109840008F8F98A3D1012D913D914D915C911397EC
:1098500028AF39AF4AAF5BAF26303105410551051E
:10986000FCF414960D911D912D913C9117970630A3
:10987000110521053105A4F418960D911D912D9126
:109880003C911B9706301105210531054CF4DC0194
:10989000CB01BF77F10186A797A7A0ABB1AB25C0DD
:1098A000C301B2010E9479B62B013C01C501B4018C
:1098B0000E9479B69B01AC01C301B2010E9420B2A3
:1098C0004B015C01C701B6010E9479B69B01AC0156
:1098D000C501B4010E9420B20E943BB6D1019E9600
:1098E0006D937D938D939C93D197D1019E962D91ED
:1098F0003D914D915C91D19765962CAF3DAF4EAFA8
:109900005FAF659760E070E080E89FE30E9400B37E
:109910009B01AC016BA17FA18FA59BA50E94CEB539
:109920002B013C019091120A8091110AE92FF0E07D
:10993000E81BF109EF70FF27F8ABEFA7A301920135
:1099400060E074E284E799E40E9400B30E949EB54F
:109950006B017C012FA538A9223031050CF442C0DF
:109960004901AA2497FCA094BA2CC501B4010E9415
:109970009BB320E030E040E051E40E94F9B287FF61
:1099800031C08091640F9091650FA091660FB091E6
:10999000670FC816D906EA06FB0620F5BC01CD0103
:1099A0006C197D098E099F09660F771F881F991F03
:1099B000A50194010E94CAB6CA01B9010E9499B3D7
:1099C0000E949EB56C0D7D1D8E1D9F1D0E9499B33A
:1099D0009B01AC0160E074E284E799E40E9400B36B
:1099E0002B013C01A301920165966CAD7DAD8EAD5E
:1099F0009FAD65970E94CEB529966CAF7DAF8EAFB7
:109A00009FAF2997D10192966D937D938D939C93EF
:109A1000959750966D917D918D919C9153970E9451
:109A200099B36BA37CA38DA39EA3A30192010E9473
:109A3000CEB50E94E6B20E946DB36B017C01F101CC
:109A400060AF71AF82AF93AF8E010F5E1F4F24E501
:109A50003FE061963FAF2EAF6197AE014F5D5F4F24
:109A60005AA349A3CE0101962F969FAF8EAF2F9791
:109A70001FA21BA690E89BABAFE3AFABF8016191CF
:109A80007191819191918F01A30192010E94CEB5B4
:109A90002F96AEADBFAD2F976D937D938D939D9314
:109AA0002F96BFAFAEAF2F979B01AC015F772D967E
:109AB0002CAF3DAF4EAF5FAF2D976196AEADBFAD52
:109AC00061978D909D90AD90BD906196BFAFAEAF08
:109AD0006197A50194012D966CAD7DAD8EAD9FADC6
:109AE0002D970E94FCB41816F4F42D962CAD3DADC4
:109AF0004EAD5FAD2D97C501B4010E9400B3B62EE7
:109B0000A72E982E892E262F372F482F592F6FA139
:109B10007BA58BA99FA90E94F9B287FD04C0BFA2B3
:109B2000ABA69BAA8FAAE9A1FAA10E171F0709F0FD
:109B3000A5CF20E030E040E85FE36FA17BA58BA9D3
:109B40009FA90E94F9B287FF3FC05E01F1E1AF0E0D
:109B5000B11C8E010F5F1F4F2FA13BA54BA95FA921
:109B6000D8016D917D918D919C910E94CEB5F801A7
:109B700061937193819391938F01EA15FB0561F7CE
:109B80002FA13BA54BA95FA929966CAD7DAD8EADEC
:109B90009FAD29970E94CEB5D10192966D937D938A
:109BA0008D939C939597C701B6010E9499B32FA1FD
:109BB0003BA54BA95FA90E94CEB50E946DB3F101F0
:109BC00060AF71AF82AF93AF65962CAD3DAD4EAD3A
:109BD0005FAD65976BA17CA18DA19EA10E9400B392
:109BE0006B017C0128AD39AD4AAD5BAD232B242B35
:109BF000252B59F5F10184819581A681B781892BA7
:109C00008A2B8B2B11F580859185A285B385892BB5
:109C10008A2B8B2BD1F42091280F3091290F409162
:109C20002A0F50912B0FC701B6010E94CEB50E949A
:109C3000E6B281010C5B1F4F0E946DB3D8016D939A
:109C40007D938D939C931397F6C020912C0F3091A8
:109C50002D0F40912E0F50912F0FC701B6010E947A
:109C6000CEB50E94E6B20E946DB381010C5B1F4F1E
:109C7000F80160837183828393834090080F509032
:109C8000090F60900A0F70900B0F0E9499B34B015F
:109C90005C0168AD79AD8AAD9BAD0E949BB39B0121
:109CA000AC01C501B4010E94CEB52BA13CA14DA1D0
:109CB0005EA10E9400B34B015C01C301B2010E948E
:109CC00099B39B01AC01C501B4010E94FCB4181604
:109CD00034F4D8014D925D926D927C92139740902E
:109CE0000C0F50900D0F60900E0F70900F0FF80139
:109CF00060817181828193810E9499B34B015C01E3
:109D0000D10114966D917D918D919C9117970E9430
:109D10009BB39B01AC01C501B4010E94CEB52BA140
:109D20003CA14DA15EA10E9400B34B015C01C301A7
:109D3000B2010E9499B39B01AC01C501B4010E941C
:109D4000FCB418162CF4F8014082518262827382AE
:109D50004090140F5090150F6090160F7090170FD1
:109D600081010C5B1F4FD8016D917D918D919C916C
:109D70000E9499B34B015C0125966CAD7DAD8EAD13
:109D80009FAD25970E949BB39B01AC01C501B40117
:109D90000E94CEB52BA13CA14DA15EA10E9400B3B3
:109DA0004B015C01C301B2010E9499B39B01AC015C
:109DB000C501B4010E94FCB418162CF4F8014082CD
:109DC0005182628273824090100F5090110F609008
:109DD000120F7090130FD8016D917D918D919C9110
:109DE0000E9499B34B015C01F10160857185828508
:109DF00093850E949BB39B01AC01C501B4010E94F5
:109E0000CEB52BA13CA14DA15EA10E9400B34B0198
:109E10005C01C301B2010E9499B39B01AC01C50171
:109E2000B4010E94FCB4181634F4D8014D925D922E
:109E30006D927C921397F101EC5BFF4F6081718111
:109E4000828193810E9499B34B015C01A701960125
:109E50000E9400B3A5966CAF7DAF8EAF9FAFA59764
:109E6000F10162AB73AB84AB95AB2DEB37E346E00E
:109E700051E4C501B4010E94CEB50E9468B3D1017E
:109E80005C966D937D938D939C935F97C090240F08
:109E9000D090250FE090260FF090270F20E030E0C3
:109EA00040E05FE3C701B6010E94CEB56BA37FA37C
:109EB0008C0129853A854B855C85A9962CAF3DAFF1
:109EC0004EAF5FAFA9978091200F9091210FA09185
:109ED000220FB091230F25968CAF9DAFAEAFBFAFD1
:109EE000259720E030E040E05FE3BC01CD010E9417
:109EF000CEB5B62EA72E982E892EA9966CAD7DAD27
:109F00008EAD9FADA9979F772B2D3A2D492D582DBA
:109F10000E94FCB418167CF42B2D3A2D492D582D97
:109F20006BA17FA1C8010E94F9B287FD04C0BBA24A
:109F3000AFA2092D182D2D853E854F855889AD96E8
:109F40002CAF3DAF4EAF5FAFAD9780911C0F90919E
:109F50001D0FA0911E0FB0911F0F29968CAF9DAFC2
:109F6000AEAFBFAF299720E030E040E05FE3BC0137
:109F7000CD010E94CEB5B62EA72E982E892EAD9675
:109F80006CAD7DAD8EAD9FADAD979F772B2D3A2DEE
:109F9000492D582D0E94FCB418167CF42B2D3A2D17
:109FA000492D582D6BA17FA1C8010E94F9B287FDF0
:109FB00004C0BBA2AFA2092D182DD1019296BC916D
:109FC000BBA7F101F3A1FBABD1019496BC91BFAB50
:109FD000F101F5A1F8AF2BA53BA94B2F5F2F6BA18A
:109FE0007FA1C8010E94F9B287FD06C02BA52BA353
:109FF0003BA93FA30FA918AD4FA558A94230510561
:10A000000CF409C15091E40E5FA78091E50E2A96E9
:10A010008FAF2A979091E60E2E969FAF2E97A09124
:10A02000E70E6096AFAF609727E137EB41ED58E35D
:10A030006FA5782F892F9A2F0E94FCB418160CF068
:10A04000EAC02091E80E3091E90E4091EA0E50915D
:10A05000EB0E69817A818B819C810E941FB22B015A
:10A060003C012091EC0E3091ED0E4091EE0E50919E
:10A07000EF0E6D817E818F8198850E941FB24B010A
:10A080005C01A3019201C301B2010E94CEB52B0174
:10A090003C01A5019401C501B4010E94CEB59B010C
:10A0A000AC01C301B2010E9420B20E943BB64B0139
:10A0B0005C01A70196010E94FCB418164CF4A5019E
:10A0C0009401C701B6010E9400B35B014C0106C0B8
:10A0D000A12CB12C50E8852E6FE3962E2091F00E26
:10A0E0003091F10E4091F20E5091F30EA9966CADA5
:10A0F0007DAD8EAD9FADA9970E941FB26B017C0113
:10A10000E894F7F825962CAD3DAD4EAD5FAD2597A3
:10A11000C701B6010E94FCB41816E4F4A701960129
:10A1200025966CAD7DAD8EAD9FAD25970E9400B399
:10A13000F62EE72ED82EC92E262F372F482F592F2F
:10A14000B501C4010E94F9B287FD04C0AF2CBE2C3A
:10A150008D2C9C2C2091F40E3091F50E4091F60E32
:10A160005091F70EAD966CAD7DAD8EAD9FADAD97B8
:10A170000E941FB26B017C01E894F7F829962CAD80
:10A180003DAD4EAD5FAD2997C701B6010E94FCB44D
:10A190001816E4F4A701960129966CAD7DAD8EAD3D
:10A1A0009FAD29970E9400B3F62EE72ED82EC92E18
:10A1B000262F372F482F592FB501C4010E94F9B21D
:10A1C00087FD04C0AF2CBE2C8D2C9C2C9501A401C6
:10A1D0006BA57BA98FA998AD0E94CEB54B015C0100
:10A1E0009B01AC016FA52A967FAD2A972E968FAD65
:10A1F0002E9760969FAD60970E94F9B287FF0EC0C0
:10A200008FA42A969FAC2A972E96AFAC2E97609675
:10A21000BFAC609703C08BA09FA05801C401D501BB
:10A22000F10182A793A7A4A7B5A7A5966CAD7DADB4
:10A230008EAD9FADA59790589B01AC010E9420B2B6
:10A2400065962CAD3DAD4EAD5FAD65970E94CEB528
:10A250009B01AC016BE077ED83E29BE30E941FB2B0
:10A260000E943BB67B01D82EC92E9B01482F592F47
:10A27000B401C5010E94F9B287FD03C04701AD2CAE
:10A28000BC2CC401D501F10186A397A3A0A7B1A757
:10A2900097014D2D5C2D6BA57BA98FA998AD0E94D0
:10A2A000F9B218162CF081E0D101D7968C9302C038
:10A2B000F10117AA81E0D101D6968C9380E1FE01CD
:10A2C0003196A8EEBEE001900D928A95E1F78BA53C
:10A2D0009BA9AFA9B8AD8093E40E9093E50EA0932F
:10A2E000E60EB093E70E9C01AD016BA17FA1C80102
:10A2F0000E9400B36B017C012BA53BA94FA958AD6F
:10A30000B401C5010E9400B3AB01BC0197018601F5
:10A31000C1010E9451432196BFAD2197B093120A0B
:10A3200069962CAD3DAD4EAD5FAD69972093F80EAB
:10A330003093F90E4093FA0E5093FB0E6D968CAD50
:10A340009DADAEADBFAD6D978093FC0E9093FD0EAD
:10A35000A093FE0EB093FF0EA1962CAD3DAD4EAD79
:10A360005FADA1972093000F3093010F4093020F30
:10A370005093030F8CAD9DADAEADBFAD8093040F78
:10A380009093050FA093060FB093070F0E94084704
:10A39000C459DF4F0FB6F894DEBF0FBECDBFDF91BB
:10A3A000CF911F910F91FF90EF90DF90CF90BF90D2
:10A3B000AF909F908F907F906F905F904F903F9065
:10A3C0002F900C944563C459DF4F0FB6F894DEBF4D
:10A3D0000FBECDBFDF91CF911F910F91FF90EF90F6
:10A3E000DF90CF90BF90AF909F908F907F906F90B5
:10A3F0005F904F903F902F900895EF92FF920F93B0
:10A400001F93CF93DF937B018A01E9012091440FD1
:10A410003091450F4091460F5091470FFC016081EC
:10A420007181828193810E94CEB50E949EB5609316
:10A43000F80E7093F90E8093FA0E9093FB0E209114
:10A44000480F3091490F40914A0F50914B0FF7013F
:10A4500060817181828193810E94CEB50E949EB5F8
:10A460006093FC0E7093FD0E8093FE0E9093FF0E92
:10A4700020914C0F30914D0F40914E0F50914F0F46
:10A48000F80160817181828193810E94CEB50E9422
:10A490009EB56093000F7093010F8093020F90930D
:10A4A000030F2091500F3091510F4091520F509156
:10A4B000530F688179818A819B810E94CEB50E9469
:10A4C0009EB56093040F7093050F8093060F9093D1
:10A4D000070F24E03FE040E05FE06CEF7EE088EFB4
:10A4E0009EE00E947F6A1092E40E1092E50E109298
:10A4F000E60E1092E70E1092E80E1092E90E1092FE
:10A50000EA0E1092EB0E1092EC0E1092ED0E1092DD
:10A51000EE0E1092EF0E1092F00E1092F10E1092BD
:10A52000F20E1092F30E1092F40E1092F50E10929D
:10A53000F60E1092F70EDF91CF911F910F91FF90C1
:10A54000EF9008952091500F3091510F4091520F8C
:10A550005091530FFC0160817181828193810E942F
:10A56000CEB50E949EB56093040F7093050F809343
:10A57000060F9093070F84E09FE00C94BB6A6093F2
:10A5800040027093410280934202909343020895E7
:10A59000CF92DF92EF92FF920F931F93CF93DF93AF
:10A5A00000D01F92CDB7DEB7F4E3CF2EFFE0DF2E51
:10A5B000A4E4EA2EAFE0FA2E08E01FE0F601619174
:10A5C0007191819191916F01F701219131914191A7
:10A5D00051917F0129833A834B835C830E9499B315
:10A5E00029813A814B815C810E94CEB50E946DB376
:10A5F000F80161937193819391938F01F4E4CF16E5
:10A60000FFE0DF06D9F60F900F900F900F90DF91CB
:10A61000CF911F910F91FF90EF90DF90CF90089511
:10A620008FEF8EBD0DB407FEFDCF8EB508958EBDA4
:10A630000DB407FEFDCF089561E0FC0180810C940C
:10A6400012AEFC012281322F306A36953CBD20FDCE
:10A6500006C031E0263009F430E0232F01C020E0AD
:10A660002DBD60E0FC0180810C9412AECF92DF9290
:10A67000EF92FF920F931F93CF93DF93EC018B0127
:10A680007A010E940BAC6B01CBDF8B838F3F49F4C7
:10A690000E940BAC6C197D096D327140A8F381E109
:10A6A00003C08E3F31F08FE08983CE01C5DF80E0AB
:10A6B00024C0E114F104E1F081E0E81AF1088FEF21
:10A6C0008EBDF8012FEFCF01801B910B8E159F05DA
:10A6D00038F40DB407FEFDCF8EB581932EBDF3CFB8
:10A6E0000DB407FEFDCF8EB5F801EE0DFF1D808382
:10A6F00097DF96DFCE01A0DF81E0DF91CF911F9140
:10A700000F91FF90EF90DF90CF9008950F931F93DC
:10A71000CF93DF93EB010E940BAC8B0181DF8F3F66
:10A7200049F00E940BAC601B710B6C177D07B0F3F6
:10A7300080E001C081E0DF91CF911F910F910895DA
:10A74000CF92DF92FF920F931F93CF93DF9300D0AE
:10A750001F92CDB7DEB76C01F62E29833A834B8367
:10A760005C836FDF6CE271E0C601D0DF8F2D806407
:10A770005EDF08E110E05C814B813A812981DA01DA
:10A78000C901002E04C0B695A795979587950A94A0
:10A79000D2F729833A834B835C8349DF0850110940
:10A7A00029813A814B815C81083F8FEF180739F787
:10A7B000FF2029F0E8E0FE1621F08FEF03C085E9C5
:10A7C00001C087E834DFFCE0FF1201C029DF10E0A0
:10A7D00027DFF601838387FF04C01F3F11F01F5F4F
:10A7E000F7CF0F900F900F900F90DF91CF911F91A7
:10A7F0000F91FF90DF90CF900895BF92CF92DF929C
:10A80000EF92FF920F931F93CF93DF93EC01B62E3D
:10A810001C82198248830E940BAC8B0161E0888105
:10A820000E94D9ADCE0108DF60E082E30E94D9AD7D
:10A8300061E083E30E94D9AD61E084E30E94D9AD79
:10A8400061E085E30E94D9AD61E085E30E9412AE2C
:10A8500085E08A8382E58CBD1DBC2AE0F22E8FEF55
:10A86000E6DEFA94E1F720E030E0A90160E0CE01F5
:10A8700067DFF82E8B8381E0F81649F00E940BAC5D
:10A88000601B710B613D774070F381E046C02AEA9E
:10A8900031E040E050E068E0CE0152DF82FF02C0CC
:10A8A000FC820CC094E0F92EBBDE8B83FA94E1F7B6
:10A8B0008A3A11F082E031C082E08C838C81823050
:10A8C00031F4C12CD12CE12C80E4F82E03C0C12C32
:10A8D000D12C760120E030E0A90167E3CE0130DF22
:10A8E000A701960169E2CE012BDF8B83882349F013
:10A8F0000E940BAC601B710B613D774058F38AE0FE
:10A900000CC08C818230B1F420E030E0A9016AE310
:10A91000CE0116DF882329F088E08983CE018CDE02
:10A9200014C07EDE807C803C11F483E08C8378DE72
:10A9300077DE76DECE0180DE86E08B1518F488E1C6
:10A94000898303C0BA8281E001C080E0DF91CF91AA
:10A950001F910F91FF90EF90DF90CF90BF900895DF
:10A960000F931F93CF93DF93EC0189018C81833088
:10A9700039F039E0440F551F661F771F3A95D1F71C
:10A980009A01AB0161E1CE01DBDE811109C040E03B
:10A9900052E0B801CE01DF91CF911F910F9166CEA9
:10A9A00084E08983CE0148DE80E0DF91CF911F9162
:10A9B0000F910895CF93DF93EC016EBD20E030E05E
:10A9C0000DB407FEFDCFFA01E20FF31F80818EBDAB
:10A9D0000DB407FEFDCF81818EBD2E5F3F4F211547
:10A9E00082E0380769F70DB407FEFDCF8FEF1FDE59
:10A9F0008FEF1DDE15DE8B838F71853031F083E1A3
:10AA00008983CE0119DE80E001C081E0DF91CF9122
:10AA100008950F931F93CF93DF93EC0189018C81ED
:10AA2000833039F089E0440F551F661F771F8A95E0
:10AA3000D1F79A01AB0168E1CE0182DE882311F0E3
:10AA400086E01EC0A8016EEFCE01B4DF8823C9F0F6
:10AA500068E572E0CE015ADE182F811102C087E14D
:10AA60000FC020E030E0A9016DE0CE0169DE811168
:10AA700006C0D6DD811103C0CE01DEDD05C086E152
:10AA80008983CE01D9DD10E0812FDF91CF911F9115
:10AA90000F910895CF93DF93EC019C012C5F3F4F02
:10AAA00041E050E060E070E0898D9A8D0E94066080
:10AAB000882399F04D895E896F89788D452B462BC7
:10AAC000472B59F44C815D816E817F814D8B5E8B6C
:10AAD0006F8B788F998190689983DF91CF910895DA
:10AAE000CF92DF92EF92FF920F931F93CF93DF935A
:10AAF000EC0189899A89AB89BC89803E9F4FAF411F
:10AB0000B10510F080E06AC0CE01C4DF8823D1F324
:10AB10000E941A5E182F8823A9F3E98DFA8DCC8044
:10AB2000DD80EE80FF8032E0C31AD108E108F10831
:10AB3000058404C0CC0CDD1CEE1CFF1C0A94D2F76B
:10AB400086859785A089B189C80ED91EEA1EFB1E8D
:10AB500081E080936E0FC0927111D0927211E092D9
:10AB60007311F092741180E092E0E1E7FFE0DF0101
:10AB70009C011D9221503040E1F701E0E98DFA8DF2
:10AB80008481081788F421E73FE0B701A601400F50
:10AB9000511D611D711D80916F0F9091700F39DFF4
:10ABA0008823E1F00F5FEACFC12C82E0D82EE12CA0
:10ABB000F12C058404C0CC0CDD1CEE1CFF1C0A9497
:10ABC000D2F749895A896B897C894C0D5D1D6E1DB0
:10ABD0007F1D498B5A8B6B8B7C8B812FDF91CF91A3
:10ABE0001F910F91FF90EF90DF90CF900895CF933A
:10ABF000DF93EC0141E0611101C040E06C857D858F
:10AC00008E859F850E945A5E882341F0888920E2C4
:10AC1000829FC00111248F58904F02C080E090E0C5
:10AC2000DF91CF91089530E020E04EE2DC015C91AD
:10AC3000503271F0383029F4FB01E20FF11D4083EE
:10AC40002F5FFB01E20FF11DDC015C9150832F5F50
:10AC50003F5F01963B3051F7FB01E20FF11D10827F
:10AC60000895CF93DF93EB01FC012381211102C0F2
:10AC700080E00EC02250223020F48FE288831982B7
:10AC800006C060E0B4DF009799F3BE01CCDF81E03D
:10AC9000DF91CF910895FB012BE030E231932150F9
:10ACA000E9F7DC0190E027E03A2FEB2F8D9181113D
:10ACB0000AC0DA013C931196EC9381E0FB0190818C
:10ACC000903239F525C08F32A1F38E3219F0E6EEBD
:10ACD000F7E008C02A30E1F098E02AE0E5CF3196AD
:10ACE0003817B1F034913111FACF291788F03FEDC0
:10ACF000380F3E3568F431E0390FFB01E90FF11DE3
:10AD00009FE9980F9A3108F480528083932FCCCF1B
:10AD100080E008950F931F93CF93DF93EC018B0195
:10AD20008B81882311F080E042C0FB01878980314C
:10AD300039F18032C1F783E08B83F801428D538D66
:10AD4000648D758D4D8B5E8B6F8B788F9E012F5E22
:10AD50003F4FC8010E94115F882329F31A8F098F82
:10AD600081E089831C821D821E821F8218861986BB
:10AD70001A861B861C861D861E861F86188A17C08B
:10AD800082E08B831D8A1E8A1F8A188EFB01408DEC
:10AD9000518D60E070E095E0440F551F661F771FEE
:10ADA0009A95D1F7498B5A8B6B8B7C8BD7CFDF91E0
:10ADB000CF911F910F9108952F923F924F925F92E2
:10ADC0006F927F928F929F92AF92BF92CF92DF92BB
:10ADD000EF92FF920F931F93CF93DF93EC015B01F0
:10ADE0006A018B81811103C08FEF9FEFC6C08981FB
:10ADF00080FFFACF49895A896B897C898885998532
:10AE0000AA85BB852601612C712C8A019B01081B38
:10AE1000190B2A0B3B0B401651066206730618F0FD
:10AE20006A01C81AD90A76013E0124E0620E711C3B
:10AE3000E114F10409F476C0488559856A857B855B
:10AE40004A0181E098222B811A012B01E9E05694F6
:10AE5000479437942794EA95D1F7898D9A8DFC0110
:10AE6000223049F4628D738D848D958D620D731D32
:10AE7000841D951D3CC01481115012218114910430
:10AE8000C1F4111116C0452B462B472B49F48D896F
:10AE90009E89AF89B88D8C839D83AE83BF8309C0A3
:10AEA0004C815D816E817F8193013CD7882309F4B9
:10AEB0009BCFE98DFA8D6C817D818E819F8162505F
:10AEC000710981099109058404C0660F771F881FE5
:10AED000991F0A94D2F72685378540895189620FD8
:10AEE000731F841F951F610F711D811D911D20E02F
:10AEF00032E02819390987012E153F0508F4890128
:10AF00000115F2E01F0761F5209171113091721166
:10AF1000409173115091741162177307840795075C
:10AF200019F41EC0C60129C09501AB01BC01809176
:10AF30006F0F9091700F14DD882309F455CFA00E88
:10AF4000B11E88859985AA85BB85800F911FA11D9B
:10AF5000B11D88879987AA87BB87E01AF10A68CF55
:10AF600040E0A8D6882309F43FCFB4016F58704F52
:10AF7000A801C5010E9438BAE2CFDF91CF911F919D
:10AF80000F91FF90EF90DF90CF90BF90AF909F9088
:10AF90008F907F906F905F904F903F902F9008958B
:10AFA000CF93DF931F92CDB7DEB741E050E0BE01F3
:10AFB0006F5F7F4F01DF019719F4898190E002C034
:10AFC0008FEF9FEF0F90DF91CF910895CF92DF9297
:10AFD000EF92FF920F931F93CF93DF936C01EB01DE
:10AFE0007A01FC018381823060F000851185228521
:10AFF00033850F71112722273327012B022B032BB7
:10B0000011F08FEF5CC04115510511F0F70110826E
:10B010001DE040E250E0BE01C601CEDE8032910567
:10B0200039F021E0892B09F420E0822F819547C077
:10B0300028812223C1F0253E61F32E3251F33B8556
:10B040003F733F3061F4E114F10449F04A8D5B8DA8
:10B05000452B29F42F713FEF320F323030F02B8522
:10B0600023FDD7CF2CC080E02AC030E02150310929
:10B07000129FC001139F900D1124F701E80FF91FD3
:10B08000298120832B8121832D8122832F8123837A
:10B09000298524832E852583288926832A89278349
:10B0A0002C8920872E892187288D22872C8D238724
:10B0B0002E8D2487288126FFD2CF1586D0CFDF9111
:10B0C000CF911F910F91FF90EF90DF90CF90089557
:10B0D0001F93CF93DF93EC018B81823018F480E0D3
:10B0E00090E023C0488559856A857B85A5E07695E3
:10B0F000679557954795AA95D1F7142F1F70CE01E4
:10B100004FDF97FDECCF488559856A857B85415E89
:10B110005F4F6F4F7F4F488759876A877B8720E251
:10B12000129FC00111248F58904FDF91CF911F9132
:10B1300008954F925F926F927F92AF92BF92CF929B
:10B14000DF92EF92FF920F931F93CF93DF93EC0167
:10B150006A017B012B81222349F089899A89AB8975
:10B16000BC8984179507A607B70710F480E06BC069
:10B17000223009F463C0C114D104E104F10449F49C
:10B180001C821D821E821F82188619861A861B86C3
:10B1900059C088859985AA85BB85E98DFA8DE58595
:10B1A000F0E03996AC01BD014150510961097109C6
:10B1B0000E2E04C076956795579547950A94D2F759
:10B1C00097018601015011092109310904C0369502
:10B1D000279517950795EA95D2F7041715072607BF
:10B1E000370720F0892B8A2B8B2B49F48D899E8978
:10B1F000AF89B88D8C839D83AE83BF8304C0041B4D
:10B20000150B260B370B280139015E0184E0A80ECF
:10B21000B11C411451046104710481F04C815D81C1
:10B220006E817F819501898D9A8D7CD591E0491A37
:10B230005108610871088111ECCF05C0C886D98614
:10B24000EA86FB8681E0DF91CF911F910F91FF90FD
:10B25000EF90DF90CF90BF90AF907F906F905F9016
:10B260004F9008950F931F93CF93DF93EC018B8141
:10B270008823D1F1898187FF32C061E0CE01B7DC3C
:10B280008C01009789F1FC018081853E69F18B81F9
:10B29000823040F449895A896B897C89448F558F63
:10B2A000668F778F4D895E896F89788DF801538F0E
:10B2B000428F758B648BE091680FF091690F309726
:10B2C00059F0B8016A5E7F4FC80148961995F80198
:10B2D000808D918D938B828B89818F778983DF918C
:10B2E000CF911F910F91A6C481E0888380E0DF9108
:10B2F000CF911F910F910895CF93DF93EC01B2DFAF
:10B300001B82DF91CF910895FC0123812111F4CF9D
:10B3100008954F925F926F927F92AF92BF92CF92B9
:10B32000DF92EF92FF920F931F93CF93DF9300D0A2
:10B330001F92CDB7DEB75C016A017B01FC018381FE
:10B340008130E9F4818181FF1AC0F50181899289F8
:10B35000A389B48984179507A607B70780F0892BBE
:10B360008A2B8B2B09F472C0F501408451846284CE
:10B370007384B701A601C501DCDE811102C080E043
:10B3800066C0F501818D928DC114D104E104F104F0
:10B3900069F4458956896789708D41D7882379F387
:10B3A000F501158A168A178A108E37C0F501448177
:10B3B0005581668177819E012F5F3F4FB3D48823EB
:10B3C000F1F249815A816B817C81F501818D928DE9
:10B3D000FC012789203139F4483FFFEF5F07610501
:10B3E0007105D8F407C0483F2FEF520762072FE0DE
:10B3F000720798F414D7882309F4C1CFF50144816A
:10B400005581668177810FEF1FEF2FEF3FE0818D30
:10B41000928D6DD5882309F4B2CFF501C18AD28A05
:10B42000E38AF48A818180688183C5011BDF8823D8
:10B4300009F4A5CFB701A6014C145D046E047F0486
:10B4400010F4B301A201C50174DE01C081E00F90C8
:10B450000F900F900F90DF91CF911F910F91FF9060
:10B46000EF90DF90CF90BF90AF907F906F905F9004
:10B470004F900895FF920F931F93CF93DF93EC01AA
:10B48000F42E80E2689FF0011124EF58F04F83857D
:10B49000817121F0842F827109F04EC08091711169
:10B4A00090917211A0917311B09174118C879D8746
:10B4B000AE87BF87688B4489558960E070E0BA0128
:10B4C00055274427028D138D20E030E0402B512B6F
:10B4D000622B732B4D8B5E8B6F8B788F838588717E
:10B4E00051F4048D158D268D378D098B1A8B2B8B7E
:10B4F0003C8B81E00BC08031F9F49E012F5E3F4F01
:10B50000898D9A8D8ED48823B9F084E08B838F2D1A
:10B510008F7089831C821D821E821F821886198665
:10B520001A861B86F4FE0BC040E050E0BA01CE0143
:10B53000F0DE811104C011C01B8280E00EC0F5FE58
:10B540000BC049895A896B897C89CE01DF91CF91E3
:10B550001F910F91FF90EDCD81E0DF91CF911F9171
:10B560000F91FF900895AF92BF92CF92DF92EF922A
:10B57000FF920F931F93CF93DF937C01EB016A013E
:10B58000B22E898D9A8DF701928F818F40E050E025
:10B59000BA01CE01CEDDA12C088519852A853B850F
:10B5A00089899A89AB89BC89081719072A073B073B
:10B5B000A0F585E036952795179507958A95D1F7DB
:10B5C0000F70CE0185DD009709F481C0FC01208158
:10B5D000222311F0253EB9F4A1100EC04091711143
:10B5E000509172116091731170917411F701448739
:10B5F000558766877787008BFC018081AA24A394F6
:10B600008111CACF0AC04BE050E0BC01C6010E94C4
:10B610002BBA892B09F0C0CF58C08B2D827482348D
:10B6200009F055C0AA2049F0F701008961E0C7017F
:10B63000DEDAEC01009769F44AC08B81823009F4AC
:10B6400046C0CE014DDA882309F441C0C1E7DFE0EE
:10B6500000E080E2FE0111928A95E9F78BE0F601A5
:10B66000DE0101900D928A95E1F7E091680FF0916B
:10B67000690F309739F0BE01625F7F4FCE0140966F
:10B68000199508C081E298E2998B888B80E098E058
:10B690009F878E87888999899B8B8A8B998F888FC2
:10B6A0008E859F859F8B8E8BC5D2882381F04B2DF5
:10B6B000602FC701DF91CF911F910F91FF90EF9005
:10B6C000DF90CF90BF90AF90D5CEB7FEF0CF80E0A7
:10B6D000DF91CF911F910F91FF90EF90DF90CF906E
:10B6E000BF90AF9008953F924F925F926F927F927A
:10B6F0008F929F92AF92BF92CF92DF92EF92FF9282
:10B700000F931F93CF93DF93CDB7DEB7C354D10907
:10B710000FB6F894DEBF0FBECDBF5C016B0124965F
:10B720005FAF4EAF2497522E1C8E1F8E19821C8243
:10B730006115710511F410E073C0FC018381811162
:10B74000FACF2496EEADFFAD249780818F3211F0B1
:10B7500076011DC02496EEADFFAD249780818F3217
:10B7600031F431962496FFAFEEAF2497F3CFF60174
:10B7700083818250823060F3F601618D728DCE013B
:10B780000196C8DA8823B9F2CE0101967C018E01B8
:10B79000045E1F4F3801FE0131964F01402E312EBD
:10B7A00019C08823A9F121E0AE01495C5F4FB701C0
:10B7B000C801D9DE882309F4BECFEC14FD0411F0D2
:10B7C000C7019ADD0615170501F1942D832D780127
:10B7D000092F182FAE014E5B5F4FBE01695C7F4F92
:10B7E00024968EAD9FAD249756DA882309F4A3CF13
:10B7F0002496EEADFFAD249780818F3291F631967D
:10B800002496FFAFEEAF2497F3CF982D892DDFCF8D
:10B81000252DAE01495C5F4FB701C501A4DE182F8D
:10B82000CE01019671DDCE014C966EDD812FCD5B90
:10B83000DF4F0FB6F894DEBF0FBECDBFDF91CF91C3
:10B840001F910F91FF90EF90DF90CF90BF90AF903E
:10B850009F908F907F906F905F904F903F90089552
:10B86000CF93DF93EC0140E050E0BA0152DD882332
:10B8700061F061E0CE01BBD9009739F025EEFC0103
:10B8800020831B82DF91CF91D5C180E0DF91CF91E2
:10B8900008951F93CF93DF93CDB7DEB76B970FB6A5
:10B8A000F894DEBF0FBECDBFAB0119821C8222E02F
:10B8B000BC01CE01019617DF182F882321F0CE019D
:10B8C0000196CEDF182FCE0101961EDD812F6B96DB
:10B8D0000FB6F894DEBF0FBECDBFDF91CF911F91A1
:10B8E00008952F923F924F925F926F927F928F9224
:10B8F0009F92AF92BF92CF92DF92EF92FF920F93FF
:10B900001F93CF93DF9300D01F921F92CDB7DEB766
:10B910008C015B013A01DC0113968C911397813005
:10B92000C1F411968C9181FF14C082FF18C0F801F8
:10B93000418952896389748980859185A285B385FF
:10B9400084179507A607B70751F0C801F2DB8111EC
:10B9500006C081E0F80180838FEF9FEF37C163015C
:10B9600083C0D80159968D919C915A97FC01F4811E
:10B97000F1501A012B0169E05694479437942794AB
:10B980006A95D1F7F221FD834A0121E09222FF233B
:10B9900009F476C080E092E08819990976018C1547
:10B9A0009D0508F47C01D8015996ED91FC915A97B8
:10B9B00014962D903D904D905C901797B2E02B1A05
:10B9C000310841085108058404C0220C331C441C72
:10B9D000551C0A94D2F786859785A089B189280ECF
:10B9E000391E4A1E5B1EED812E0E311C411C511C5E
:10B9F000E114F2E0FF0609F089C080917111909185
:10BA00007211A0917311B091741182159305A40560
:10BA1000B50569F410926E0F8FEF9FEFDC018093F4
:10BA2000711190937211A0937311B09374119501D9
:10BA3000B201A10180916F0F9091700F0E94095582
:10BA4000882309F486CFF80180859185A285B38586
:10BA50008E0D9F1DA11DB11D80879187A287B38781
:10BA6000AE0CBF1CCE18DF08D80118964D915D9121
:10BA70006D917C911B97C114D10409F072CF7AC0EB
:10BA80008114910409F086CF14964D915D916D91CA
:10BA90007C911797411551056105710559F455962B
:10BAA0008D919D910D90BC91A02D0097A105B105A0
:10BAB00039F520C09E012F5F3F4F34D1882309F410
:10BAC00048CF89819A81AB81BC81F801218D328D6B
:10BAD000F9012789203139F4883FFFEF9F07A1053D
:10BAE000B10540F40DC0883F2FEF9207A2072FE069
:10BAF000B20730F0C8010E944A5581114BCF29CFBF
:10BB0000F80184839583A683B78344CF811491047D
:10BB100011F5D80118964D915D916D917C911B970F
:10BB200051968D919D910D90BC91A02D481759076C
:10BB30006A077B0780F07ED0882309F40ACF81E072
:10BB400080936E0F20927111309272114092731196
:10BB50005092741107C041E0C201B101ABD08823FB
:10BB600009F4F7CEA701B501C4018F58904F0E9488
:10BB700038BA69CF51968D919D910D90BC91A02DB1
:10BB8000F801218184179507A607B70738F4418B80
:10BB9000528B638B748B206821830CC08091680F5B
:10BBA0009091690F892B31F06114710419F02068AC
:10BBB000F8012183D80111968C9183FD02C0C30145
:10BBC00005C0C8014FDB8111FACFC3CE0F900F9093
:10BBD0000F900F900F90DF91CF911F910F91FF90D9
:10BBE000EF90DF90CF90BF90AF909F908F907F901D
:10BBF0006F905F904F903F902F900895CF93DF9379
:10BC00001F92CDB7DEB7698341E050E0BE016F5FA0
:10BC10007F4F049666DE0F90DF91CF910895FB0170
:10BC200001900020E9F7AF0141505109461B570B25
:10BC3000049657CECF9380916E0F8823B9F140912F
:10BC4000711150917211609173117091741121E70B
:10BC50003FE080916F0F9091700F0E940955C82F9F
:10BC6000811102C0C0E023C040916A0F50916B0F58
:10BC700060916C0F70916D0F411551056105710553
:10BC800091F021E73FE080916F0F9091700F0E943B
:10BC90000955882339F310926A0F10926B0F109296
:10BCA0006C0F10926D0F10926E0F01C0C1E08C2FBF
:10BCB000CF910895CF92DF92EF92FF92CF936B01D5
:10BCC0007C01C42F8091711190917211A091731118
:10BCD000B09174118C159D05AE05BF05C9F0AADFA2
:10BCE000811102C080E018C021E73FE0B701A60142
:10BCF00080916F0F9091700F0E94B054882391F340
:10BD0000C0927111D0927211E0927311F09274117D
:10BD100081E0C11180936E0FCF91FF90EF90DF9083
:10BD2000CF9008958F929F92AF92BF92CF92DF9261
:10BD3000EF92FF920F931F93CF93DF93EC016A0171
:10BD40007B01890189859A85AB85BC850196A11DFA
:10BD5000B11D84179507A607B70710F480E054C0FB
:10BD60008F89803129F49927872F762F652F0BC073
:10BD70008032A1F7CB01BA0127E096958795779598
:10BD800067952A95D1F78B889C88AD88BE88680D09
:10BD9000791D8A1D9B1D8090711190907211A09049
:10BDA0007311B0907411681579058A059B0581F4AB
:10BDB0008F89803191F4DD24EE24FF24F601EE0F0B
:10BDC000FF1FEF58F04F80819181A0E0B0E016C0D6
:10BDD00040E070DF8111ECCFC1CFE894C7F8DD24DB
:10BDE000EE24FF24F601EE0FFF1FEE0FFF1FEF58AA
:10BDF000F04F80819181A281B381BF70F80180836F
:10BE00009183A283B38381E0DF91CF911F910F9142
:10BE1000FF90EF90DF90CF90BF90AF909F908F906A
:10BE200008954F925F926F927F92AF92BF92CF929E
:10BE3000DF92EF92FF920F931F93CF93DF9300D087
:10BE40001F92CDB7DEB78C0149835A836B837C8305
:10BE50005901C12CD12C7601412C42E0542E612C89
:10BE6000712C49815A816B817C819E012F5F3F4FEC
:10BE7000C80158DF882341F1D301C201F8010584CC
:10BE800004C0880F991FAA1FBB1F0A94D2F7C80EBF
:10BE9000D91EEA1EFB1E49815A816B817C818789EC
:10BEA000803139F481E0483F5F4F6105710538F416
:10BEB000D8CF81E0483F5F4F6F4F7F4090F2F50150
:10BEC000C082D182E282F3820F900F900F900F9088
:10BED000DF91CF911F910F91FF90EF90DF90CF9066
:10BEE000BF90AF907F906F905F904F9008954F926A
:10BEF0005F926F927F928F929F92AF92BF92CF92FA
:10BF0000DF92EF92FF920F931F93CF93DF93EC0199
:10BF10004A015B0128013901423051056105710573
:10BF200008F462C049855A856B857C854F5F5F4FF9
:10BF30006F4F7F4F481559056A057B0508F454C0BB
:10BF40008F89803129F4FF24EB2CDA2CC92C0CC00A
:10BF5000803209F049C07501640177E0F694E794F6
:10BF6000D794C7947A95D1F74B895C896D897E897E
:10BF7000C40ED51EE61EF71E41E0C701B6019ADECB
:10BF8000882391F19F89903159F49924AA24BB24E4
:10BF9000F401EE0FFF1FEF58F04F5182408210C0A6
:10BFA000E89487F89924AA24BB24F401EE0FFF1F1C
:10BFB000EE0FFF1FEF58F04F408251826282738272
:10BFC0009A89923090F04D815E816F8178854C0D19
:10BFD0005D1D6E1D7F1D40936A0F50936B0F609324
:10BFE0006C0F70936D0F01C080E0DF91CF911F91B6
:10BFF0000F91FF90EF90DF90CF90BF90AF909F9008
:10C000008F907F906F905F904F9008952F923F9206
:10C010004F925F926F927F928F929F92AF92BF9258
:10C02000CF92DF92EF92FF920F931F93CF93DF9304
:10C03000CDB7DEB72F970FB6F894DEBF0FBECDBFDA
:10C040001C014C875D876E877F873B872A87DC01D1
:10C0500019960D911D912D913C911C970F5F1F4FCB
:10C060002F4F3F4F0D831E832F833887EA85FB8533
:10C0700080809180A280B38081149104A104B104D6
:10C0800031F0FFEF8F1A9F0AAF0ABF0A10C0DC0120
:10C090008D909D90AD90BC90B1E0B9870C851D85C9
:10C0A0002E853F85013011052105310509F01986DE
:10C0B00075016401412C512C3201F1018185928579
:10C0C000A385B485481659066A067B0608F04EC05B
:10C0D0000D811E812F8138850C151D052E053F050C
:10C0E00050F4F2E0CF2ED12CE12CF12CA2E08A2EDC
:10C0F000912CA12CB12C9E012F5F3F4FB701A601BF
:10C10000C10110DE882391F149815A816B817C81C4
:10C11000D701C6010196A11DB11D452B462B472B0A
:10C1200019F04C015D010FC0AC01BD01481959095E
:10C130006A097B090C851D852E853F8540175107AF
:10C140006207730741F01FEF411A510A610A710A31
:10C150006C017D01B2CF0FEF1FEF2FEF3FE0B70172
:10C16000A601C101C4DE8D83811113C01D823DC0B3
:10C170002601370121E0421A510861087108970130
:10C180008601B301A201C101B2DE882379F37301F4
:10C1900062018C149D04AE04BF0450F3AA85BB85D4
:10C1A0004D915D916D917C91411551056105710530
:10C1B000A9F4EA85FB8580829182A282B382F98507
:10C1C000FF2399F00FEF801A900AA00AB00AD1015C
:10C1D0008D929D92AD92BC92139707C095018401F8
:10C1E000C10185DE8111E5CFC1CF8D812F960FB6BC
:10C1F000F894DEBF0FBECDBFDF91CF911F910F919D
:10C20000FF90EF90DF90CF90BF90AF909F908F9076
:10C210007F906F905F904F903F902F900895AF92D6
:10C22000BF92CF92DF92EF92FF920F931F93CF9323
:10C23000DF9300D01F92CDB7DEB75C016A017B01AE
:10C2400082E090E0A0E0B0E0F50180839183A283DA
:10C25000B3839E012F5F3F4FB701A601C50162DD89
:10C26000811102C080E023C000E010E09801B70116
:10C27000A601C5013CDE8823A9F3C980DA80EB80E2
:10C28000FC80F5018789803149F481E0F8EFCF1611
:10C29000FFEFDF06E104F10450F4DBCF81E098EF1B
:10C2A000C9169FEFD906E9069FE0F90690F20F90B4
:10C2B0000F900F900F90DF91CF911F910F91FF90F2
:10C2C000EF90DF90CF90BF90AF9008957F928F92C4
:10C2D0009F92AF92BF92CF92DF92EF92FF920F9315
:10C2E0001F93CF93DF93EC01142F7093700F609323
:10C2F0006F0F1F8A82E090E0A0E0B0E0888399830E
:10C30000AA83BB8310926E0F10926A0F10926B0F6C
:10C3100010926C0F10926D0F8FEF9FEFDC018093E6
:10C32000711190937211A0937311B09374114423FF
:10C3300049F1453008F0DEC040E060E070E0CB013C
:10C34000B9DC882309F4D6C020E1129FF001112442
:10C35000E15EFE4E80818F7709F0CCC084859585A3
:10C36000A685B78584369105A105B10508F4C2C03C
:10C37000C084D184E284F384C114D104E104F104C3
:10C3800021F4B8C0C12CD12C760140E0C701B60120
:10C3900091DC782E882309F4ADC080917C0F9091B8
:10C3A0007D0F8115924009F0A5C03091810F332394
:10C3B00009F4A0C080917F0F9091800F892B09F420
:10C3C00099C020917E0F222309F494C03A8B2C83CC
:10C3D0001D8630E041E050E06D85062FCA01062E33
:10C3E00002C0880F991F0A94E2F72817390731F025
:10C3F00081E0860F8D87683078F37CC02091870FAD
:10C400003091880F2115310519F040E050E008C047
:10C410002091950F3091960F4091970F5091980F62
:10C420002D833E834F83588780917F0F9091800F9B
:10C4300046015701880E991EA11CB11C8B8A9C8A4B
:10C44000AD8ABE8AE091820FF091830FF98FE88F59
:10C45000A091810FB0E00E940EB7680D791D8A1D72
:10C460009B1D6A8F7B8F8C8F9D8FB5E0EE0FFF1F1A
:10C47000BA95E1F7E150FE4FEF2FFF27E695DC017B
:10C48000CB018E0F9F1FA11DB11D8E879F87A88B8B
:10C49000B98B8090840F9090850F8114910419F0CE
:10C4A000A12CB12C08C08090910F9090920FA09079
:10C4B000930FB090940FA7019601281B390B4A0BDC
:10C4C0005B0BDA01C901880D991DAA1DBB1D04C0B3
:10C4D000B695A795979587950A95D2F789879A87F4
:10C4E000AB87BC87853F3FE09307A105B10520F4EA
:10C4F0008CE08F8B712C15C0853F9F4FA105B10536
:10C5000010F480E10DC080919D0F90919E0FA0913D
:10C510009F0FB091A00F8A8F9B8FAC8FBD8F80E251
:10C520008F8B872DDF91CF911F910F91FF90EF900F
:10C53000DF90CF90BF90AF909F908F907F900895A5
:10C5400080918A11811109C080918911811105C0E2
:10C5500080918811811101C00895E1E4F0E1849196
:10C56000882341F09091C00095FFFCCF8093C600D6
:10C570003196F5CFE2E3F8E08491882341F0909181
:10C58000C00095FFFCCF8093C6003196F5CF809117
:10C590008A118823F1F060918B1170918C11809138
:10C5A0008D1190918E110E949BB32091440F309178
:10C5B000450F4091460F5091470F0E9400B3AB01C9
:10C5C000BC018EE298E00E94DD218EE198E00E949D
:10C5D0002E85809189118823F1F060918F117091DF
:10C5E000901180919111909192110E949BB3209192
:10C5F000480F3091490F40914A0F50914B0F0E94C4
:10C6000000B3AB01BC018AE198E00E94DD218AE021
:10C6100098E00E942E85809188118823F1F0609126
:10C6200093117091941180919511909196110E949F
:10C630009BB320914C0F30914D0F40914E0F509174
:10C640004F0F0E9400B3AB01BC0186E098E00E944E
:10C65000DD2186EF97E00E942E858091C00085FF46
:10C66000FCCF8AE08093C60010928A111092891143
:10C6700010928811089510928A11109289111092C7
:10C6800088110895809354020895EFE6F0E08081C8
:10C690008260808308951F920F920FB60F9211242B
:10C6A0000BB60F920F931F932F933F934F935F936C
:10C6B0006F937F938F939F93AF93BF93EF93FF936A
:10C6C0008091BB119091BC11892B09F086C190918A
:10C6D000120A8091110A981771F0E091110A8DE405
:10C6E000E89FF0011124ED5EF54FDF01A45BBF4F21
:10C6F00081E08C9302C0E0E0F0E0F093BC11E093A5
:10C70000BB11309709F463C1DF01A45BBF4F81E027
:10C710008C9310929E1110929F111092A011109262
:10C72000A11160AD71AD61349CE9790728F46132E3
:10C730009EE4790748F002C060E47CE9769567954D
:10C740007695679584E007C0613197E2790730F00C
:10C750007695679582E080939B1107C080939B112B
:10C760006032710510F460E270E060527109611589
:10C7700088E07807D0F0872F9927880F991F880FB6
:10C78000991F8F5B934FFC01329645915491AA27D4
:10C79000659F9001649F210D3A1F06942A1F3A1F3E
:10C7A0001124FC01859194911DC0CB01969587952C
:10C7B0008C7F8F5B974FFC01459154910296FC0151
:10C7C00085919491FB01E770FF278E9F90018F9FC9
:10C7D000300D9E9F300D1124E3E036952795EA95A4
:10C7E000E1F7CA01821B930B84369105A0F4E3E1C3
:10C7F000F4E08191882339F09091C00095FFFCCF3F
:10C800008093C600F6CF4AE050E084E995E00E94AC
:10C81000BD1F84E690E090939A11809399118091C6
:10C820009B11992787FD909590939811809397116C
:10C83000E091BB11F091BC1164AD75AD70939D1189
:10C8400060939C1161349CE9790728F461328EE48D
:10C85000780748F002C060E47CE9769567957695A4
:10C86000679584E007C0613197E2790730F07695EB
:10C87000679582E080939B1108C081E080939B11B3
:10C880006032710510F460E270E060527109611568
:10C8900088E07807E0F0872F9927880F991F880F85
:10C8A000991F8F5B934FFC01329625913491AA27F3
:10C8B000639FA001629F410D5A1F06944A1F5A1F91
:10C8C0001124FC0125913491241B350B1EC0CB0192
:10C8D000969587958C7F8F5B974FFC0125913491BE
:10C8E0000296FC0145915491FB01E770FF274E9F92
:10C8F000C0014F9F900D5E9F900D1124F3E096951F
:10C900008795FA95E1F7281B390B24363105A0F4F9
:10C91000E3E1F4E08191882339F09091C00095FF24
:10C92000FCCF8093C600F6CF4AE050E084E995E062
:10C930000E94BD1F24E630E0C901A0E0B0E0809372
:10C94000A2119093A311A093A411B093A5113093B9
:10C95000890020938800E091BB11F091BC1180897F
:10C960009189A289B389B695A79597958795B09532
:10C97000A095909581959F4FAF4FBF4F8093B61173
:10C980009093B711A093B811B093B9118093B211DD
:10C990009093B311A093B411B093B5118093AE11DD
:10C9A0009093AF11A093B011B093B1118093AA11DD
:10C9B0009093AB11A093AC11B093AD111092A6114E
:10C9C0001092A7111092A8111092A91106C080ED23
:10C9D00097E09093890080938800E091BB11F091DB
:10C9E000BC11309709F4DCC480A18093BA1180FF98
:10C9F00041C0899A8FEF809350028091540288231E
:10CA0000E9F12CB131E025FB222720F9232779F128
:10CA100080918711882359F1E091BB11F091BC11ED
:10CA200080819181A281B381181619061A061B060E
:10CA3000F4F48091751190917611A0917711B091D5
:10CA4000781180938B1190938C11A0938D11B093DA
:10CA50008E1130938A1180899189A289B38980933C
:10CA6000A6119093A711A093A811B093A911209398
:10CA7000871104C0899881E0809350028091BA1197
:10CA800081FF41C08F9A8FEF8093510280915402B1
:10CA90008823E9F12091030131E0269521702327B5
:10CAA00079F180918611882359F1E091BB11F091C1
:10CAB000BC1184819581A681B781181619061A06C2
:10CAC0001B06F4F48091791190917A11A0917B1159
:10CAD000B0917C1180938F1190939011A09391113C
:10CAE000B09392113093891180899189A289B38979
:10CAF0008093A6119093A711A093A811B093A911A8
:10CB00002093861104C08F9881E080935102809118
:10CB1000BA119FB782FF48C0F89480910B018D7FB6
:10CB200080930B019FBF8FEF80935202809154023C
:10CB3000882309F443C029B131E023FB222720F9DF
:10CB4000232779F180918511882359F1E091BB1158
:10CB5000F091BC1180859185A285B38518161906C0
:10CB60001A061B06F4F480917D1190917E11A0911C
:10CB70007F11B09180118093931190939411A093A1
:10CB80009511B09396113093881180899189A2896B
:10CB9000B3898093A6119093A711A093A811B09385
:10CBA000A911209385110AC0F89480910B0182602D
:10CBB00080930B019FBF81E0809352028091BA1154
:10CBC000E091BB11F091BC1183FF08C081A18130BD
:10CBD00011F4439801C0169A8FEF07C081A18130EC
:10CBE00011F4439A01C0169881E08093530220E02B
:10CBF00080919B1128170CF0C7C18091C00087FF5E
:10CC000019C03091C6004091150650911606CA0110
:10CC100001968F77992760911706709118068617ED
:10CC2000970741F0FA01EB56FA4F308390931606BE
:10CC300080931506E091BB11F091BC118091B61163
:10CC40009091B711A091B811B091B9114081518163
:10CC500062817381840F951FA61FB71F8093B61141
:10CC60009093B711A093B811B093B9111816190683
:10CC70001A061B06CCF5889AE091BB11F091BC1105
:10CC80008091B6119091B711A091B811B091B911DE
:10CC90004089518962897389841B950BA60BB70B58
:10CCA0008093B6119093B711A093B811B093B911B6
:10CCB000409150028091751190917611A091771159
:10CCC000B0917811552747FD5095652F752F840F2A
:10CCD000951FA61FB71F8093751190937611A0938F
:10CCE0007711B09378118898E091BB11F091BC1145
:10CCF0008091B2119091B311A091B411B091B5117E
:10CD00004481558166817781840F951FA61FB71FC7
:10CD10008093B2119093B311A093B411B093B51155
:10CD2000181619061A061B06CCF58E9AE091BB114F
:10CD3000F091BC118091B2119091B311A091B411F6
:10CD4000B091B5114089518962897389841B950B13
:10CD5000A60BB70B8093B2119093B311A093B411AB
:10CD6000B093B511409151028091791190917A114F
:10CD7000A0917B11B0917C11552747FD5095652FEF
:10CD8000752F840F951FA61FB71F8093791190935D
:10CD90007A11A0937B11B0937C118E98E091BB1116
:10CDA000F091BC118091AE119091AF11A091B01192
:10CDB000B091B1114085518562857385840F951FAF
:10CDC000A61FB71F8093AE119093AF11A093B0111F
:10CDD000B093B111181619061A061B060CF047C0BD
:10CDE0009FB7F89480910B01886080930B019FBFDF
:10CDF000E091BB11F091BC118091AE119091AF11F7
:10CE0000A091B011B091B1114089518962897389A3
:10CE1000841B950BA60BB70B8093AE119093AF11AB
:10CE2000A093B011B093B1114091520280917D1145
:10CE300090917E11A0917F11B0918011552747FDEF
:10CE40005095652F752F840F951FA61FB71F8093D0
:10CE50007D1190937E11A0937F11B09380119FB7A5
:10CE6000F89480910B01877F80930B019FBFE09125
:10CE7000BB11F091BC118091AA119091AB11A091BE
:10CE8000AC11B091AD114485558566857785840FC9
:10CE9000951FA61FB71F8093AA119093AB11A09363
:10CEA000AC11B093AD11181619061A061B060CF03A
:10CEB00043C081A1813011F4419A01C0149AE091DC
:10CEC000BB11F091BC118091AA119091AB11A0916E
:10CED000AC11B091AD114089518962897389841B6D
:10CEE000950BA60BB70B8093AA119093AB11A0934F
:10CEF000AC11B093AD11409153028091811190918A
:10CF00008211A0918311B0918411552747FD50954E
:10CF1000652F752F840F951FA61FB71F8093811152
:10CF200090938211A0938311B093841181A18130D9
:10CF300011F4419801C014988091A6119091A71105
:10CF4000A091A811B091A9110196A11DB11D8093C6
:10CF5000A6119093A711A093A811B093A911409185
:10CF6000A6115091A7116091A8117091A911E0919B
:10CF7000BB11F091BC1180899189A289B3894817AE
:10CF800059076A077B07B0F04091A6115091A7118D
:10CF90006091A8117091A911E091BB11F091BC11A1
:10CFA00084899589A689B78984179507A607B70745
:10CFB00018F4DAC02F5F1CCE4091A2115091A3113A
:10CFC0006091A4117091A511048D158D268D378D5A
:10CFD000AA27419FB12D529FC001629F900D619F72
:10CFE000800D911D429FB00D811D9A1F519FB00D64
:10CFF000811D9A1F609FB00D811D9A1F509FB10D1A
:10D000008A1F9A1FB6958A1F9A1F112444AD55ADE9
:10D01000480F591F50939D1140939C1180AD91ADC5
:10D02000A2ADB3AD60E070E084179507A607B7071F
:10D0300020F490939D1180939C1160919C117091AC
:10D040009D1161349CE9790728F461328EE47807F8
:10D0500048F002C060E47CE976956795769567951F
:10D0600084E007C0613197E2790730F076956795E3
:10D0700082E080939B1108C081E080939B11603215
:10D08000710510F460E270E060527109611588E08A
:10D090007807E0F0872F9927880F991F880F991F2D
:10D0A0008F5B934FFC01329625913491AA27639FA1
:10D0B000A001629F410D5A1F06944A1F5A1F112456
:10D0C000FC0125913491241B350B1EC0CB01969594
:10D0D00087958C7F8F5B974FFC0125913491029649
:10D0E000FC0145915491FB01E770FF274E9FC00161
:10D0F0004F9F900D5E9F900D112413E0969587959C
:10D100001A95E1F7281B390B24363105A0F4E3E129
:10D11000F4E08191882339F09091C00095FFFCCF15
:10D120008093C600F6CF4AE050E084E995E00E9483
:10D13000BD1F24E630E03093890020938800809161
:10D14000A2119091A311A091A411B091A511820FE9
:10D15000931FA11DB11D8093A2119093A311A093C1
:10D16000A411B093A511F7C04091A6115091A71139
:10D170006091A8117091A911808D918DA28DB38DB0
:10D1800084179507A607B70708F0D9C040919E11EC
:10D1900050919F116091A0117091A111048D158D76
:10D1A000268D378DAA27419FB12D529FC001629FC6
:10D1B000900D619F800D911D429FB00D811D9A1FA2
:10D1C000519FB00D811D9A1F609FB00D811D9A1F48
:10D1D000509FB10D8A1F9A1FB6958A1F9A1F11245E
:10D1E00020919C1130919D11E05CFF4F2817390769
:10D1F00018F42081318102C0281B390B8081918174
:10D20000A281B381A90160E070E0481759076A075D
:10D210007B0708F49C0121349CE9390728F421326A
:10D220008EE4380748F002C020E43CE936952795A3
:10D230003695279584E007C0213197E2390730F011
:10D240003695279582E080939B1108C081E08093FA
:10D250009B112032310510F420E230E0B901605218
:10D260007109611588E07807E0F0872F9927880F0A
:10D27000991F880F991F8F5B934FFC013296259160
:10D280003491AA27639FA001629F410D5A1F069403
:10D290004A1F5A1F1124FC0125913491241B350B80
:10D2A0001EC0CB01969587958C7F8F5B974FFC01B5
:10D2B000259134910296FC0145915491FB01E77050
:10D2C000FF274E9FC0014F9F900D5E9F900D112430
:10D2D00043E0969587954A95E1F7281B390B24364C
:10D2E0003105A0F4E3E1F4E08191882339F09091D5
:10D2F000C00095FFFCCF8093C600F6CF4AE050E017
:10D3000084E995E00E94BD1F24E630E03093890057
:10D310002093880080919E1190919F11A091A0115F
:10D32000B091A111820F931FA11DB11D80939E1179
:10D3300090939F11A093A011B093A1110CC0809164
:10D34000991190919A11909389008093880080910F
:10D35000971180939B114091A6115091A711609154
:10D36000A8117091A911E091BB11F091BC118089B5
:10D370009189A289B389481759076A077B0780F00A
:10D380001092BC111092BB119091120A8091110A57
:10D39000981731F08091110A8F5F8F708093110A76
:10D3A000FF91EF91BF91AF919F918F917F916F917D
:10D3B0005F914F913F912F911F910F910F900BBE55
:10D3C0000F900FBE0F901F901895819A879AEAE0F0
:10D3D000F1E08081826080830E9A3B9A579A5F9A2F
:10D3E000829A8A9AE7E0F1E08081816080839FB72A
:10D3F000F894E8E0F1E08081816080839FBF0A9A21
:10D40000129A3F9A479A6C98749AE4E0F1E080810E
:10D410008E7F80839FB7F894E5E0F1E080818160A2
:10D4200080839FBF6D98759AE4E0F1E080818D7FE5
:10D4300080839FB7F894E5E0F1E08081826080838B
:10D440009FBF53985B9A809A88985F9A869A8E9825
:10D450008A9AEAE0F1E08081886080839FB7F8943F
:10D46000EBE0F1E08081877F80839FBF9FB7F894D6
:10D47000E8E0F1E08081816080839FBF0C9A14987E
:10D48000129A399A4198479AA1E8B0E08C918F7E20
:10D490008C938C9188608C93E0E8F0E080818D7FA4
:10D4A000808380818E7F808380818F738083808161
:10D4B0008F7C80838C91887F82608C9380E090E465
:10D4C00090938900809388001092850010928400C8
:10D4D000EFE6F0E080818260808381E080935402F7
:10D4E000789408959091120A8091110A981731F05A
:10D4F00013D20E949B2B0E944486F4CF0895CF93B1
:10D50000DF93EFB7F894EC0188819981AA81BB8100
:10D510008093751190937611A0937711B093781141
:10D52000EB0188819981AA81BB81809379119093C5
:10D530007A11A0937B11B0937C11EA0188819981C3
:10D54000AA81BB8180937D1190937E11A0937F115E
:10D55000B0938011E90188819981AA81BB81809370
:10D56000811190938211A0938311B0938411EFBF26
:10D57000DF91CF9108952FB7F894FC0180819181BC
:10D58000A281B3818093811190938211A093831122
:10D59000B09384112FBF08952FB7F89494E0899F1A
:10D5A000F0011124EB58FE4E6081718182819381DC
:10D5B0002FBF089597DF5F9A8A9A9FB7F894E8E0A3
:10D5C000F1E08081816080839FBF129A479A08951D
:10D5D00080916F008D7F80936F009091120A8091EF
:10D5E000110A98130CC01092BC111092BB118091BB
:10D5F0006F00826080936F001092F90808959091F7
:10D60000120A8091110A981741F38091110A8F5FD5
:10D610008F708093110AE1CF2F923F924F925F92C9
:10D620006F927F928F929F92AF92BF92CF92DF9232
:10D63000EF92FF920F931F93CF93DF9300D000D010
:10D64000CDB7DEB78C01F62E21E0261760F5E1E5B7
:10D65000F1E18491882341F09091C00095FFFCCFC7
:10D660008093C6003196F5CF8F2D90E04AE050E0D0
:10D67000BC0184E995E00E94801FE7E4F0E1849119
:10D68000882341F09091C00095FFFCCF8093C600A5
:10D690003196F5CF8091C00085FFFCCF8AE0809362
:10D6A000C6000E94622B6F2D70E0FB01EE0FFF1F82
:10D6B000EB59FB4F408151815E834D83452B09F42B
:10D6C000A6C0FB01ED59FB4F50815A832D813E814D
:10D6D0002C5F3F4F81E090E089836A81861708F0D4
:10D6E0007BC0DC01F901459154910196B9016C5F51
:10D6F0007F4F041715070CF06DC00297AC01440F63
:10D70000551F440F551F4E5F5F4F6D817E81460F41
:10D71000571FFA0165917491880F991F880F991FFF
:10D72000ED81FE818E0F9F1FFC01A590B490FD013D
:10D73000EE0FFF1FEE0FFF1F3296AD81BE81EA0F85
:10D74000FB1FC590D490FA01E590F490F901259063
:10D750003490FC01259134913C832B83882777FDFD
:10D760008095982F0E949BB32B013C01B8016A1948
:10D770007B09882777FD8095982F0E949BB34B01EA
:10D780005C01B6016E197F09882777FD8095982F77
:10D790000E949BB39B01AC01C501B4010E94CEB5B0
:10D7A0006B017C01B1014B815C81641B750B882787
:10D7B00077FD8095982F0E949BB39B01AC01C70118
:10D7C000B6010E9400B39B01AC01C301B2010E94EB
:10D7D00020B206C09B0180CF60E070E080E090E066
:10D7E000A981BA81AB132BC02D813E81E4E0AE9FAD
:10D7F000200D311D112422503109F90165917491D8
:10D80000882777FD8095982F0E949BB318C0B80198
:10D81000882777FD8095982F0E949BB320E030E009
:10D820004AEF5EE30E94CEB520E030E040E85DE3E1
:10D830000E94CEB520E030E0A9010E9420B22696D9
:10D840000FB6F894DEBF0FBECDBFDF91CF911F9111
:10D850000F91FF90EF90DF90CF90BF90AF909F908F
:10D860008F907F906F905F904F903F902F90089592
:10D8700060E08091321290913312CEDE60932A12D2
:10D8800070932B1280932C1290932D1261E0809153
:10D89000341290913512C0DE60932E1270932F12C5
:10D8A000809330129093311210922412109225120C
:10D8B00010922612109227128FB7F894109223120A
:10D8C0008FBF0895209166023091670240916802EF
:10D8D0005091690260E070E08FE793E40E9400B32A
:10D8E0006093E3117093E4118093E5119093E61136
:10D8F0006093E7117093E8118093E9119093EA1116
:10D90000089597FF03C08091DA1104C0FC01E5522D
:10D91000FE4E808190E008952F923F924F925F9249
:10D920006F927F928F929F92AF92BF92CF92DF922F
:10D93000EF92FF920F931F93CF93DF93CDB7DEB794
:10D94000A2970FB6F894DEBF0FBECDBF8091231211
:10D95000882309F4D2C18CDF80916A0290916B0216
:10D96000A0916C02B0916D028D8B9E8BAF8BB88FA6
:10D970008091660290916702A0916802B09169025D
:10D98000898F9A8FAB8FBC8F8091620290916302D6
:10D99000A0916402B09165028D8F9E8FAF8FB8A366
:10D9A000AAE2B2E1BA8BA98BE8E3F2E1F88BEF8748
:10D9B00083EF91E19A878987ABEDB1E1BA83A983BF
:10D9C000E6E5F2E0F887EF8382ED91E19C8B8B8BAB
:10D9D00001EE11E14BE1242E42E1342EA3E1B2E14C
:10D9E000BC83AB83EBEFF1E1FE83ED831AA219A2B6
:10D9F000A989BA898D909D90AD90BD90BA8BA98B65
:10DA0000EF85F88961907190F88BEF87B3018827D3
:10DA100077FD8095982F0E949BB3A50194010E94E9
:10DA20001FB26B017C01A985BA856D937D938D939F
:10DA30009D93BA87A98720E030E040E251E40E943C
:10DA4000FCB4181624F421E0F8012083D6C020E0AD
:10DA500030E040E251ECC701B6010E94F9B287FD07
:10DA600002C0672821F4E1E0D801EC93CDC0D801D1
:10DA70008C91882331F0F10110821182128213827D
:10DA80001C92A70196016D897E898F89988D0E94CD
:10DA9000CEB56B877C878D879E87E9A1FAA1E55F6C
:10DAA000FD4E6083718382839383D1012D913D91DB
:10DAB0004D915C91C701B6010E9420B26B017C01BF
:10DAC000E9A1FAA1E551FE4E508061807280438049
:10DAD000252D362D472D542D0E94F9B287FD16C0F5
:10DAE000E9A1FAA1ED51FE4E508061807280438021
:10DAF000252D362D472D542DB601C7010E94FCB4AB
:10DB0000181624F05C2C6D2C7E2C4F2C852D962D18
:10DB1000A72DB42DF10180839183A283B383252D9A
:10DB2000362D472D542D698D7A8D8B8D9C8D0E94BD
:10DB3000CEB52B013C01E9A1FAA1ED5FFD4E60835A
:10DB4000718382839383AB81BC812D913D914D91F3
:10DB50005C91C501B4010E941FB29B01AC016D8DA7
:10DB60007E8D8F8D98A10E94CEB520ED3CEC4CE4CB
:10DB70005DE30E94CEB56B017C0123E333E343E711
:10DB80005FE3ED81FE8160817181828193810E94DA
:10DB9000CEB59B01AC01C701B6010E9420B26B015A
:10DBA0007C01AD81BE816D937D938D939C93139782
:10DBB000EB81FC8180829182A282B382A3019201D7
:10DBC0006B857C858D859E850E9420B2A70196017C
:10DBD0000E941FB26B017C0120E030E0A9010E948D
:10DBE000F9B287FD11C020E030E040E853E4C701FE
:10DBF000B6010E94FCB4181654F4C12CD12C30E8A4
:10DC0000E32E33E4F32E03C0C12CD12C7601AB8973
:10DC1000BC898D919D91BC8BAB8BBC01882777FD16
:10DC20008095982F0E949BB39B01AC01C501B40164
:10DC30000E94FCB41816F4F4EF81F885808191817C
:10DC4000BC01882777FD8095982F0E949BB39B018C
:10DC5000AC01C501B4010E94F9B287FF0BC0C70136
:10DC6000B6010E9468B3CB0195958795A981BA81C9
:10DC70008C9303C0E981FA81108289A19AA104964C
:10DC80009AA389A3A981BA811196BA83A983EF8146
:10DC9000F8853296F887EF830F5F1F4FF4E02F0E61
:10DCA000311C8B819C8104969C838B83AD81BE81CA
:10DCB0001496BE83AD83E9A1FAA1389709F098CEF6
:10DCC0000E940BAC0091DD111091DE112091DF114B
:10DCD0003091E011601B710B820B930B683873411C
:10DCE0008105910550F00E940BAC6093DD1170939B
:10DCF000DE118093DF119093E011A2960FB6F89495
:10DD0000DEBF0FBECDBFDF91CF911F910F91FF906E
:10DD1000EF90DF90CF90BF90AF909F908F907F90CB
:10DD20006F905F904F903F902F900895CF93DF9327
:10DD3000C0915602D09157021092EB111092EC1143
:10DD40001092ED111092EE1120916602309167024F
:10DD5000409168025091690260E070E08FE793E4BF
:10DD60000E9400B36093E3117093E4118093E51176
:10DD70009093E611D0935902C09358021092EF117C
:10DD80001092F0111092F1111092F2116093E711BC
:10DD90007093E8118093E9119093EA11249A80918D
:10DDA0000101806180930101809101018062809373
:10DDB00001018091010180648093010187ED8093CE
:10DDC0007A0010927E0010927D0080917D0080622A
:10DDD00080937D0080917D00806880937D0080919C
:10DDE0007D00806480937D0080E888BD80916E0016
:10DDF000846080936E006AEF70E080E090E00E94A3
:10DE00003AAC85E090E09093D3118093D21160E01A
:10DE100080915A0290915B02FFDB20E030E040EA03
:10DE200050E40E94F9B287FF0AC080915A02909193
:10DE30005B02409790935B0280935A02E8CF80E4A4
:10DE400091E0909357028093560260E08091D61142
:10DE50009091D711E1DB20E030E040EA53E40E94EA
:10DE6000FCB4181654F48091D6119091D7114096B5
:10DE70009093D7118093D611E8CF85E090E09093EE
:10DE8000D5118093D41161E080915C0290915D0284
:10DE9000C3DB20E030E040EA50E40E94F9B287FFA3
:10DEA0000AC080915C0290915D02409790935D0260
:10DEB00080935C02E8CF80E491E0909359028093D4
:10DEC000580261E08091D8119091D911A5DB20E032
:10DED00030E040EA53E40E94FCB4181654F48091F8
:10DEE000D8119091D91140969093D9118093D8115F
:10DEF000E8CFDF91CF9108950895109239121092D2
:10DF00003812EAE3F2E11182108210923712109275
:10DF100036121092DB112C981092DC119FB7F894F6
:10DF2000E2E0F1E080818F7E80839FBF1092371204
:10DF3000109236121092DA119FB7F89480818F7D7B
:10DF400080839FBF08952F923F924F925F926F926E
:10DF50007F928F929F92AF92BF92CF92DF92EF9279
:10DF6000FF920F931F93CF93DF93CDB7DEB7AE979A
:10DF70000FB6F894DEBF0FBECDBF6C8F7D8F8E8F36
:10DF80009F8F5EA74DA73CA72BA70E940BAC69A350
:10DF90007AA38BA39CA32DA53EA5233031051CF4A9
:10DFA000E6E2F4E017C0E9E3F4E08191882339F078
:10DFB0009091C00095FFFCCF8093C600F6CF809172
:10DFC000C00085FFFCCF15C29091C00095FFFCCF2B
:10DFD0008093C60081918111F7CF8091C00085FFA9
:10DFE000FCCF8AE08093C60088DF4DA55EA580E85F
:10DFF00057FF43C08093DA1189A19AA1ABA1BCA1BC
:10E00000898B9A8BAB8BBC8B8D879E87AF87B88BA8
:10E010001D8290E4998FACE1AA8FB6E4BB8F1D8A74
:10E020001E8A1F8A188E20E830E040E050E02983E5
:10E030003A834B835C83F0E84F2E512C612C712C7A
:10E040001DA21EA21FA218A631E038A31C861B86A3
:10E05000312C00E010E0212C4DA55EA545525E4E0E
:10E060005AA749A78DA59EA5880F991F880F991FAC
:10E07000865D9D4E9A87898708C0EDA5FEA5E5526D
:10E08000FE4E8083B9CF0E9444868091231288235C
:10E0900009F4DCC0EDDBADA5BEA5B7FF09C030902B
:10E0A000241200912512109126122090271206C0EA
:10E0B000E985FA853080018112812380232D302F5C
:10E0C000412F522D6D897E898F89988D0E94FCB4D5
:10E0D000181624F03D8A0E8B1F8B288E232D302F8F
:10E0E000412F522D6D81798D8A8D9B8D0E94F9B2C1
:10E0F00087FD04C03D82098F1A8F2B8EF8A1FF2364
:10E1000009F451C02C8D3D8D4E8D5F8D632D702F88
:10E11000812F922D0E94FCB418160CF097C00E941B
:10E120000BAC29893A894B895C89621B730B840B80
:10E13000950B693873418105910508F487C0D301B7
:10E14000C20129813A814B815C81821B930BA40B14
:10E15000B50B4DA55EA5B595A7959795879557FFE6
:10E1600003C08093DA1103C0E9A5FAA580830E9459
:10E170000BAC6D877E878F87988B9B01AC0189895B
:10E180009A89AB89BC89281B390B4A0B5B0B2DA3E1
:10E190003EA34FA358A79C8D9D8BAD8DAE8BBE8D9E
:10E1A000BF8BEF8DE88F2C8D3D8D4E8D5F8D632D58
:10E1B000702F812F922D0E94F9B287FFF0C20E942A
:10E1C0000BAC2D853E854F855889621B730B840BE4
:10E1D000950B693873418105910508F4E0C20E94EE
:10E1E0000BAC698B7A8B8B8B9C8BDC01CB012D85E7
:10E1F0003E854F855889821B930BA40BB50B4B852D
:10E200005C85452B09F011C189819A81AB81BC8164
:10E21000840D951DA61DB71D2DA53EA5B595A795E9
:10E220009795879537FFB7C28093DA112B853C8588
:10E230002F5F3F4F3C872B873C8D3D834D8D498F12
:10E240005E8D5A8F8F8D8B8F91E098A320E030E008
:10E2500040EA51E46C8D7D8D8E8D9F8D0E9420B2A1
:10E260009B01AC01632D702F812F922D0E94FCB475
:10E27000181694F4E2EEF0E18491882341F0909135
:10E28000C00095FFFCCF8093C6003196F5CF8091FA
:10E29000C00085FFFCCFADC00E940BAC29A13AA104
:10E2A0004BA15CA1621B730B840B950B613D774006
:10E2B0008105910508F450C04DA55EA557FF10C01B
:10E2C000E090DA11F12CECEDF0E184918823C9F0B3
:10E2D0009091C00095FFFCCF8093C6003196F5CF9A
:10E2E000A9A5BAA5EC90F12CE6EDF0E18491882384
:10E2F00041F09091C00095FFFCCF8093C60031960D
:10E30000F5CF22E030E0432D502F612F722D84E9AC
:10E3100095E00E945620E2EDF0E18491882341F0DF
:10E320009091C00095FFFCCF8093C6003196F5CF49
:10E330004AE050E0B70184E995E00E94801F809197
:10E34000C00085FFFCCF8AE08093C6000E940BAC22
:10E3500069A37AA38BA39CA30E940BAC6B017C01E5
:10E360000E940BAC89889A88AB88BC882D853E8535
:10E370004F855889820E931EA41EB51EC818D90851
:10E38000EA08FB08C60ED71EE81EF91E31E8C316C0
:10E390003FE4D30632E1E306F10490F0E5EBF0E16F
:10E3A0008491882341F09091C00095FFFCCF809329
:10E3B000C6003196F5CF8091C00085FFFCCF19C013
:10E3C0004B855C858BA59CA5841795070CF05BCECF
:10E3D000E4E6F0E18491882341F09091C00095FF3C
:10E3E000FCCF8093C6003196F5CF8091C00085FFA9
:10E3F000FCCF8AE08093C600AE960FB6F894DEBFDD
:10E400000FBECDBFDF91CF911F910F91FF90EF9085
:10E41000DF90CF90BF90AF909F908F907F906F9044
:10E420005F904F903F902F9008958DA09EA0AFA039
:10E43000B8A4880E991EAA1EBB1E2DA13EA14FA1F5
:10E4400058A5281B390B4A0B5B0BCA01B90129815E
:10E450003A814B815C810E9494B6A50194010E948F
:10E46000ECB6240D351D461D571D243131054105DF
:10E47000510504F129013A013DEE431651046104AE
:10E4800071042CF07CEE472E512C612C712C41E84C
:10E490004416510461047104DCF08FEF90E0A0E0B9
:10E4A000B0E084199509A609B70989839A83AB83DB
:10E4B000BC8312C064E1462E512C612C712C24E1E6
:10E4C00030E040E050E029833A834B835C8304C012
:10E4D00049825A826B827C82E9E4F1E1849188234B
:10E4E00041F09091C00095FFFCCF8093C60031961B
:10E4F000F5CF2AE030E0B301A20184E995E00E9463
:10E500005D1FE4E4F1E18491882341F09091C00023
:10E5100095FFFCCF8093C6003196F5CF2AE030E01E
:10E5200049815A816B817C8184E995E00E945D1F5D
:10E53000EDE3F1E18491882341F09091C00095FFD3
:10E54000FCCF8093C6003196F5CF22E030E04D81BC
:10E55000598D6A8D7B8D84E995E00E945620E6E313
:10E56000F1E18491882341F09091C00095FFFCCFA8
:10E570008093C6003196F5CF22E030E04D895E8968
:10E580006F89788D84E995E00E9456208091C000C3
:10E5900085FFFCCF8AE08093C6002B853C85233025
:10E5A00031050CF431CE69817A818B819C810E9486
:10E5B0009BB320E030E040E850E40E94CEB56B0110
:10E5C0007C012D81398D4A8D5B8D6D897E898F8986
:10E5D000988D0E941FB220ED3FE049E450E40E9474
:10E5E000CEB520E030E040E05FE30E94CEB59B0175
:10E5F000AC01C701B6010E9400B36B017C01C501EB
:10E60000B4010E949BB320E030E04AE754E40E944A
:10E6100000B34B015C01E0E3F1E18491882341F018
:10E620009091C00095FFFCCF8093C6003196F5CF46
:10E6300022E030E0B701A60184E995E00E9456206F
:10E64000EAE2F1E18491882341F09091C00095FFC6
:10E65000FCCF8093C6003196F5CF22E030E0B501C3
:10E66000A40184E995E00E9456208091C00085FFB6
:10E67000FCCF8AE08093C6002AE939E949E15FE3EB
:10E68000C701B6010E94CEB56B017C019B01AC01B4
:10E690000E9420B2A50194010E9400B36D837E8385
:10E6A0008F839887A5019401C701B6010E94CEB55A
:10E6B00020E030E040E05EE30E94CEB54B015C011B
:10E6C000EDE1F1E18491882341F09091C00095FF44
:10E6D000FCCF8093C6003196F5CF8091C00085FFB6
:10E6E000FCCF8AE08093C600E7E1F1E184918823C2
:10E6F00041F09091C00095FFFCCF8093C600319609
:10E70000F5CF22E030E0B701A60184E995E00E9450
:10E7100056208091C00085FFFCCF8AE08093C60020
:10E72000E1E1F1E18491882341F09091C00095FFEF
:10E73000FCCF8093C6003196F5CF22E030E04D81CA
:10E740005E816F81788584E995E00E9456208091F2
:10E75000C00085FFFCCF8AE08093C600EBE0F1E1CA
:10E760008491882341F09091C00095FFFCCF809365
:10E77000C6003196F5CF22E030E0B501A40184E96E
:10E7800095E00E9456208091C00085FFFCCF8AE072
:10E790008093C60039CDE9A5FAA5808347CD18A29C
:10E7A00055CD1F920F920FB60F9211240BB60F92F8
:10E7B0002F933F934F935F936F937F938F939F9389
:10E7C000AF93BF93EF93FF9380915502811127C0C0
:10E7D0008091DB118093D111882329F08091FD086D
:10E7E000811101C02C9A8091DC118093D011882373
:10E7F00041F09FB7F89480910201806180930201FB
:10E800009FBF8091DA118093CF11882341F09FB789
:10E81000F894809102018062809302019FBF9091E1
:10E82000D11180915502891728F08091FD0881113E
:10E8300001C02C989091D01180915502891740F019
:10E840009FB7F894809102018F7E809302019FBF51
:10E850009091CF1180915502891740F09FB7F8949D
:10E86000809102018F7D809302019FBF80915502AC
:10E870008F5F8F77809355028091CE1190E0883022
:10E88000910508F08DC0FC01EE58FF4F0C9408B7BD
:10E8900088E080937B0085E480937C0080917A00FF
:10E8A000806480937A000E94C58581E019C0209120
:10E8B0007800309179008091CA119091CB11A0918C
:10E8C000CC11B091CD11820F931FA11DB11D80936A
:10E8D000CA119093CB11A093CC11B093CD1182E0CB
:10E8E0008093CE115DC088E080937B0086E48093A6
:10E8F0007C0080917A00806480937A000E94C585B4
:10E9000083E0EECF20917800309179008091C6119C
:10E910009091C711A091C811B091C911820F931F96
:10E92000A11DB11D8093C6119093C711A093C8116A
:10E93000B093C91184E0D4CF88E080937B0087E452
:10E9400080937C0080917A00806480937A000E949A
:10E95000C58585E0C5CF2091780030917900809100
:10E96000C2119091C311A091C411B091C511820F31
:10E97000931FA11DB11D8093C2119093C311A09349
:10E98000C411B093C51186E0ABCF0E94C58587E066
:10E99000A7CF1092CE118091C1118F5F8093C111CA
:10E9A0008091C111803108F441C0809123128111FE
:10E9B00018C08091CA119091CB119093331280931B
:10E9C00032128091C2119091C311909335128093AD
:10E9D00034128091C6119091C7119093291280939F
:10E9E000281281E0809323121092C1111092CA1153
:10E9F0001092CB111092CC111092CD111092C21125
:10EA00001092C3111092C4111092C5111092BD1131
:10EA10001092BE111092BF111092C0111092C61127
:10EA20001092C7111092C8111092C911FF91EF9165
:10EA3000BF91AF919F918F917F916F915F914F9116
:10EA40003F912F910F900BBE0F900FBE0F901F9014
:10EA500018952DEB37E346E05EE30C94CEB52DEB35
:10EA600037E346E05EE30C9400B32DEB37E346E07A
:10EA70005EE30C9400B32DEB37E346E05EE30C94C9
:10EA8000CEB510926212109263121092641210921C
:10EA9000651282E29DE9909398028093970208950F
:10EAA000109239121092381210923B1210923A12B0
:10EAB0001092371210923612E4CF10926212109216
:10EAC0006312109264121092651283EE9EE7909387
:10EAD00098028093970282E0809396020895FB014A
:10EAE000609197027091980270935B1260935A1232
:10EAF0006091621270916312709359126093581270
:10EB000062E06093960262E57CE9709398026093FC
:10EB100097029093571280935612F0935512E093F8
:10EB20005412662757FD6095762F409350125093EC
:10EB300051126093521270935312C901AA2797FD84
:10EB4000A095BA2F80934C1290934D12A0934E1221
:10EB5000B0934F1280819181AA2797FDA095BA2F7B
:10EB60008093621290936312A0936412B093651223
:10EB70000895CF93DF93262FFC01EB5BFF4F40817D
:10EB80005181EC01CD5BDF4F6881798104960E9451
:10EB90005EA728813981280F311D87FD3A95398379
:10EBA000288381E090E0DF91CF91089581E090E0AB
:10EBB0009093B2128093B11284E190E09093B412DA
:10EBC0008093B3128091F908853019F469E674E0F6
:10EBD00004C0873031F464E774E08EE692E10E946D
:10EBE00093AE81E090E09093B2128093B1128BE2E9
:10EBF00090E09093B4128093B3126FE774E08EE6C6
:10EC000092E10C9493AECF93DF93FC016491EC01FD
:10EC10002196662331F08EE692E10E9494AECE01F9
:10EC2000F4CFDF91CF910895CF92DF92EF92FF92D0
:10EC30000F931F93CF93DF931F92CDB7DEB7E62ECE
:10EC40008901F90101900020E9F7F22EFE1A92E104
:10EC5000F90E1092B2121092B11290E001965CE09F
:10EC6000589F9001599F300D11243093B412209376
:10EC7000B312642F8EE692E179830E9494AECE2C7B
:10EC80007981D72EFE0CEF2CEC18F60164916623E7
:10EC900041F08EE692E10E9494AEEFEFCE1ADE0ACA
:10ECA000F2CF6AE38EE692E10E9494AEEE2039F054
:10ECB00060E28EE692E10E9494AEEA94F7CFB8014A
:10ECC0008EE692E10F90DF91CF911F910F91FF900F
:10ECD000EF90DF90CF900C9493AE8091050991E076
:10ECE000892780930509882319F088E595E102C0FA
:10ECF00084E595E10C947E2285E08093F9081092DA
:10ED0000FA081092FB08BDDE8FEB94E10C947E2292
:10ED1000AF92BF92CF92DF92EF92FF920F931F9329
:10ED2000CF93DF931F92CDB7DEB789EFA82E88E08F
:10ED3000B82E87E0F501808380E090E0A0E0B0E4A9
:10ED40008093EB089093EC08A093ED08B093EE0845
:10ED5000198220E030E040EA50E46091380270917E
:10ED6000390280913A0290913B020E9400B39E01C9
:10ED70002F5F3F4F69017B018C012FEE38E04BEE96
:10ED800058E067EE78E083EE98E00E947148F50164
:10ED9000108289EE9AE8909398028093970282E01D
:10EDA0008093960210926212109263121092641273
:10EDB000109265128FEF92E10E947E220F90DF91F8
:10EDC000CF911F910F91FF90EF90DF90CF90BF9068
:10EDD000AF9008959F92AF92BF92CF92DF92EF9241
:10EDE000FF920F931F93CF93DF932091E3062F5F42
:10EDF0002093E3068AE0289FE001112430E080910F
:10EE0000E8069091E9062817390720F48E01065F7D
:10EE10001F4F06C00091EA061091EB060C0F1D1F54
:10EE20009CE1E92E99E0F92E2DEAC22E22E1D22EA4
:10EE300034E1932E4AE0A42EB12CC017D10778F507
:10EE40006091E4067091E506615071096C1B7D0BC1
:10EE50007093E7066093E6068BE099E00E94AF1995
:10EE6000FF92EF92DF92CF921F929F92CE01B50157
:10EE70000E94A3B6989E9001999E300D1124255EA4
:10EE8000394F3F932F930E947BBA21968DB79EB73F
:10EE900008960FB6F8949EBF0FBE8DBFCECF8AEBFB
:10EEA00090E89093980280939702109262121092C9
:10EEB00063121092641210926512DF91CF911F912C
:10EEC0000F91FF90EF90DF90CF90BF90AF909F9009
:10EED00008959F92AF92BF92CF92DF92EF92FF92EE
:10EEE0000F931F93CF93DF932091E306215020933C
:10EEF000E3068AE0289FE001112430E08091E806D3
:10EF00009091E9062817390720F48E01065F1F4FFC
:10EF100006C00091EA061091EB060C0F1D1F5CE184
:10EF2000E52E59E0F52E6AEAC62E62E1D62E74E18E
:10EF3000972EEAE0AE2EB12CC017D10778F560917C
:10EF4000E4067091E506615071096C1B7D0B7093AE
:10EF5000E7066093E6068BE099E00E94AF19FF9206
:10EF6000EF92DF92CF921F929F92CE01B5010E9445
:10EF7000A3B6989E9001999E300D1124255E394FBD
:10EF80003F932F930E947BBA21968DB79EB7089628
:10EF90000FB6F8949EBF0FBE8DBFCECF8AEB90E820
:10EFA00090939802809397021092621210926312CB
:10EFB0001092641210926512DF91CF911F910F9100
:10EFC000FF90EF90DF90CF90BF90AF909F9008950B
:10EFD000CF92DF92EF92FF920F931F93CF93DF9325
:10EFE0001F921F92CDB7DEB7D82EE62E8901C90138
:10EFF00049837A830E94E1B9F1E1FF2EF81A109259
:10F00000B2121092B112ED2DF0E031962CE02E9F4D
:10F01000C0012F9F900D11249093B4128093B312CE
:10F020004981642F8EE692E10E9494AECE2C7A81C3
:10F03000D72EFE0CEF2CEC18F6016491662341F0FC
:10F040008EE692E10E9494AE8FEFC81AD80AF2CFF2
:10F050006AE38EE692E10E9494AEEE2039F060E21F
:10F060008EE692E10E9494AEEA94F7CFC8010F9029
:10F070000F90DF91CF911F910F91FF90EF90DF9054
:10F08000CF90C1CDDF92EF92FF920F931F93CF935A
:10F09000DF93D82FF62ED72EC42FE22E61E082E721
:10F0A00092E14E3311F04632A9F40E9444A98CE05B
:10F0B000D89FA00111244D5F5F4F0CE010E020E8C5
:10F0C00030E060E070E082E792E10E949BAB60E09C
:10F0D00082E792E10E9444A91092B2121092B112FA
:10F0E0008D2F90E001962CE0289FF001299FF00DD4
:10F0F0001124F093B412E093B312CE3311F06C2FBD
:10F1000001C060E28EE692E10E9494AECF2DDD2D2B
:10F1100011E11F0D912F9C1BFE016491662331F0BC
:10F120008EE692E10E9494AE2196F4CFC92FCC23B3
:10F1300039F060E28EE692E10E9494AEC150F7CFC2
:10F140006E2D8EE692E10E9494AE60E28EE692E130
:10F150000E9494AE61E082E792E1DF91CF911F912E
:10F160000F91FF90EF90DF900C9444A9CF92DF9223
:10F17000EF92FF920F931F93CF93DF931F92CDB720
:10F18000DEB7E091FA0828E0E29FF0011124E2598D
:10F19000FD4F80819181A281B3818093E308909398
:10F1A000E408A093E508B093E60884819581A681E0
:10F1B000B7818093E7089093E808A093E908B0939B
:10F1C000EA08198220E030E040E752E46091300222
:10F1D0007091310280913202909133020E9400B30B
:10F1E0009E012F5F3F4F69017B018C012FEE38E0BC
:10F1F0004BEE58E067EE78E083EE98E00E947148AD
:10F200000E94726A1092EB081092EC081092ED08BE
:10F210001092EE08198220E030E040E251E4609163
:10F2200038027091390280913A0290913B020E941B
:10F2300000B37B018C012FEE38E04BEE58E067EE17
:10F2400078E083EE98E00E9471480E94726A0F9005
:10F25000DF91CF911F910F91FF90EF90DF90CF90B2
:10F260000895CF92DF92EF92FF920F931F93CF9367
:10F27000DF931F92CDB7DEB787E08093F90880E077
:10F2800090E0A0E0B0E48093EB089093EC08A093AA
:10F29000ED08B093EE08198220E030E040EA50E437
:10F2A000609138027091390280913A0290913B024C
:10F2B0000E9400B39E012F5F3F4F69017B018C01CB
:10F2C0002FEE38E04BEE58E067EE78E083EE98E002
:10F2D0000E947148D6DB8091FA0881508093FA0829
:10F2E000813039F48091FB08823040F41092FB08A1
:10F2F00005C0811103C084E08093FA0837DF0F90C6
:10F30000DF91CF911F910F91FF90EF90DF90CF9001
:10F310000895CF92DF92EF92FF920F931F93CF93B6
:10F32000DF931F92CDB7DEB787E08093F90880E0C6
:10F3300090E0A0E0B0E48093EB089093EC08A093F9
:10F34000ED08B093EE08198220E030E040EA50E486
:10F35000609138027091390280913A0290913B029B
:10F360000E9400B39E012F5F3F4F69017B018C011A
:10F370002FEE38E04BEE58E067EE78E083EE98E051
:10F380000E9471487EDB8091FA088F5F8093FA08B3
:10F39000853031F484E08093FB0881E08093FA08A3
:10F3A000E5DE0F90DF91CF911F910F91FF90EF90CD
:10F3B000DF90CF900895CF9382E0809396020E94D1
:10F3C0000BAC6C507E4F8F4F9F4F609368127093C1
:10F3D000691280936A1290936B12389ACAE0409A2D
:10F3E00063E070E080E090E00E943AAC409863E017
:10F3F00070E080E090E00E943AACC15081F7CF917C
:10F400000895109262121092631210926412109278
:10F41000651282E79EE79093980280939702CBCF84
:10F42000CF92DF92EF92FF920F931F93CF93DF93D0
:10F430008091621290916312A0916412B091651252
:10F4400081309048A105B10540F0109262121092EF
:10F4500063121092641210926512609162127091A0
:10F460006312809164129091651225E030E040E0D3
:10F4700050E00E94CAB680916C1290E0A0E0B0E02B
:10F48000281739074A075B0710F420936C12D091B4
:10F490006C12C0E0A5E0CA2ED12CE12CF12C11E0B9
:10F4A0006091621270916312809164129091651262
:10F4B000D11137C020919602222369F026E26530EF
:10F4C00071058105910510F446E201C040E268E44F
:10F4D00075E18C2FD7DD80916D1282FD12C020E086
:10F4E00030E040E251E460914812709149128091FD
:10F4F0004A1290914B120E94F9B287FD77C003E047
:10F50000E2C08091621290916312A0916412B09156
:10F5100065120597A105B10510F74DDF89EE9BE750
:10F520001CC1D13081F520919602222391F0A701D0
:10F5300096010E94CAB6213031054105510519F4E2
:10F540002AEF4EE302C02AEF40E261E475E18C2F1E
:10F5500099DD80916D1282FFC2CF6091621270912D
:10F5600063128091641290916512A70196010E9426
:10F57000CAB6213031054105510509F0B0CF1BDF76
:10F5800086E999E8EAC0D23009F0A9CF2091960225
:10F59000222391F0A70196010E94CAB622303105BC
:10F5A0004105510519F42AEF4EE302C02AEF40E26B
:10F5B0006AE375E18C2F66DD80916D1282FF8FCF3B
:10F5C0006091621270916312809164129091651241
:10F5D000A70196010E94CAB62230310541055105A6
:10F5E00009F07DCFE8DE8FEE98E8B7C06091621237
:10F5F000709163128091641290916512D33089F5F5
:10F6000020919602222391F0A70196010E94CAB68A
:10F61000233031054105510519F42AEF4EE302C0AC
:10F620002AEF40E263E375E18C2F2CDD80916D12AF
:10F6300082FD02C005E047C06091621270916312C2
:10F640008091641290916512A70196010E94CAB63A
:10F65000233031054105510569F7ADDE84EB97E8AC
:10F660007CC0D43039F720919602222391F0A70173
:10F6700096010E94CAB6243031054105510519F49E
:10F680002AEF4EE302C02AEF40E26AE275E18C2FD6
:10F69000F9DC80916D1282FFCDCF60916212709182
:10F6A00063128091641290916512A70196010E94E5
:10F6B000CAB6243031054105510509F0BBCF7BDEC8
:10F6C00084E798E84AC06091621270916312809159
:10F6D000641290916512A70196010E94CAB6802F0C
:10F6E00090E0A0E0B0E0281739074A075B0788F0F0
:10F6F00025E0029FC00111240197AA2797FDA0953C
:10F70000BA2F8093621290936312A0936412B09305
:10F7100065126091621270916312809164129091EF
:10F720006512A70196010E94CAB680916C1290E002
:10F730000496422F50E0841795074CF48CEF820F0B
:10F7400080936C1210939602DBEFD20FCFEFCF5F56
:10F75000DF5FC53008F4A4CE0CC09093980280936C
:10F760009702109262121092631210926412109219
:10F770006512DF91CF911F910F91FF90EF90DF9075
:10F78000CF9008958DEC9CECACECBDE380934812D7
:10F7900090934912A0934A12B0934B1241CE80E04D
:10F7A00090E0A0E8BFE38093481290934912A093A1
:10F7B0004A12B0934B1234CE80E090E0A0E2B1E464
:10F7C0008093481290934912A0934A12B0934B121F
:10F7D00027CE8F929F92AF92BF92CF92DF92EF92FD
:10F7E000FF921F93CF93DF938091621290916312E7
:10F7F000A0916412B091651281309048A105B105C5
:10F8000040F01092621210926312109264121092E1
:10F8100065126091621270916312809164129091EE
:10F82000651225E030E040E050E00E94CAB68091C9
:10F830006C1290E0A0E0B0E0281739074A075B0798
:10F8400010F420936C12D0916C12C0E0B5E0CB2E76
:10F85000D12CE12CF12C13E1812E912CA12CB12C77
:10F8600011E0609162127091631280916412909124
:10F870006512D11122C020919602222369F026E25E
:10F88000653071058105910510F446E201C040E242
:10F8900065E175E18C2FF6DB80916D1282FF2AC045
:10F8A0008091621290916312A0916412B0916512DE
:10F8B0000597A105B105F0F4D1C0D13009F045C0DC
:10F8C00020919602222391F0A70196010E94CAB6C8
:10F8D000213031054105510519F42AEF4EE302C0EC
:10F8E0002AEF40E26BE075E18C2FCCDB80916D124A
:10F8F00082FD16C08091621290916312A0916412F1
:10F90000B09165124497A105B10508F483C08092B7
:10F91000621290926312A0926412B09265127AC041
:10F9200060916212709163128091641290916512DD
:10F93000A70196010E94CAB6213031054105510543
:10F94000C9F639DD8CED9BE78CC0D23081F5209172
:10F950009602222391F0A70196010E94CAB6223096
:10F9600031054105510519F42AEF4EE302C02AEF93
:10F9700040E262E075E18C2F85DB80916D1282FFA1
:10F98000B9CF60916212709163128091641290916C
:10F990006512A70196010E94CAB6223031054105C1
:10F9A000510509F0A7CF07DD8FEC9BE75AC0D33094
:10F9B00009F0A0CF20919602222391F0A701960191
:10F9C0000E94CAB6233031054105510519F42AEFCA
:10F9D0004EE302C02AEF40E267EF74E18C2F52DB66
:10F9E00080916D1282FF86CF6091621270916312D6
:10F9F0008091641290916512A70196010E94CAB687
:10FA0000233031054105510509F074CFD4DC82EC77
:10FA10009BE727C06091621270916312809164121B
:10FA200090916512A70196010E94CAB680916C124E
:10FA300090E00496422F50E0841795074CF48CEF29
:10FA4000820F80936C1210939602DBEFD20FCFEFF0
:10FA5000CF5FDF5FC53008F404CF0FC0ACDC80EBB4
:10FA600092E99093980280939702109262121092FA
:10FA700063121092641210926512DF91CF911F9160
:10FA8000FF90EF90DF90CF90BF90AF909F908F90BE
:10FA900008958091C1129091C2129093391280936F
:10FAA000381290933B1280933A128091BF1290913A
:10FAB000C01290933712809336128091BD129091AC
:10FAC000BE129093C9088093C8080E9441750C9497
:10FAD0007C6F8091BB129091BC12909339128093ED
:10FAE000381290933B1280933A128091B912909100
:10FAF000BA1290933712809336128091B712909178
:10FB0000B8129093C9088093C8080E9441750C945C
:10FB10007C6F8BE099E00E94651A10926C12089538
:10FB20003F924F925F926F927F928F929F92AF928D
:10FB3000BF92CF92DF92EF92FF920F931F93CF93DA
:10FB4000DF9380910E09882309F4BAC08091960250
:10FB5000811104C080916D1282FFB2C08BE099E0E8
:10FB60000E94051A9093E5068093E4069093E706B9
:10FB70008093E6066AE070E00E94A3B67093E906FF
:10FB80006093E8068C019093EB068093EA06672B5E
:10FB900009F093C01092E3066FE079E08FE599E0F9
:10FBA0000E94315680910F098F32F1F41092EC06C9
:10FBB000C0E0D0E08CE1482E89E0582E9FEE692EFF
:10FBC00094E1792E24E1322E3AE0E32EF12C4FE03D
:10FBD000C42E49E0D42E5FE8A52E54E0B52E62EF86
:10FBE000862E64E1962E38C081E08093EC06E0CF4B
:10FBF0006091E4067091E506615071096C1B7D0B04
:10FC00007093E7066093E6068BE099E00E94AF19D7
:10FC100080913709882321F1DF92CF92BF92AF9272
:10FC20009F928F921F923F92CE01B7010E94A3B67E
:10FC3000389E9001399E300D1124255E394F3F9337
:10FC40002F930E947BBA8DB79EB70A960FB6F89491
:10FC50009EBF0FBE8DBF2196C017D10749F61EC0AB
:10FC60005F924F927F926F921F923F92CE01B701A7
:10FC70000E94A3B6389E9001399E300D1124255E56
:10FC8000394F3F932F930E947BBA8DB79EB708964A
:10FC90000FB6F8949EBF0FBE8DBFDDCF8AEB90E804
:10FCA00090939802809397021092621210926312BE
:10FCB000109264121092651203C00AE010E06ACF3D
:10FCC000DF91CF911F910F91FF90EF90DF90CF9038
:10FCD000BF90AF909F908F907F906F905F904F906C
:10FCE0003F900895CF93DF93C1E0D0E0D093B2125C
:10FCF000C093B11289E090E09093B4128093B31254
:10FD000061E974E08EE692E10E9493AED093B21264
:10FD1000C093B11286E190E09093B4128093B31235
:10FD200060EA74E08EE692E10E9493AE6BEA74E0C2
:10FD30008EE692E10E9493AED093B212C093B112BC
:10FD400083E290E09093B4128093B31260EB74E07E
:10FD50008EE692E10E9493AED093B212C093B1129C
:10FD600080E390E09093B4128093B31262EC74E05D
:10FD70008EE692E10E9493AED093B212C093B1127C
:10FD80008DE390E09093B4128093B31268ED74E029
:10FD90008EE692E10E9493AE80916D1282FF10C0B8
:10FDA0008091FD08882319F080E490E902C080EB7F
:10FDB00092E99093980280939702DF91CF91FBCACA
:10FDC000DF91CF910895EF92FF920F931F93CF93FE
:10FDD000DF93C1E0D0E0D093B212C093B11289E0BA
:10FDE00090E09093B4128093B31264EE74E08EE6C8
:10FDF00092E10E9493AED093B212C093B11283E10C
:10FE000090E09093B4128093B31260EF74E08EE6AA
:10FE100092E10E9493AED093B212C093B1128DE1E1
:10FE200090E09093B4128093B31265E075E08EE693
:10FE300092E10E9493AE75EEE72E70E2F72E00E29B
:10FE400010E024E030E04EE150E060E370E082E753
:10FE500092E10E94EDA380916D1282FF17C081E0B4
:10FE60008093FD08109205098BE08093F90889EED4
:10FE70009AE890939802809397029DDA109262120A
:10FE8000109263121092641210926512DF91CF915A
:10FE90001F910F91FF90EF900895CF92DF92EF9214
:10FEA000FF920F931F93CF93DF9388E090E090939E
:10FEB000B2128093B1128DE090E09093B4128093CF
:10FEC000B31268E175E08EE692E10E9493AE8091F4
:10FED000FA08823038F08091FB08823018F481E013
:10FEE0008093FB088091621290916312A09164123A
:10FEF000B091651281309048A105B10540F0109293
:10FF00006212109263121092641210926512609144
:10FF1000621270916312809164129091651225E0D3
:10FF200030E040E050E00E94CAB680916C1290E050
:10FF3000A0E0B0E0281739074A075B0710F42093C8
:10FF40006C12D0916C12C2E0E5E0CE2ED12CE12CE7
:10FF5000F12C11E0DD2371F02091FB086091621219
:10FF6000709163128091641290916512211134C0D6
:10FF700001E061C0809196028823A1F08091621215
:10FF800090916312A0916412B091651220E20597DE
:10FF9000A105B10510F44EE301C040E26FE073E14A
:10FFA0008C2F70D880916D1282FFD6CF8091621213
:10FFB00090916312A0916412B09165120597A1050A
:10FFC000B10550F6F8D9DF91CF911F910F91FF90B5
:10FFD000EF90DF90CF909DC9D13061F520919602CE
:10FFE000222391F0A70196010E94CAB62130310563
:10FFF0004105510519F420E24EE302C020E240E23F
:020000021000EC
:100000006AE073E18C2F3ED880916D1282FF49C067
:1000100060916212709163128091641290916512E6
:10002000A70196010E94CAB621303105410551054C
:10003000C1F58BC002E00D1335C02091960222233A
:10004000B1F0A70196010E94CAB6802F90E0A0E00F
:10005000B0E0281739074A075B0719F420E24EE39E
:1000600002C020E240E263E073E18C2F0BD8809164
:100070006D1282FF17C060916212709163128091BD
:10008000641290916512A70196010E94CAB6802F52
:1000900090E0A0E0B0E0281739074A075B0711F4A9
:1000A0005EC002E00F5F60916212709163128091F6
:1000B000641290916512A70196010E94CAB6802F22
:1000C00090E0A0E0B0E0281739074A075B0788F006
:1000D00025E0029FC00111240197AA2797FDA09552
:1000E000BA2F8093621290936312A0936412B0931C
:1000F0006512609162127091631280916412909106
:100100006512A70196010E94CAB680916C1290E018
:100110000496422F50E0841795074CF48CEF820F21
:1001200080936C1210939602DBEFD20FCFEFCF5F6C
:10013000DF5FC53008F40ECFDF91CF911F910F9193
:10014000FF90EF90DF90CF90089535D9DF91CF9158
:100150001F910F91FF90EF90DF90CF9082C82BD925
:10016000DF91CF911F910F91FF90EF90DF90CF9093
:100170000C9488762F923F924F925F926F927F926B
:100180008F929F92AF92BF92CF92DF92EF92FF92A7
:100190000F931F93CF93DF93CDB7DEB7A9970FB619
:1001A000F894DEBF0FBECDBF80919602811104C0CE
:1001B00080916D1282FF6BC32091E3063AE0239F8A
:1001C000F0011124FAA3E9A330E08091E8069091B0
:1001D000E9062817390738F429A13AA1265F3F4FCD
:1001E00038A32F8F0AC08091EA069091EB06E9A10F
:1001F000FAA1E80FF91FF8A3EF8F80916212909196
:100200006312A0916412B091651281309048A105EB
:10021000B10540F0109262121092631210926412B3
:100220001092651260916212709163128091641253
:100230009091651225E030E040E050E00E94CAB69F
:1002400080916C1290E0A0E0B0E0281739074A07CF
:100250005B0710F420936C1220906C12312CA5E0F7
:10026000CA2ED12CE12CF12C8091E306811132C0F1
:10027000222031F08091EC0681115CC011E05EC05B
:10028000809196028823A9F0809162129091631266
:10029000A0916412B091651226E20597A105B105FF
:1002A00010F446E201C040E265ED72E1832D0E9448
:1002B000427880916D1282FFDDCF80916212909121
:1002C0006312A0916412B09165120597A105B10562
:1002D00088F6CDC22110CECF809196028823A9F056
:1002E0008091621290916312A0916412B091651294
:1002F00020E20597A105B10510F44EE301C040E2EC
:100300006CEC72E1832D0E94427880916D1282FF25
:10031000B1CF8091621290916312A0916412B0915A
:1003200065120597A105B10508F0A4CF44D80E9435
:100330006977ADC221E0221619F112E03CE0339E4C
:10034000C0011124FC013396FCA3EBA39C01245FA4
:100350003F4F3EA32DA3832D90E001962CE0289FD4
:10036000F001299FF00D1124F8A7EFA389A09AA00E
:1003700031E0320D39A7422C512C612C712C4AC02E
:10038000809196028823D9F0609162127091631275
:100390008091641290916512A70196010E94CAB6DD
:1003A000213031054105510519F420E24EE302C028
:1003B00020E240E269EC72E1832D0E944278809154
:1003C0006D1282FFBACF60916212709163128091B8
:1003D000641290916512A70196010E94CAB621305D
:1003E00031054105510509F0A8CF0E94DB7991DB69
:1003F0004EC28091E4069091E5060197881999090B
:100400009093E7068093E606121551F01F5FFFEF09
:100410008F1A9F0A2F8D38A18216930650F305C1BB
:1004200080919602882309F49DC0609162127091B8
:1004300063128091641290916512A70196010E9447
:10044000CAB6C4016AE070E02415350546055705B3
:1004500009F054C00E94A3B644E1489F5001499F4F
:10046000B00C1124C501855E994F5C01FC018081AF
:100470008111138A61E082E792E10E9444A90CE0B5
:1004800010E020E830E04BA15CA160E070E082E782
:1004900092E10E949BAB60E082E792E10E9444A956
:1004A0001092B2121092B1122DA13EA13093B4124B
:1004B0002093B31260E28EE692E10E9494AE850131
:1004C00033E1A30E8A2D801BF80161918F01662311
:1004D00029F08EE692E10E9494AEF4CF182F1123FA
:1004E00039F060E28EE692E10E9494AE1150F7CFAF
:1004F00061E082E792E10E9444A934C00E94A3B661
:10050000F4E1F89F8001F99F100D1124055E194F49
:10051000F80180818111138A1092B2121092B112E7
:100520002FA138A53093B4122093B31260E28EE667
:1005300092E10E9494AE58010D5E102F1A19F50138
:1005400061915F01662329F08EE692E10E9494AEEC
:10055000F4CF112339F060E28EE692E10E9494AE6E
:100560001150F7CF80916D1282FF7AC160916212B3
:10057000709163128091641290916512A7019601A7
:100580000E94CAB6241535054605570509F068C10D
:100590000E94DB791092F6066091E6068BE099E006
:1005A0000E94AF198FE099E09F938F9383EA92E1C5
:1005B0009F938F938E010F5F1F4F1F930F930E9486
:1005C000B7BAECE1F9E00F900F900F900F900F90F9
:1005D0000F908191882339F09091C00095FFFCCF56
:1005E0008093C600F6CF8091C00085FFFCCF8AE0E3
:1005F0008093C6007E01F5E0EF0EF11CF7018081CB
:10060000882349F0992787FD90950E94D2B9F70178
:1006100081937F01F3CFC8010E940B228FE992E101
:100620000E947E220E94417532C14091E80650919D
:10063000E9062091EA063091EB0660916212709112
:10064000631280916412909165124115510509F46D
:1006500062C02115310509F45EC02091E30630E047
:1006600024173507C0F5121176C020919602222377
:10067000B9F0A70196010E94CAB6812F90E0A0E0D0
:10068000B0E0281739074A075B0719F420E24EE368
:1006900002C020E240E26FEB72E1832D0E944278BB
:1006A00080916D1282FF57C0609162127091631247
:1006B0008091641290916512A70196010E94CAB6BA
:1006C000812F90E0A0E0B0E0281739074A075B07C8
:1006D00009F041C0C7C02417350709F073C01211D3
:1006E0003AC020919602222309F452C0A701960134
:1006F0000E94CAB6812F90E0A0E0B0E02817390729
:100700004A075B0719F426E246E202C026E240E20D
:100710006AEB72E13AC026303105D8F012111BC0E5
:10072000209196022223A1F1A70196010E94CAB648
:10073000812F90E0A0E0B0E0281739074A075B0757
:1007400019F426E246E202C026E240E265EB72E1DD
:100750001CC0121511F01F5F35C020919602222394
:10076000B9F0A70196010E94CAB6812F90E0A0E0DF
:10077000B0E0281739074A075B0719F426E246E27A
:1007800002C026E240E260EB72E1832D0E944278D3
:1007900080916D1282FFDFCF6091621270916312BF
:1007A0008091641290916512A70196010E94CAB6C9
:1007B000812F90E0A0E0B0E0281739074A075B07D7
:1007C00051F655C06091621270916312809164126B
:1007D00090916512A70196010E94CAB6812F90E000
:1007E000A0E0B0E0281739074A075B0788F035E03A
:1007F000139FC00111240197AA2797FDA095BA2F36
:100800008093621290936312A0936412B093651266
:1008100060916212709163128091641290916512DE
:10082000A70196010E94CAB680916C1290E00496CE
:10083000422F50E08417950764F48CEF820F809369
:100840006C1241E040939602FBEF2F2E220E3324D0
:100850003A943394239484E0831508F005CD17C0AF
:1008600019A5D5CD0E94DB790E94EA7610C00E94BE
:10087000DB7989EE9AE89093980280939702109220
:100880006212109263121092641210926512A9966D
:100890000FB6F894DEBF0FBECDBFDF91CF911F9191
:1008A0000F91FF90EF90DF90CF90BF90AF909F900F
:1008B0008F907F906F905F904F903F902F90089512
:1008C000CF93DF93FC01E95BFF4F2081EC0124967D
:1008D000211105C081E08083CE010E94E4A8CE01F1
:1008E000DF91CF910C9417A9EF92FF920F931F9372
:1008F00061E081E40E94D9AD61E081E40E9412AE22
:100900008EE692E1DDDF6AE378E182E792E10E9420
:10091000D1A761E082E792E10E9444A9009174129C
:1009200010917512209172123091731240E050E0D4
:1009300060E070E082E792E10E949BAB61E082E7B9
:1009400092E10E9444A982E792E10E941BA98111D1
:10095000DACF8EE692E1B4DFB5EAEB2EBCE1FB2EF6
:1009600000E410E020E130E040E050E060E070E0C2
:1009700082E792E10E94EDA382E792E10E941BA927
:100980008111EACF1F910F91FF90EF900895AF92E0
:10099000BF92CF92DF92EF92FF920F931F93CF936C
:1009A000DF935C01EB011EE6C12E12E1D12EF601B0
:1009B000268137812552310901EBE02E02E1F02E2C
:1009C000F7011182108203EB12E1F80131832083D9
:1009D0006AE378E182E792E10E94D1A7C5010E9413
:1009E00003766AE3C6010E9494AEF6018681978180
:1009F0008597FE0101900020E9F79F012150310900
:100A00002C1B3D0B67EF6203A001639F500D112467
:100A10009A0122583F4FF70131832083F8019183D7
:100A20008083BE01C601DF91CF911F910F91FF908E
:100A3000EF90DF90CF90BF90AF900C9493AE209149
:100A4000B61221110AC044E150E0BC0189E992E0EC
:100A50000E946CBA82E08093960208952091B612AB
:100A600021110AC044E150E0BC0189E992E00E94F2
:100A700002BA82E0809396020895CF93DF9310929A
:100A80000D098BE099E00E949A190E94E86A83EEB2
:100A900094E10E947E228091F606882329F010922C
:100AA000F60681E0809306028091E30E8823F9F038
:100AB0001092E30EC091CA08D0E0CC0FDD1FC85CD5
:100AC000DD4E68817981882777FD8095982F0E9477
:100AD0009BB3209148023091490240914A025091C3
:100AE0004B020E94FCB4181614F4198218828FED80
:100AF00094E10E947E220E94417585ED94E1AEDF73
:100B00000E940BAC6093F7067093F8068093F90689
:100B10009093FA0681E08093F908DF91CF910895D0
:100B20008091000980FD16C092E09093F9089091A1
:100B3000FF08992341F087FF06C01092000980ED5D
:100B400094E10E947E228BE099E00E94B81483EC2D
:100B500094E184CF08958BE099E00E94BF1483E074
:100B60008093F9088091000980FF03C082EE92E132
:100B700002C08AED92E172CF71DF81E08093B612FC
:100B80000C9441751092B6120895CF92DF92EF92B5
:100B9000FF92CF93C6B1C6FBCC27C0F981E0C8272E
:100BA000349BC260C0906812D0906912E0906A12C3
:100BB000F0906B120E940BACC616D706E806F90639
:100BC00010F4329B39C0C0936D1280916D12817008
:100BD00090916D1291FD826090916712891721F1B9
:100BE0008130F1F028F0823089F08330A1F01CC010
:100BF000913021F4909166129F5F05C09230A1F46C
:100C0000909166129150909366120EC0992391F3C1
:100C1000933051F4F5CF923069F3913029F4F0CF4D
:100C2000933041F3992361F380936712CF91FF9042
:100C3000EF90DF90CF900895C460C5CF55DE60E09F
:100C40008FE10E94D9AD60E081E20E94D9AD60E001
:100C500081E30E94D9AD469A449A60E083E20E9403
:100C6000D9AD429A9FB7F894EBE0F1E080818160C2
:100C700080839FBF8091090180958170809361126C
:100C800084DF109266120895CF92DF92EF92FF9266
:100C9000CF93DF937ADF80910901817091E08927FA
:100CA000209161128217E1F082E080939602809198
:100CB0000901817089278093611216DE809161128B
:100CC000882339F08BE099E00E94EF1381E992E1EB
:100CD00006C08BE099E00E94B41484E892E1BEDE85
:100CE000C0905D12D0905E12E0905F12F0906012A2
:100CF0000E940BACC616D706E806F90608F0C3C07A
:100D000040916612442361F181E080939602552759
:100D100047FD5095652F752F809162129091631257
:100D2000A0916412B0916512840F951FA61FB71F82
:100D30008093621290936312A0936412B093651231
:100D4000109266120E940BAC6856754C8F4F9F4FE5
:100D500060933C1270933D1280933E1290933F1229
:100D600080916D1282FF0EC00E940BAC6856754CCC
:100D70008F4F9F4F60933C1270933D1280933E12B1
:100D800090933F128091C3128F5F8093C3128EE6BF
:100D900092E196DDCDE7D0E06AE378E182E792E187
:100DA0000E94D1A7D093B212C093B1121092B41284
:100DB0001092B3128091C31280FF02C061E001C0A3
:100DC00060E082E792E10E9444A94FE350E06FE7C0
:100DD00070E082E792E10E9429A961E082E792E156
:100DE0000E9444A9E0919702F09198021995809190
:100DF0009602811107C08091F9089BEF980F9430FB
:100E000068F007C082E792E10E941BA98111C4CF5C
:100E1000F2CFC1E08C3018F4C0E001C0C1E0C09056
:100E20003C12D0903D12E0903E12F0903F120E9492
:100E30000BACC616D706E806F90648F4809197026F
:100E40009091980282529D4911F0CC23B1F080918B
:100E50009602882319F08150809396020E940BAC71
:100E60006C597F4F8F4F9F4F60935D1270935E124E
:100E700080935F129093601206C00E94417582E0D9
:100E800080939602E4CFDF91CF91FF90EF90DF90B7
:100E9000CF90089580916D1282FB882780F9089584
:100EA000FC01808190E02AE030E0B9010E94B7B6F1
:100EB000482FCB01B9010E94B7B6805D80934012E4
:100EC000405D409341121092421280E492E10895F5
:100ED00020E030E040E251E4FC01608171818281D8
:100EE00093810E94CEB50E9468B377FD02C02BE2C9
:100EF00001C02DE2209340129B0177FF04C02227FE
:100F00003327261B370BC90168EE73E00E94B7B682
:100F1000CB01EAE0F0E0BF010E94B7B6805D8093AC
:100F20004112C90164E670E00E94B7B6CB01BF016F
:100F30000E94B7B6805D80934212C901BF010E9432
:100F4000B7B6282FCB01BF010E94B7B6805D809352
:100F500043128EE280934412205D2093451210923A
:100F6000461280E492E10895CF92DF92EF92FF92D1
:100F70000F931F938091621290916312A09164125B
:100F8000B09165120097A105B10509F480C02091C8
:100F9000FD08BC01882777FD8095982F213039F412
:100FA0000E949BB32DEC3CEC4CEC5DE30AC00E942C
:100FB0009BB3209148123091491240914A125091AE
:100FC0004B120E94CEB59B01AC016091EB08709171
:100FD000EC088091ED089091EE080E9420B2609399
:100FE000EB087093EC088093ED089093EE0820E0F6
:100FF00030E0A9016091EB087091EC088091ED0858
:101000009091EE080E94F9B287FF08C01092EB0899
:101010001092EC081092ED081092EE0820E030E0FB
:1010200048EC53E46091EB087091EC088091ED0876
:101030009091EE080E94FCB4181664F480E090E0F1
:10104000A8ECB3E48093EB089093EC08A093ED0830
:10105000B093EE0810926212109263121092641212
:10106000109265129AECC92E98E0D92EE12CF12C41
:1010700000E712E42FEE38E04BEE58E067EE78E040
:1010800083EE98E00E94714881E0809396028091FF
:101090009602882339F08BEE98E01ADFBC0182E5D6
:1010A00095E175DC80916D1282FF17C00E94DB799B
:1010B0008091FD08813019F480E490E902C080E15C
:1010C0009AE790939802809397021092621210927E
:1010D000631210926412109265121F910F91FF908B
:1010E000EF90DF90CF900895CF92DF92EF92FF9232
:1010F0000F931F938091621290916312A0916412DA
:10110000B09165120097A105B10509F442C0BC0178
:10111000882777FD8095982F0E949BB320914812D5
:101120003091491240914A1250914B120E94CEB513
:101130009B01AC016091EF087091F0088091F1087B
:101140009091F2080E9420B26093EF087093F0082B
:101150008093F1089093F208109262121092631239
:1011600010926412109265123AECC32E38E0D32E1E
:10117000E12CF12C00EA11E42FEE38E04BEE58E0C0
:1011800067EE78E083EE98E00E94714881E08093FA
:10119000960280919602882339F08FEE98E098DECF
:1011A000BC0181E295E1F3DB80916D1282FF10C0FA
:1011B0000E94DB7980E19AE79093980280939702EE
:1011C00010926212109263121092641210926512C1
:1011D0001F910F91FF90EF90DF90CF900895CF92E5
:1011E000DF92EF92FF920F931F9380916212909182
:1011F0006312A0916412B09165120097A105B10528
:1012000009F46EC0BC01882777FD8095982F0E9455
:101210009BB3209148123091491240914A1250914B
:101220004B120E94CEB52091E7083091E80840911A
:10123000E9085091EA080E9420B26B017C0120E08D
:1012400030E0A9010E94F9B287FD09C0C092E70809
:10125000D092E808E092E908F092EA0808C01092FB
:10126000E7081092E8081092E9081092EA0820E0D6
:1012700030E048EC53E46091E7087091E808809111
:10128000E9089091EA080E94FCB4181664F480E022
:1012900090E0A8ECB3E48093E7089093E808A0936B
:1012A000E908B093EA081092621210926312109249
:1012B0006412109265125AECC52E58E0D52EE12C1E
:1012C000F12C06E114E42FEE38E04BEE58E067EE27
:1012D00078E083EE98E00E94714881E08093960266
:1012E00080919602882339F087EE98E0F1DDBC0109
:1012F0008FE195E14CDB80916D1282FF10C00E945E
:10130000DB7980E19AE7909398028093970210929C
:1013100062121092631210926412109265121F9161
:101320000F91FF90EF90DF90CF900895CF92DF92D2
:10133000EF92FF920F931F9380916212909163122C
:10134000A0916412B09165120097A105B10509F44E
:101350006EC0BC01882777FD8095982F0E949BB3B3
:10136000209148123091491240914A1250914B12EB
:101370000E94CEB52091E3083091E4084091E50841
:101380005091E6080E9420B26B017C0120E030E021
:10139000A9010E94F9B287FD09C0C092E308D0926A
:1013A000E408E092E508F092E60808C01092E3082D
:1013B0001092E4081092E5081092E60820E030E070
:1013C0004DEC53E46091E3087091E4088091E508E6
:1013D0009091E6080E94FCB4181664F480E090E056
:1013E000ADECB3E48093E3089093E408A093E508A0
:1013F000B093E60810926212109263121092641277
:10140000109265127AECC72E78E0D72EE12CF12CE1
:1014100006E114E42FEE38E04BEE58E067EE78E09A
:1014200083EE98E00E94714881E08093960280915B
:101430009602882339F083EE98E04ADDBC018DE105
:1014400095E1A5DA80916D1282FF10C00E94DB79D0
:1014500080E19AE79093980280939702109262122B
:101460001092631210926412109265121F910F91E4
:10147000FF90EF90DF90CF90089520E030E040E2C1
:1014800051E4FC0160817181828193810E94CEB51B
:101490000E9468B3FB0177FD2FC0CB0168EE73E0BB
:1014A0000E94B7B6CB012AE030E0B9010E94B7B67E
:1014B000805D80934012CF0164E670E00E94B7B671
:1014C000CB01B9010E94B7B6805D80934112CF0174
:1014D000B9010E94B7B6482FCB01B9010E94B7B637
:1014E000805D809342128EE280934312405D409370
:1014F00044121092451235C02DE220934012EE277F
:10150000FF27E61BF70BCF0168EE73E00E94B7B62A
:10151000CB012AE030E0B9010E94B7B6805D80932C
:101520004112CF0164E670E00E94B7B6CB01B90169
:101530000E94B7B6805D80934212CF01B9010E942C
:10154000B7B6482FCB01B9010E94B7B6805D809332
:1015500043128EE280934412405D409345121092F4
:10156000461280E492E10895FC01808191818436E5
:1015700091055CF064E670E00E94B7B6CB016AE0CA
:1015800070E00E94B7B6805D01C080E28093401297
:10159000808191818A3091055CF02AE030E0B901C8
:1015A0000E94B7B6CB01B9010E94B7B6805D01C0F9
:1015B00080E280934112808191816AE070E00E9414
:1015C000B7B6805D809342121092431280E492E19C
:1015D0000895CF92DF92EF92FF920F931F93CF93D4
:1015E000DF938091F908813011F41092F90880910D
:1015F000621290916312A0916412B09165128130D1
:101600009048A105B10540F0109262121092631249
:1016100010926412109265126091621270916312BE
:10162000809164129091651225E030E040E050E036
:101630000E94CAB680916C1290E0A0E0B0E028173A
:1016400039074A075B0710F420936C12D0916C1293
:10165000C0E011E0A5E0CA2ED12CE12CF12CDD2355
:1016600069F02091FD08609162127091631280917F
:10167000641290916512222379F136C2809196020C
:101680008823A9F08091621290916312A091641254
:10169000B091651226E20597A105B10510F446E266
:1016A00001C040E268EE76E18C2F0E944278809182
:1016B0006D1282FFD6CF8091621290916312A09139
:1016C0006412B09165120597A105B10550F60E940C
:1016D000DB7982E29DE9BFC42091F90822502230D3
:1016E00008F07BC0D13099F520919602222399F021
:1016F000A70196010E94CAB6213031054105510566
:1017000019F42AEF4EE302C02AEF40E263EE76E1DD
:101710008C2F0E94427880916D1282FD02C003E0FE
:1017200001C1609162127091631280916412909174
:101730006512A70196010E94CAB621303105410504
:10174000510569F70E94DB7987E39AE984C4D230B6
:1017500031F720919602222309F1A70196010E94F8
:10176000CAB68091FF08223031054105510549F480
:10177000882319F025ED36E102C021ED36E14EE374
:1017800008C0882319F02DEC36E102C029EC36E1BF
:1017900040E269ED76E18C2F0E94E87780916D122E
:1017A00082FFBDCF609162127091631280916412CA
:1017B00090916512A70196010E94CAB622303105A8
:1017C0004105510509F0ABCF0E94DB798091FF08FC
:1017D00091E089278093FF084AC4D13099F5209180
:1017E0009602222399F0A70196010E94CAB62130E1
:1017F00031054105510519F42AEF4EE302C02AEFE5
:1018000040E261EC76E18C2F0E94427880916D126B
:1018100082FD02C004E086C0609162127091631282
:101820008091641290916512A70196010E94CAB638
:10183000213031054105510569F70E94DB7980EBC4
:1018400092E909C4D23091F520919602222399F0B1
:10185000A70196010E94CAB6223031054105510503
:1018600019F420E24EE302C020E240E268EB76E1A8
:101870008C2F0E94427880916D1282FFCBCF6091B5
:101880006212709163128091641290916512A701A7
:1018900096010E94CAB6223031054105510509F072
:1018A000B9CF0E94DB7984EB96E1C7C3D33009F04E
:1018B000B1CF20919602222399F0A70196010E94B0
:1018C000CAB6233031054105510519F420E24EE333
:1018D00002C020E240E265EA76E18C2F0E94427865
:1018E00080916D1282FF96CF6091621270916312A7
:1018F0008091641290916512A70196010E94CAB668
:10190000233031054105510509F084CF0E94DB7970
:10191000DF91CF911F910F91FF90EF90DF90CF90CB
:101920000C947C7620910E09609162127091631282
:101930008091641290916512222309F4B9C020911C
:10194000E209222309F498C020910D092223B9F15C
:101950000D1337C0209196022223B9F0A7019601FA
:101960000E94CAB6802F90E0A0E0B0E028173907A7
:101970004A075B0719F420E24EE302C020E240E28E
:1019800069E976E18C2F0E94427880916D1282FF86
:1019900018C06091621270916312809164129091EC
:1019A0006512A70196010E94CAB6802F90E0A0E0C0
:1019B000B0E0281739074A075B0719F410C30D1761
:1019C00021F00F5F0D137EC235C0209196022223B5
:1019D000B9F0A70196010E94CAB6802F90E0A0E05E
:1019E000B0E0281739074A075B0719F420E24EE3F5
:1019F00002C020E240E26CE876E18C2F0E9442783F
:101A000080916D1282FFDDCF60916212709163123E
:101A10008091641290916512A70196010E94CAB646
:101A2000802F90E0A0E0B0E0281739074A075B0755
:101A300041F6E1C280919602882309F4F0C16091D9
:101A40006212709163128091641290916512A701E5
:101A500096010E94CAB6802F90E0A0E0B0E028175F
:101A600039074A075B0719F420E24EE302C020E27F
:101A700040E261E876E1D0C10D1324C220919602C4
:101A8000222309F403C2A70196010E94CAB6802F3F
:101A900090E0A0E0B0E0281739074A075B0719F487
:101AA0002AEF4EE302C02AEF40E26EE676E1EBC198
:101AB0000D1308C220919602222309F420C2A70127
:101AC00096010E94CAB6802F90E0A0E0B0E02817EF
:101AD00039074A075B0719F420E24EE302C020E20F
:101AE00040E266E676E108C2213009F02DC220917D
:101AF000F9082250223008F03FC0D13011F002E046
:101B0000E3C0209196022223B9F0A70196010E941A
:101B1000CAB68EE292E0213031054105510521F42B
:101B200023DD9C014EE303C01FDD9C0140E260E623
:101B300076E18C2F0E94147680916D1282FFDFCFA8
:101B4000609162127091631280916412909165129B
:101B5000A70196010E94CAB6213031054105510501
:101B600071F60E94DB7927EE33E04AE050E06EE246
:101B700072E08AE596E157C2D13099F5209196023C
:101B8000222399F0A70196010E94CAB6213031059F
:101B90004105510519F42AEF4EE302C02AEF40E255
:101BA0006BE476E18C2F0E94427880916D1282FD69
:101BB00002C004E089C0609162127091631280914A
:101BC000641290916512A70196010E94CAB6213055
:101BD00031054105510569F70E94DB7980E490E900
:101BE0003AC2D230E1F5209196022223B9F0A70142
:101BF00096010E94CAB682E099E022303105410583
:101C0000510521F4B1DC9C014EE303C0ADDC9C0125
